:020000040800F2
:10780000000011002200330044005500660077009C
:1078100088009900AA00BB00CC00DD00EE00FF004C
:020000040800F2
:10800000A8520020FD0501083104010833040108CD
:10801000370401083B0401083F0401080000000088
:108020000000000000000000000000004304010800
:108030004504010800000000470401084904010844
:108040001706010817060108170601081706010898
:108050001706010817060108170601081706010888
:108060001706010817060108170601081706010878
:108070001706010817060108170601081706010868
:108080001706010817060108170601081706010858
:10809000170601081706010817060108118A0008CB
:1080A0001706010817060108170601081706010838
:1080B000A989000817060108437204081706010879
:1080C0001706010817060108170601081706010818
:1080D0001706010817060108170601081706010808
:1080E0005D8A00081706010817060108170601082F
:1080F00017060108170601081706010817060108E8
:1081000017060108170601081706010817060108D7
:10811000137104085B6202081706010817060108BC
:10812000170601081706010817060108F79200084C
:10813000DFF80CD03FF0ACFE004800479581000806
:10814000A8520020EFF30980704780F30988704738
:10815000EFF30880704780F30888704740BA704793
:10816000C0BA70474FF0010080F3138801480249FC
:108170000160FEE70CED00E00400FA054FF001009D
:1081800080F31388014802490160FEE70CED00E02E
:108190000400FA05A248A34908600BF044FC3DE145
:1081A00000F053FE6DE00EF07EF94FF400619E4842
:1081B00008F0CCFD08B9012000E00020044622466A
:1081C0004FF40061984808F0D2FD56E09748407996
:1081D000012852D19648007C01284ED100209349B5
:1081E000487100F043FE4FF400618F4808F0AEFD87
:1081F00008B9012000E00020044622464FF4006147
:10820000894808F0B4FD01F0A9FF17F021FC17F030
:10821000E9FC1DF0A7FC1DF0D1FC1AF0F6FA19F0EC
:1082200074FD00F023FE4FF400617F4808F08EFDDE
:1082300008B9012000E00020044622464FF4006106
:10824000794808F094FD0CF0D7FD07F0D3F81EF044
:1082500023FB3AF05BFF0EF014FB13F0F6F813F07B
:1082600014FA3CF027FB0DF077FC16F01BFB0CF02A
:10827000D7FE11F0F4FC0CF06EFD6D48007801287B
:10828000A4D06B48007801288DD08DE00EF07BF9EA
:108290004FF40061644808F059FD08B9012000E07E
:1082A0000020044622464FF400615F4808F05FFD5D
:1082B00076E05E484079012872D15D48007C002854
:1082C0006ED15A49487100F08EFD00F0CFFD4FF499
:1082D0000061554808F03AFD08B9012000E000208F
:1082E000044622464FF400614F4808F040FD01F07B
:1082F00035FF17F077FC4F4991F8551061B14D49A2
:1083000091F8551001290CD14949088E00EBD07124
:108310004910A0EB410121B91DF082FC01201DF0A4
:10832000AAFC1AF072FA19F0F0FC07F063F800F0FA
:108330009DFD4FF400613C4808F008FD08B901209C
:1083400000E00020044622464FF40061364808F061
:108350000EFD1EF0A1FA3AF0D9FE0EF092FA0CF0E2
:108360001CFD13F072F83CF0A5FA0DF0F5FB16F0C9
:1083700099FA2F48007C012801D02D4840790CF053
:108380004FFE11F06CFC0CF0E6FC0EF030F838B942
:1083900012F0A0FD012108460AF03CFB00F034FB7E
:1083A00023480078022884D02148007802283FF42E
:1083B0006DAF21E00DF0EAFF18E00CF01DFD0A2082
:1083C00000F079F80EF05FF800F050FD4FF4006116
:1083D000154808F0BBFC08B9012000E00020044665
:1083E00022464FF40061104808F0C1FC10480078A4
:1083F0000328E2D00DF0D5FF0D4800780328D9D02E
:1084000008E003E012F090FC16F0A6FA08480078A5
:108410000428F7D0064800780428F2D0C0E600000F
:108420000080000808ED00E0000801400400002082
:10843000A21600204224002010B5042008F03FF9C5
:108440002F48006800EB400080002E49B0FBF1F09F
:108450002D4908700846007800EB4001C1EBC010C0
:108460004FF6FF7101EAC0002849088010BD01469F
:10847000254A12784A434FF0E0235A6100229A615C
:108480001A46126942F001021A6100BF4FF0E02261
:10849000106900F001021AB100F48032002AF5D010
:1084A0004FF0E022126922F001024FF0E0231A613E
:1084B00000229A6170470146144A12884A434FF0DD
:1084C000E0235A6100229A611A46126942F00102C1
:1084D0001A6100BF4FF0E022106900F001021AB1EA
:1084E00000F48032002AF5D04FF0E022126922F029
:1084F00001024FF0E0231A6100229A6170470000E8
:1085000030000020001BB700000000200200002007
:1085100008B50121202008F035FE4FF4E050ADF8F9
:10852000000010208DF8030003208DF8020069463A
:108530003D4808F06BFB08BD10B5002404E00120A5
:10854000FFF795FF601CC4B2042CF8DB10BD2DE9C9
:10855000FC5F834658463FF01AFB05460022334B2A
:108560003FF028FB01D2DFF8C8B0324958463FF04F
:1085700077FB01D2DFF8BCB058463FF008FB074656
:108580002D4A2E4B3FF040F905462D4A2D4B3FF02A
:1085900094F8CDE900013FF03DFB8346254958465C
:1085A0003FF05EFB01D2DFF88CB058463FF0EFFAA7
:1085B00000221E4BCDE900013FF020F90546224A7A
:1085C000224B3FF093F907463FF08BFA814609F5BD
:1085D000605A002411E000201D490860C4F1100019
:1085E0002AFA00F01B49C1F8A801FFF7A5FF0120F6
:1085F00017490860FFF7A0FF641C112CEBD3002083
:10860000134908601349C1F8A801FFF795FF01203D
:108610000F49091D0860FFF78FFF00200D49C1F8C1
:10862000B001BDE8FC9F00000014014000000C40B8
:10863000000060400000C041A01A2FDD2406F03F7A
:108640007F87A2409FC8933F74479CA1FAFF2F3FAA
:10865000AC8122420080224210B586B0044601213E
:108660004FF4047008F08EFD4FF4004008F0EEFC6B
:108670000820ADF8000000208DF8030003208DF8DD
:1086800002006946A64808F0C1FA002001908DF862
:1086900008008DF809004FF460200390002004903A
:1086A0000D208DF8140001A99E4808F04EF8012C09
:1086B00002D1012008F006FA01219A4808F071F869
:1086C000984808F090F800BF964808F091F8002804
:1086D000FAD1944808F096F800BF924808F097F84D
:1086E0000028FAD106B010BD38B5044600214FF479
:1086F000007008F047FD012C02D1002008F0E2F9DB
:10870000884807F0FBFF0021864808F04AF8082057
:10871000ADF8000000208DF8030003208DF8020062
:1087200069467F4808F072FA38BD70B504460523E3
:10873000012221467B4808F0A0F80121794808F081
:1087400070F800BF0221774808F0DCF90028F9D062
:10875000744808F0F9F80546284670BD10B50121A7
:10876000704808F05EF800BF02216E4808F0CAF9B0
:108770000028F9D06B4808F0E7F810BD2DE9F04764
:108780008CB08246894600254846FFF765FF0024E5
:108790000AE05046FFF7C9FF01A921F8140001A81B
:1087A00030F814000544641C142CF2D34846FFF73B
:1087B0009BFFBDF80870BDF80880032410E001A8F5
:1087C00030F81400B84202D201A830F8147001A8A1
:1087D00030F81400404502D901A830F81480641C18
:1087E000132CECD30025022604E001A830F8160073
:1087F0000544761C132EF8D3E81BA0EB08050F20C8
:10880000B5FBF0F5A8B20CB0BDE8F0872DE9F04754
:10881000AEB0804600202B90FFF71EFF00251DE024
:10882000D8F8001031F815003FF0EEF802AA02EB7C
:10883000C50203C22B983FF0E7F8CDE9000102A87A
:1088400000EBC500D0E90063324600983EF035FFEA
:1088500081463FF046F92B90681C85B2142DDFDB72
:108860002B983FF0D1F8064600222F4B3FF03EF800
:10887000CDE92C0100202B90DDE92C013FF0CAF955
:108880000646DDE92C013FF0C5F90746DDE9022186
:1088900010463FF0BFF98146DDE9042110463FF064
:1088A000B9F9824633463A46494616F008F9022499
:1088B00025E002A800EBC400D0E9002110463FF0FB
:1088C000A9F9074616F005F906463FF060F902AA35
:1088D00002EBC40203C22B983FF096F8814602A82F
:1088E00000EBC400D0E90063324648463EF0E5FEA6
:1088F000CDE900013FF0F5F82B90601C84B2142CF8
:10890000D7DB2B983FF080F806460022074B3EF05D
:10891000EDFFCDE92C01DDE92C012EB0BDE8F0879B
:1089200000100140002401400000344000003240AB
:1089300010B501217C2008F025FC0121084608F033
:1089400021FC0121C80308F02AFC0121880408F059
:1089500026FC0121084608F008FC0121102008F03F
:1089600011FC0121C80408F01AFC0121880308F059
:1089700009FC0121080508F005FC10BD38B50446C6
:108980001C208DF8000001208DF801008DF80200F8
:10899000012C02D18DF8030002E000208DF80300C5
:1089A000684607F042FE38BD10B50121880709F07E
:1089B0004AFB50B10121880709F056FB0020FE490F
:1089C0008871FE490860FFF7D9FF10BD10B54FF45C
:1089D000803008F089FA08F0C6FA0446012C10D15C
:1089E000002008F006FBA00208F00CFBA00208F033
:1089F00012FB012008F0EFFA00BF08F0F5FA042896
:108A0000FBD1FFF795FF10BD10B5FFF7DFFF10BDDD
:108A100010B540200AF098FBF8B140200AF0A5FB01
:108A2000FFF7F2FF06F02AFBE548006858B90A2074
:108A3000FFF741FDE248006878B90120E149087379
:108A40000220487309E00A20FFF735FDDC48006882
:108A5000012802D1DB490873487310BD10B54FF4EB
:108A600000400AF071FBA0B14FF400400AF07DFB1A
:108A7000D5488078012802D1D349487102E001200D
:108A8000D1494871D148D0F80500401CCF49C1F800
:108A900005004FF400600AF057FB30B14FF400605E
:108AA0000AF063FB0120CA49887410BD3EB5044634
:108AB0004FF0804008F0CEFB0121084608F06FFB24
:108AC0006000401E80B2ADF8040041F26F70ADF856
:108AD00000000020ADF80600ADF8020069464FF036
:108AE000804008F08BFC0121880709F0A9FA0122D7
:108AF0001146900708F0F9FF0120FFF73FFF012121
:108B0000880708F0D7FF3EBD0EB54FF4E06007F0D0
:108B100087FD28208DF8080000208DF809008DF8C9
:108B20000A0001208DF80B0002A807F07EFD0F213E
:108B3000042008F081F94FF40040009000208DF8E7
:108B400004000C208DF8050001208DF80600684611
:108B50000AF094FA0EBD0EB54FF4E06007F060FD28
:108B600028208DF8080000208DF809008DF80B00F2
:108B700002A807F05AFD0F21042008F05DF94FF418
:108B80000040009000208DF804000C208DF80500B6
:108B900000208DF8060068460AF070FA0EBD0EB58A
:108BA00017208DF8080001208DF8090000208DF8AD
:108BB0000A0001208DF80B0002A807F036FD0621FF
:108BC000022008F039F94020009000208DF80400C0
:108BD00010208DF8050001208DF8060068460AF087
:108BE0004DFA0EBD0EB54FF4A06007F019FD172029
:108BF0008DF8080001208DF8090000208DF80A008A
:108C00008DF80B0002A807F010FD0621022008F0E5
:108C100013F94020009000208DF804000C208DF8FE
:108C2000050000208DF8060068460AF027FA0EBD00
:108C30000EB528208DF8080001208DF809008DF868
:108C40000A008DF80B0002A807F0EFFC0B210220B0
:108C500008F0F2F84FF40060009000208DF8040056
:108C60000C208DF8050001208DF8060068460AF0FA
:108C700005FA0EBD0EB54FF4A06007F0D1FC282018
:108C80008DF8080001208DF809008DF80A000020F9
:108C90008DF80B0002A807F0C8FC0B21022008F099
:108CA000CBF84FF40060009000208DF804000820FD
:108CB0008DF8050000208DF8060068460AF0DEF900
:108CC0000EBD10B580200AF03FFA044614B1802092
:108CD0000AF04BFA10BD10B5044607F0A3FBFFF7EE
:108CE00013FFFFF75CFFFFF7A3FF002080F310885E
:108CF00000BF10BD10B504462046FFF7D7FE012087
:108D00002E49086010BD10B501217C2008F03AFA08
:108D10000121084608F036FA11F0F6FF4FF4006121
:108D20002C4808F013F808B9012000E000200446A0
:108D300022464FF40061274808F019F811F0C9FCE9
:108D400011F0F8FC11F014FD06F07AF900201C492E
:108D50006831086011F081FF11F056FE11F0A3FF99
:108D600000201D49C1F8940111F08BFF0020144927
:108D70006C31086011F08CFE12F058F811F06AFCAA
:108D800011F00FFE11F0BAFE11F0C3FD11F0C9FE93
:108D900011F0F7FE21F08DFB00201049C1F884018D
:108DA00006F06CF9FFF7B4FB3AF058FC3AF05CFCC3
:108DB0003AF07AFC14E00000A2160020BC812242A6
:108DC00018012242F60F0020040000205F1A002044
:108DD000D9470020000801400000224200802242C2
:108DE00012F05BF810BD10B501217C2008F0CAF923
:108DF0000121084608F0C6F911F086FF4FF4006122
:108E00001C4807F0A3FF08B9012000E00020044639
:108E100022464FF40061174807F0A9FF11F01DFF2B
:108E200012F004F811F0F0FD10BD10B50121C803D7
:108E300008F0B5F90121084608F0A4F901210E480F
:108E400007F0B5FF00F08AFA10BD10B545F2555095
:108E50000AF094F905200AF094F94FF4EA700AF048
:108E600093F90AF094F90AF097F910BD10B50AF0D9
:108E70008EF910BD000801400002300030B587B007
:108E800004460D46444808F0E5F90121042008F0A5
:108E900086F90121084608F075F90121080307F059
:108EA00086FF601E80B2ADF81400681E80B2ADF877
:108EB00010000020ADF81600ADF8120004A93648E5
:108EC00008F09CFA6020ADF800000120ADF8020027
:108ED000204604EBD071C1F34F01ADF8061002201B
:108EE000ADF8080069462C4808F007FB08212A481D
:108EF00008F019FF0121284808F0DCFE012126486E
:108F000008F0D8FD07B030BD30B587B005460C4637
:108F1000224808F09FF90121022008F040F90121C0
:108F2000084608F02FF901211D4807F040FF4FF4D3
:108F30007A70ADF8140040F6B830ADF810004FF478
:108F40000070ADF816000020ADF8120004A9134817
:108F500008F054FA7020ADF800000120ADF80200CE
:108F6000ADF806400020ADF8080069460B4808F04F
:108F7000C4FA0821094808F0D6FE0821074809F07C
:108F800009F80621054809F017F80121034808F0FF
:108F900091FD07B030BD0000000800400004004013
:108FA00000081A0070B50024012528E080214C48F3
:108FB00007F0BFFE06464FF48071494807F0B9FE3E
:108FC00046EA00264FF40071454807F0B2FE46EA33
:108FD00000440120FFF76FFA8021414807F0A9FE05
:108FE00006464FF480713E4807F0A3FE46EA00268D
:108FF0004FF400713A4807F09CFE46EA0045AC4247
:10900000D4D1204670BD70B5002401250CE00121AB
:10901000344807F08EFE04460120FFF74CFA012188
:10902000304807F086FE0546AC42F0D1204670BDC0
:109030001CB50721022007F0FFFE802000900020D1
:109040008DF804000C208DF8050000208DF8060036
:1090500068460AF013F81CBD1CB50721022007F072
:10906000EBFE8020009000208DF804000C208DF88D
:10907000050000208DF80600684609F0FFFF1CBDC2
:109080001FB58020ADF8000048208DF80300694628
:10909000134807F0BBFD4FF4E06007F0C1FA17205A
:1090A0008DF8040001208DF805008DF806008DF87C
:1090B000070001A807F0B9FA0721022007F0BCFE5B
:1090C0008020029000208DF80C000C208DF80D00FF
:1090D00001208DF80E0002A809F0D0FF1FBD00008E
:1090E00000100140000C014010B590B00446012171
:1090F000880308F047F80121084608F036F80C9478
:109100000020ADF83400ADF83600ADF83800ADF809
:109110003C000C20ADF83A000CA9204809F071F988
:1091200001211E4809F0F9F91D4809F02BFB1B48E5
:10913000001D01901B48029000200390C82004905D
:1091400000200590802006900020079008902020A5
:10915000099000020A9000200B9001A9104809F024
:10916000B3FB012240210D4809F008FA01210C4807
:1091700009F0D5FB10B010BD10B5044600BF40216A
:10918000064809F0A5FA0028F9D04021034809F063
:10919000ACFA2146014809F02DFA10BD0038014013
:1091A00058000240EC09002010B590B0044601219F
:1091B000482007F0E7FF0121880407F0F0FF0121B4
:1091C000084607F0D2FF0C940020ADF83400ADF84B
:1091D0003600ADF83800ADF83C000C20ADF83A0090
:1091E0000CA9584809F00DF90121564809F095F9E4
:1091F000002055490860554809F0C4FA5148001D3F
:10920000019053480290002003904FF46170049045
:1092100000200590802006900020079008902020D4
:1092200009904FF440500A9000200B9001A9474844
:1092300009F04AFB01224021424809F09FF901212F
:10924000424809F06CFB10B010BD30B58BB005463C
:109250000C463E48143809F095FA3A48001D009033
:109260000195102002900394002004908020059026
:1092700000200690079008904FF4005009900020BD
:109280000A9069463148143809F01EFB01228021FA
:109290002C4809F073F90BB030BD70B505460E4689
:1092A00001202949086000240CE000BF4021254826
:1092B00009F00EFA0028F9D0295D224809F09AF940
:1092C000601C84B2B442F0DB00BF40211D4809F0AD
:1092D000FFF90028F9D000201B49086070BD10B5C7
:1092E0000346002000BF03E00C5C1C54441CE0B2A9
:1092F0009042F9DB10BD10B5164809F03FFB002184
:109300001248143809F00BFB4FF49670FFF7AFF8D2
:1093100000200D49086010BD70B5044601200A49BF
:10932000086020463EF0DEF8C5B229462046FFF729
:10933000B4FF0120FFF7BFF800200749C1F88801FA
:1093400070BD000000480040880123423000024008
:109350007E0B0020000002100000234200B585B003
:109360000020ADF800004FF48270ADF8020000203C
:10937000ADF80400ADF80600ADF808004FF4007039
:10938000ADF80A000020ADF80C00ADF80E00072083
:10939000ADF810006946534808F090FE012151488D
:1093A00008F031FF05B000BD70B505460E4600243B
:1093B00005E0601CC4B2C82C01DD002070BD022194
:1093C000284608F0A4FF0028F3D03146284608F0CC
:1093D0004BFF002405E0601CC4B2C82C01DD002056
:1093E000ECE70121284608F092FF0028F3D0284638
:1093F00008F03CFFC0B2E1E770B50546002405E087
:10940000601CC4B2C82C01DD002070BD02213648AA
:1094100008F07DFF0028F3D02946334808F024FFE8
:10942000002405E0601CC4B2C82C01DD0020ECE77C
:1094300001212D4808F06BFF0028F3D02A4808F0DE
:1094400015FFC0B2E1E770B50546002405E0601CD9
:10945000C4B2C82C01DD002070BD0221214808F0F3
:1094600056FF0028F3D029461E4808F0FDFE0024D0
:1094700005E0601CC4B2C82C01DD0020ECE701212E
:10948000184808F044FF0028F3D0164808F0EEFE14
:10949000C0B2E1E770B50546002405E0601CC4B227
:1094A000C82C01DD002070BD0221104808F02FFFFC
:1094B0000028F3D029460D4808F0D6FE002405E028
:1094C000601CC4B2FF2C01DD0020ECE7012107483D
:1094D00008F01DFF0028F3D0044808F0C7FEC0B212
:1094E000E1E70000003C004000300140003800404F
:1094F00010B50A20FEF7BBFFF9480078012808D014
:109500008021F84807F031FC8021F74807F02BFC58
:1095100007E08021F44807F028FC8021F14807F09B
:1095200022FC0520FFF78FFFFF20FFF78CFF04468A
:109530008021EC4807F017FC8021EB4807F013FC72
:10954000204610BD10B500BFFFF7D2FF00F00100AC
:109550000028F9D110BD70B506460D462C46E048EE
:109560000078012808D08021DE4807F0FEFB80212A
:10957000DD4807F0F8FB07E08021DB4807F0F5FB4A
:109580008021D84807F0EFFB0620FFF75CFF802121
:10959000D44807F0E8FB8021D34807F0E4FBD0482B
:1095A0000078012808D08021CE4807F0DEFB80211A
:1095B000CD4807F0D8FB07E08021CB4807F0D5FB6A
:1095C0008021C84807F0CFFB0220FFF73CFFC4F31F
:1095D0000740FFF738FFC4F30720FFF734FFE0B27E
:1095E000FFF731FF3046FFF72EFF8021BD4807F01F
:1095F000BAFB8021BC4807F0B6FBFFF7A3FF70BDA4
:1096000070B505462C46B6480078012808D0802160
:10961000B44807F0AAFB8021B34807F0A4FB07E099
:109620008021B14807F0A1FB8021AE4807F09BFBE9
:109630000320FFF708FFC4F30740FFF704FFC4F35C
:109640000720FFF700FFE0B2FFF7FDFEFF20FFF766
:10965000FAFE06468021A34807F085FB8021A24838
:1096600007F081FB304670BD10B504469C48007879
:10967000012808D080219B4807F077FB80219A4879
:1096800007F071FB07E08021974807F06EFB80210F
:10969000944807F068FB0620FFF7D5FE802191482B
:1096A00007F061FB8021904807F05DFB8C48007853
:1096B000012808D080218B4807F057FB80218A4879
:1096C00007F051FB07E08021874807F04EFB80211F
:1096D000844807F048FB0120FFF7B5FE2046FFF75E
:1096E000B2FE80217F4807F03EFB80217E4807F0D4
:1096F0003AFB10BD10B50A20FEF7B9FE7848007895
:10970000012808D08021774807F02FFB8021764878
:1097100007F029FB07E08021734807F026FB802132
:10972000704807F020FBB920FFF78DFE80216D48BF
:1097300007F019FB80216C4807F015FB10BD70B5D0
:1097400005460A20FEF793FE65480078012808D0F8
:109750008021644807F009FB8021634807F003FB80
:1097600007E08021604807F000FB80215D4807F09A
:10977000FAFA9F20FFF767FE002405E0FF20FFF7BD
:1097800062FE2855601CC4B2092CF7DB80215548C5
:1097900007F0E9FA8021544807F0E5FA70BD38B5C2
:1097A00004462046FFF72CFF8DF80000601CFFF7F1
:1097B00027FF8DF80100A01CFFF722FF8DF80200A3
:1097C000E01CFFF71DFF8DF80300009838BD2DE960
:1097D000F74F82B082469046B8F57A6F03DD0020DD
:1097E00005B0BDE8F08FD1464FF0000B039C464614
:1097F0006EB1012000EB1425C4EB0520B04201D36B
:10980000374601E0C4EB05274FF0010B01E04FF0B4
:10981000000B74E032480078012808D080213148DC
:1098200007F0A3FA8021304807F09DFA07E0802175
:109830002D4807F09AFA80212A4807F094FA06206A
:10984000FFF701FE8021274807F08DFA8021264886
:1098500007F089FA22480078012808D080212148A1
:1098600007F083FA8021204807F07DFA07E0802185
:109870001D4807F07AFA80211A4807F074FA02208E
:10988000FFF7E1FDC4F30740FFF7DDFDC4F3072058
:10989000FFF7D9FDE0B2FFF7D6FD0020019007E009
:1098A00019F8010BFFF7CFFD0198401C80B2019021
:1098B0000198B842F4D380210A4807F054FA802175
:1098C000094807F050FA3C44F61BA6B1012000EB12
:1098D0001425C4EB0520B04208D3374608E0000049
:1098E0000A00002000140140000C0140C4EB0527D1
:1098F0004FF0010B01E04FF0000BFFF723FEBBF12F
:10990000000F87D100206BE738B504460D4600955F
:10991000042221466846FFF75AFF38BD1CB50446AD
:109920002046FFF76DFE8DF80000601CFFF768FE13
:109930008DF80100A01CFFF763FE8DF80200E01C0B
:10994000FFF75EFE8DF80300201DFFF759FE8DF82E
:109950000400601DFFF754FE8DF80500A01DFFF701
:109960004FFE8DF80600E01DFFF74AFE8DF8070058
:109970009DF80000FF281ED19DF80100FF281AD194
:109980009DF80200FF2816D19DF80300FF2812D190
:109990009DF80400FF280ED19DF80500FF280AD18C
:1099A0009DF80600FF2806D19DF80700FF2802D188
:1099B000002100910191DDE900011CBD7CB5064646
:1099C00014461D46CDE90045082231466846FFF79A
:1099D000FEFE7CBD38B504462046FFF711FE8DF82B
:1099E0000000601CFFF70CFE8DF80100A01CFFF7C3
:1099F00007FE8DF80200E01CFFF702FE8DF8030061
:109A0000009838BD38B504460D460095042221461D
:109A10006846FFF7DCFE38BD38B504462046FFF740
:109A2000EFFD8DF80000601CFFF7EAFD8DF80100E6
:109A3000BDF8000038BD38B504460D460095022239
:109A400021466846FFF7C3FE38BD2DE9F0410646C2
:109A50000C46174634480078012808D08021334846
:109A600007F083F98021324807F07DF907E0802173
:109A70002F4807F07AF980212C4807F074F9032069
:109A8000FFF7E1FCC4F30740FFF7DDFCC4F3072058
:109A9000FFF7D9FCE0B2FFF7D6FC002505E0FF2078
:109AA000FFF7D1FC7055681C85B2BD42F7DB802101
:109AB0001E4807F058F980211D4807F054F9FFF7B8
:109AC00041FDBDE8F08170B504460D461646012003
:109AD00015490870324629462046FFF778FE0020D7
:109AE0001149087070BD70B504460D461646012038
:109AF0000D490870324629462046FFF7A6FF002090
:109B00000949087070BDADF5007D002000BF06E07A
:109B100040AA105400210DF80010411C88B2FF2803
:109B2000F6DD00BFFEE700000A000020001401403F
:109B3000000C014070B50346A1F16400142590FBB0
:109B4000F5F503F10A0000EB400606EB001005EB0B
:109B5000800452F8240070BD2DE9F04780460E467F
:109B600017463F4940463EF07BF801D228250BE0DE
:109B70003C4940463EF06AF802D26FF0090503E026
:109B800040463DF062FF0546374930463EF068F8F2
:109B900002D24FF4C8640AE0344930463EF056F829
:109BA00001D2642403E030463DF04FFF0446012F0C
:109BB00004D0022F09D0032F15D10DE02C4A2146E5
:109BC0002846FFF7B7FF814614E02A4A2146284677
:109BD000FFF7B0FF81460DE0274A21462846FFF7F0
:109BE000A9FF814606E0224A21462846FFF7A2FF48
:109BF000814600BF00BF4846BDE8F0872DE9FF4F12
:109C000087B08A46934650463DF0C1FF80464FF0EC
:109C100066321A4B3DF051FD04460D4658463DF064
:109C2000B6FF064622462B463DF060FECDE9020116
:109C300007983DF0ACFF0446114A124B3DF0E4FD9D
:109C4000CDE90001DDE902233DF0DEFDCDE90401AF
:109C50003DF0E0FF069006980BB0BDE8F08F0000E5
:109C600000002042000020C10000C8440000C8429B
:109C7000A48F040834CC0408C40805086612714097
:109C8000FA74B4FB3325074010B5FE48006820F095
:109C90007060FC4908600846006840F04070086049
:109CA0000120F9490860F949C1F8B8010A20FEF716
:109CB000DEFB0020F449091D08600A20FEF7D7FBEF
:109CC0000020F249C1F8B4010A20FEF7D0FB10BD14
:109CD00010B5EC48006820F07060EA49086008465A
:109CE000006840F0407008600020E749091D0860E6
:109CF0000A20FEF7BCFB0120E449C1F8B4010A20A8
:109D0000FEF7B5FB0120E049091D0860002404E0CE
:109D10000A20FEF7ACFB601CC4B2052CF8DB10BDBA
:109D200010B50024D748006820F07060D54908605D
:109D30000846006840F0006008600A20FEF797FBC4
:109D40000A20FEF794FB07E0601CC4B2FA2C03DD86
:109D5000FFF7BEFF012010BDCB487C38006800280B
:109D6000F2D1C949086000BFF5E710B5C5480068E1
:109D700020F07060C34908600846006840F04070F9
:109D800008600020C049091D08600A20FEF76FFB2B
:109D90000120BE49C1F8B4010A20FEF768FB00208B
:109DA000B94908600A20FEF762FB10BD10B5B5483E
:109DB000006820F07060B34908600846006840F011
:109DC000407008600120B049091D08600A20FEF7B4
:109DD0004EFB0120AD49C1F8B4010A20FEF747FB54
:109DE0000020A94908600A20FEF741FB10BD70B5AC
:109DF0000446A448006820F07060A2490860084644
:109E0000006840F04070086000251CE004F080000D
:109E100020B101209C49091D086003E000209A49F7
:109E2000091D08606006040E0A20FEF720FB0120D1
:109E3000954908600A20FEF71AFB00209349C1F8F3
:109E4000B401681CC5B2082DE0DB0A20FEF70FFB49
:109E500001208D4908600A20FEF709FB00208B498C
:109E6000C1F8B40170BD70B506460024854800688D
:109E700020F07060834908600846006840F0006088
:109E80000860002515E001207F4908600A20FEF7E0
:109E9000EEFA6006040E7D48D0F8380108B144F0AF
:109EA00001040020784908600A20FEF7E0FA681CE7
:109EB000C5B2082DE7DB7348006820F07060714977
:109EC00008600846006840F040700860204670BD99
:109ED0002DE9F04107460D461646FFF7D5FE6420F2
:109EE000FFF785FF3846FFF782FFFFF7CDFE6520BD
:109EF000FFF77DFF002407E00120FFF7B4FF28559E
:109F0000FFF733FF601CC4B2701EA042F4DC0020D7
:109F1000FFF7A9FF2855FFF749FFFFF7D9FEBDE876
:109F2000F0812DE9F04107460D461646FFF7ACFEDD
:109F30006420FFF75CFF3846FFF759FF002404E078
:109F4000285DFFF754FF601CC4B2B442F8DBFFF792
:109F5000BFFEBDE8F0811CB500208DF800008DF833
:109F6000010002208DF8020000208DF8030060201F
:109F70008DF80400052269460B20FFF7D2FF1CBDB7
:109F80002DE9FC4704460D4616461F46DDE90B9AAF
:109F9000DDF828800A209AFBF0F100FB11A00A21CD
:109FA0009AFBF1F140EA0110C0B28DF800000A20DE
:109FB00099FBF0F100FB11900A2199FBF1F140EAC5
:109FC0000110C0B28DF801000A2098FBF0F100FBEF
:109FD00011800A2198FBF1F140EA0110C0B28DF81E
:109FE00002008DF803700A2096FBF0F100FB11606F
:109FF0000A2196FBF1F140EA0110C0B28DF804008D
:10A000000A2095FBF0F100FB11500A2195FBF1F1BC
:10A0100040EA0110C0B28DF805000A2094FBF0F16F
:10A0200000FB11400A2194FBF1F140EA0110C0B29B
:10A030008DF80600072269460020FFF772FFBDE891
:10A04000FC872DE9FC4704460D4616461F46DDE910
:10A050000B9ADDF82880642094FBF0F100FB11409E
:10A0600084B20A209AFBF0F100FB11A00A219AFBAE
:10A07000F1F140EA0110C0B28DF800000A2099FB0E
:10A08000F0F105E004180140B4012342000023422E
:10A0900000FB11900A2199FBF1F140EA0110C0B2D6
:10A0A0008DF801000A2098FBF0F100FB11800A21D5
:10A0B00098FBF1F140EA0110C0B28DF802008DF872
:10A0C00003700A2096FBF0F100FB11600A2196FB59
:10A0D000F1F140EA0110C0B28DF804000A2095FBAE
:10A0E000F0F100FB11500A2195FBF1F140EA01105B
:10A0F000C0B28DF805000A2094FBF0F100FB11407E
:10A100000A2194FBF1F140EA0110C0B28DF806007B
:10A11000072269460020FFF704FFBDE8FC872DE910
:10A12000FC4704460D4616461F46DDE90B9ADDF84E
:10A1300028808DF800A08DF801908DF802808DF8B0
:10A1400003708DF804608DF805508DF806400722E5
:10A1500069460020FFF7E5FEBDE8FC8710B5072241
:10A1600038490020FFF7B4FE364880793649087038
:10A170003448407948703348007988703148807895
:10A18000C8703048407808712E48007848712D48D2
:10A19000007800F00F002B490978090901EB8101D3
:10A1A00000EB4100294988702648407800F00F00F4
:10A1B00024494978090901EB810100EB4100234959
:10A1C00048702048807800F00F001E4989780909FE
:10A1D00001EB810100EB41001C4908701948C0786F
:10A1E00048711848007900F00F00164909790909EB
:10A1F00001EB810100EB41001449087111484079DD
:10A2000000F00F000F494979090901EB810100EBCA
:10A2100041000E49C8700B488079000900EB8000AE
:10A220004FF4FA6101EB40000649897901F00F0112
:10A2300008440649C88010BD03E04FF45E70FEF785
:10A240003AF9FAE71A000020140000200C00002060
:10A2500010B5FB48006820F00F00F9490860084677
:10A26000006840F0030008600120F6490860F649E4
:10A27000C1F8A0010A20FEF7FAF80020F149091FF1
:10A2800008600A20FEF7F3F80020EF49C1F8A401A6
:10A290000A20FEF7ECF810BD10B5E948006820F080
:10A2A0000F00E74908600846006840F003000860B6
:10A2B0000020E449091F08600A20FEF7D8F80120B1
:10A2C000E149C1F8A4010A20FEF7D1F80120DD49D7
:10A2D000091F0860002404E00A20FEF7C8F8601C8B
:10A2E000C4B2052CF8DB10BD10B50024D4480068BA
:10A2F00020F00F00D24908600846006840F00800CE
:10A3000008600A20FEF7B3F80A20FEF7B0F807E06D
:10A31000601CC4B2FA2C03DDFFF7BEFF012010BDA4
:10A32000C848843800680028F2D1C649086000BFD8
:10A33000F5E710B5C248006820F00F00C04908607A
:10A340000846006840F0030008600020BD49091F6E
:10A3500008600A20FEF78BF80120BB49C1F8A40170
:10A360000A20FEF784F80020B64908600A20FEF7AC
:10A370007EF810BD10B5B248006820F00F00B0495B
:10A3800008600846006840F0030008600120AD49FD
:10A39000091F08600A20FEF76AF80120AA49C1F8DF
:10A3A000A4010A20FEF763F80020A64908600A20ED
:10A3B000FEF75DF810BD70B50446A148006820F0B6
:10A3C0000F009F4908600846006840F003000860DD
:10A3D00000251CE004F0800020B101209949091FEC
:10A3E000086003E000209749091F08606006040E1A
:10A3F0000A20FEF73CF80120924908600A20FEF787
:10A4000036F800209049C1F8A401681CC5B2082D97
:10A41000E0DB0A20FEF72BF801208A4908600A20B9
:10A42000FEF725F800208849C1F8A40170BD70B579
:10A43000064600248248006820F00F00804908602A
:10A440000846006840F008000860002515E001207B
:10A450007C4908600A20FEF70AF86006040E7A4874
:10A46000D0F8200108B144F00104002075490860CB
:10A470000A20FDF7FCFF681CC5B2082DE7DB704819
:10A48000006820F00F006E4908600846006840F040
:10A4900003000860204670BD2DE9F04107460D46D7
:10A4A0001646FFF7D5FE7C20FFF785FF3846FFF7FD
:10A4B00082FFFFF7CDFE7D20FFF77DFF002407E040
:10A4C0000120FFF7B4FF2855FFF733FF601CC4B22B
:10A4D000701EA042F4DC0020FFF7A9FF2855FFF70B
:10A4E00049FFFFF7D9FEBDE8F0812DE9F0410746AD
:10A4F0000D461646FFF7ACFE7C20FFF75CFF3846A2
:10A50000FFF759FF002404E0285DFFF754FF601CAB
:10A51000C4B2B442F8DBFFF7BFFEBDE8F0812DE91D
:10A52000F04107460D461646FFF792FE7C20FFF7E6
:10A5300042FF8020FFF73FFF3846FFF73CFF002433
:10A5400004E0285DFFF737FF601CC4B2B442F8DBBB
:10A55000FFF7A2FEBDE8F081704710B50446232244
:10A5600021460020FFF7DBFF10BD10B5002404E0FA
:10A57000002036490855601CC4B2232CF8DB334850
:10A58000FFF7EBFF10BD08B50220FDF794FF032095
:10A590008DF80000012269468220FFF7A6FF08BD62
:10A5A00010B501202A490860FFF7EDFFFFF7DDFF36
:10A5B00010BD70B504460D46164632462146284663
:10A5C000FFF76AFF70BD002004E000211F4A11540C
:10A5D000411CC8B22328F8DB704730B5C31700EB25
:10A5E0005373DB10194CE35C0246C41700EB547440
:10A5F000E410A0EBC4050124AC4023430146C4177A
:10A6000000EB5474E410114D2B5530BD30B5C31719
:10A6100000EB5373DB100D4CE35C0246C41700EBF8
:10A620005474E410A0EBC4050124AC40A3430146DC
:10A63000C41700EB5474E410044D2B5530BD0000DA
:10A64000040C0140A481214200802142D20F00204D
:10A650008C01234230B505460C46152D82F08082D0
:10A66000DFE815F07E121500FF00E801D102BA0301
:10A67000A3048C058A0673075C0845092E0A170B8C
:10A68000000C080DF10DDA0EC30FAC1095110A2C59
:10A6900074D2DFE804F0051B31475D748AA0B6CCA4
:10A6A0000F20FFF79AFF1720FFF797FF1520FFF7FE
:10A6B00094FF0C20FFF791FF0D20FFF78EFF0E2077
:10A6C000FFF78BFF1620FFF7A1FFC7E00F20FFF772
:10A6D0009DFF1720FFF781FF1520FFF77EFF0C205D
:10A6E000FFF794FF0D20FFF791FF0E20FFF78EFF7D
:10A6F0001620FFF78BFFB1E00F20FFF76EFF17204A
:10A70000FFF76BFF1520FFF781FF0C20FFF765FFB8
:10A710000D20FFF762FF0E20FFF778FF1620FFF7EE
:10A720005CFF9BE00F20FFF758FF1720FFF755FF56
:10A730001520FFF752FF0C20FFF74FFF0D20FFF70A
:10A7400065FF0E20FFF762FF1620FFF746FF85E04A
:10A750000F20FFF75BFF1720FFF73FFF1520FFF7E4
:10A760003CFF0C20FFF752FF0D20FFF74FFF0E209C
:10A77000FFF733FF1620FFF730FF6FE06DE00F208B
:10A78000FFF72BFF1720FFF741FF1520FFF725FFED
:10A790000C20FFF722FF0D20FFF738FF0E20FFF7F8
:10A7A0001CFF1620FFF719FF58E00F20FFF715FFD9
:10A7B0001720FFF72BFF1520FFF70FFF0C20FFF7E7
:10A7C0000CFF0D20FFF709FF0E20FFF706FF1620F4
:10A7D000FFF703FF42E00F20FFF7FFFE1720FFF710
:10A7E000FCFE1520FFF7F9FE0C20FFF70FFF0D20F0
:10A7F000FFF70CFF0E20FFF709FF1620FFF706FFFB
:10A800002CE00F20FFF7E9FE1720FFF7E6FE1520EA
:10A81000FFF7E3FE0C20FFF7E0FE0D20FFF7DDFE63
:10A820000E20FFF7DAFE1620FFF7D7FE16E00F2006
:10A83000FFF7D3FE1720FFF7D0FE1520FFF7CDFE60
:10A840000C20FFF7CAFE0D20FFF7E0FE0E20FFF7F9
:10A85000C4FE1620FFF7C1FE00E000BF00BF02F0FB
:10A860007FB90A2C74D2DFE804F0051B31475D7410
:10A870008AA0B6CC1F20FFF7B0FE3E20FFF7ADFE4A
:10A880003D20FFF7AAFE1C20FFF7A7FE1420FFF7CC
:10A89000A4FE1E20FFF7A1FE1D20FFF7B7FEC7E0B4
:10A8A0001F20FFF7B3FE3E20FFF797FE3D20FFF786
:10A8B00094FE1C20FFF7AAFE1420FFF7A7FE1E201F
:10A8C000FFF7A4FE1D20FFF7A1FEB1E01F20FFF758
:10A8D00084FE3E20FFF781FE3D20FFF797FE1C20FF
:10A8E000FFF77BFE1420FFF778FE1E20FFF78EFE99
:10A8F0001D20FFF772FE9BE01F20FFF76EFE3E203B
:10A90000FFF76BFE3D20FFF768FE1C20FFF765FE9A
:10A910001420FFF77BFE1E20FFF778FE1D20FFF7B7
:10A920005CFE85E01F20FFF771FE3E20FFF755FE1D
:10A930003D20FFF752FE1C20FFF768FE1420FFF7B2
:10A9400065FE1E20FFF749FE1D20FFF746FE6FE063
:10A950006DE01F20FFF741FE3E20FFF757FE3D2030
:10A96000FFF73BFE1C20FFF738FE1420FFF74EFEDA
:10A970001E20FFF732FE1D20FFF72FFE58E01F209C
:10A98000FFF72BFE3E20FFF741FE3D20FFF725FE9F
:10A990001C20FFF722FE1420FFF71FFE1E20FFF7EA
:10A9A0001CFE1D20FFF719FE42E01F20FFF715FED9
:10A9B0003E20FFF712FE3D20FFF70FFE1C20FFF7A1
:10A9C00025FE1420FFF722FE1E20FFF71FFE1D208C
:10A9D000FFF71CFE2CE01F20FFF7FFFD3E20FFF7D6
:10A9E000FCFD3D20FFF7F9FD1C20FFF7F6FD1420CC
:10A9F000FFF7F3FD1E20FFF7F0FD1D20FFF7EDFD33
:10AA000016E01F20FFF7E9FD3E20FFF7E6FD3D20A1
:10AA1000FFF7E3FD1C20FFF7E0FD1420FFF7F6FD34
:10AA20001E20FFF7DAFD1D20FFF7D7FD00E000BF75
:10AA300000BF14E70A2C74D2DFE804F0051B31478D
:10AA40005D748AA0B6CC5F20FFF7C7FD5E20FFF7DC
:10AA5000C4FD5D20FFF7C1FD5C20FFF7BEFD542063
:10AA6000FFF7BBFD5620FFF7B8FD5520FFF7CEFDE1
:10AA7000C7E05F20FFF7CAFD5E20FFF7AEFD5D2057
:10AA8000FFF7ABFD5C20FFF7C1FD5420FFF7BEFDD3
:10AA90005620FFF7BBFD5520FFF7B8FDB1E05F2062
:10AAA000FFF79BFD5E20FFF798FD5D20FFF7AEFDF1
:10AAB0005C20FFF792FD5420FFF78FFD5620FFF733
:10AAC000A5FD5520FFF789FD9BE05F20FFF785FD81
:10AAD0005E20FFF782FD5D20FFF77FFD5C20FFF722
:10AAE0007CFD5420FFF792FD5620FFF78FFD552087
:10AAF000FFF773FD85E05F20FFF788FD5E20FFF71D
:10AB00006CFD5D20FFF769FD5C20FFF77FFD5420A1
:10AB1000FFF77CFD5620FFF760FD5520FFF75DFD38
:10AB20006FE06DE05F20FFF758FD5E20FFF76EFDE0
:10AB30005D20FFF752FD5C20FFF74FFD5420FFF72B
:10AB400065FD5620FFF749FD5520FFF746FD58E00B
:10AB50005F20FFF742FD5E20FFF758FD5D20FFF705
:10AB60003CFD5C20FFF739FD5420FFF736FD5620F1
:10AB7000FFF733FD5520FFF730FD42E05F20FFF780
:10AB80002CFD5E20FFF729FD5D20FFF726FD5C20F0
:10AB9000FFF73CFD5420FFF739FD5620FFF736FD47
:10ABA0005520FFF733FD2CE05F20FFF716FD5E20F8
:10ABB000FFF713FD5D20FFF710FD5C20FFF70DFD93
:10ABC0005420FFF70AFD5620FFF707FD5520FFF739
:10ABD00004FD16E05F20FFF700FD5E20FFF7FDFC9F
:10ABE0005D20FFF7FAFC5C20FFF7F7FC5420FFF72D
:10ABF0000DFD5620FFF7F1FC5520FFF7EEFC00E0BD
:10AC000000BF00BF2BE60A2C74D2DFE804F0051B5E
:10AC100031475D748AA0B6CC5820FFF7DEFC512086
:10AC2000FFF7DBFC5320FFF7D8FC5B20FFF7D5FCD8
:10AC30005A20FFF7D2FC5920FFF7CFFC5220FFF734
:10AC4000E5FCC7E05820FFF7E1FC5120FFF7C5FC09
:10AC50005320FFF7C2FC5B20FFF7D8FC5A20FFF718
:10AC6000D5FC5920FFF7D2FC5220FFF7CFFCB1E012
:10AC70005820FFF7B2FC5120FFF7AFFC5320FFF73D
:10AC8000C5FC5B20FFF7A9FC5A20FFF7A6FC592062
:10AC9000FFF7BCFC5220FFF7A0FC9BE05820FFF719
:10ACA0009CFC5120FFF799FC5320FFF796FC5B209A
:10ACB000FFF793FC5A20FFF7A9FC5920FFF7A6FCE9
:10ACC0005220FFF78AFC85E05820FFF79FFC5120B7
:10ACD000FFF783FC5320FFF780FC5B20FFF796FC17
:10ACE0005A20FFF793FC5920FFF777FC5220FFF71B
:10ACF00074FC6FE06DE05820FFF76FFC5120FFF708
:10AD000085FC5320FFF769FC5B20FFF766FC5A20A7
:10AD1000FFF77CFC5920FFF760FC5220FFF75DFC39
:10AD200058E05820FFF759FC5120FFF76FFC5320E3
:10AD3000FFF753FC5B20FFF750FC5A20FFF74DFC58
:10AD40005920FFF74AFC5220FFF747FC42E0582009
:10AD5000FFF743FC5120FFF740FC5320FFF73DFC79
:10AD60005B20FFF753FC5A20FFF750FC5920FFF7F8
:10AD70004DFC5220FFF74AFC2CE05820FFF72DFC39
:10AD80005120FFF72AFC5320FFF727FC5B20FFF739
:10AD900024FC5A20FFF721FC5920FFF71EFC52200B
:10ADA000FFF71BFC16E05820FFF717FC5120FFF7B8
:10ADB00014FC5320FFF711FC5B20FFF70EFC5A2018
:10ADC000FFF724FC5920FFF708FC5220FFF705FC91
:10ADD00000E000BF00BF42E50A2C74D2DFE804F0B7
:10ADE000051B31475D748AA0B6CC0B20FFF7F5FB3D
:10ADF0001220FFF7F2FB1020FFF7EFFB0820FFF710
:10AE0000ECFB0920FFF7E9FB0A20FFF7E6FB112026
:10AE1000FFF7FCFBC7E00B20FFF7F8FB1220FFF762
:10AE2000DCFB1020FFF7D9FB0820FFF7EFFB092020
:10AE3000FFF7ECFB0A20FFF7E9FB1120FFF7E6FB29
:10AE4000B1E00B20FFF7C9FB1220FFF7C6FB102073
:10AE5000FFF7DCFB0820FFF7C0FB0920FFF7BDFB75
:10AE60000A20FFF7D3FB1120FFF7B7FB9BE00B2075
:10AE7000FFF7B3FB1220FFF7B0FB1020FFF7ADFB8D
:10AE80000820FFF7AAFB0920FFF7C0FB0A20FFF705
:10AE9000BDFB1120FFF7A1FB85E00B20FFF7B6FB00
:10AEA0001220FFF79AFB1020FFF797FB0820FFF70F
:10AEB000ADFB0920FFF7AAFB0A20FFF78EFB11204C
:10AEC000FFF78BFB6FE06DE00B20FFF786FB122096
:10AED000FFF79CFB1020FFF780FB0820FFF77DFBAE
:10AEE0000920FFF793FB0A20FFF777FB1120FFF7FC
:10AEF00074FB58E00B20FFF770FB1220FFF786FB76
:10AF00001020FFF76AFB0820FFF767FB0920FFF717
:10AF100064FB0A20FFF761FB1120FFF75EFB42E0B4
:10AF20000B20FFF75AFB1220FFF757FB1020FFF70B
:10AF300054FB0820FFF76AFB0920FFF767FB0A2094
:10AF4000FFF764FB1120FFF761FB2CE00B20FFF7FC
:10AF500044FB1220FFF741FB1020FFF73EFB0820C7
:10AF6000FFF73BFB0920FFF738FB0A20FFF735FB13
:10AF70001120FFF732FB16E00B20FFF72EFB12200B
:10AF8000FFF72BFB1020FFF728FB0820FFF725FB1E
:10AF90000920FFF73BFB0A20FFF71FFB1120FFF7FB
:10AFA0001CFB00E000BF00BF59E40A2C74D2DFE8AC
:10AFB00004F0051B31475D748AA0B6CC3B20FFF737
:10AFC0000CFB3A20FFF709FB3920FFF706FB38207E
:10AFD000FFF703FB1920FFF700FB1B20FFF7FDFA2B
:10AFE0001A20FFF713FBC7E03B20FFF70FFB3A20C7
:10AFF000FFF7F3FA3920FFF7F0FA3820FFF706FBE6
:10B000001920FFF703FB1B20FFF700FB1A20FFF7B7
:10B01000FDFAB1E03B20FFF7E0FA3A20FFF7DDFA56
:10B020003920FFF7F3FA3820FFF7D7FA1920FFF796
:10B03000D4FA1B20FFF7EAFA1A20FFF7CEFA9BE0BA
:10B040003B20FFF7CAFA3A20FFF7C7FA3920FFF78B
:10B05000C4FA3820FFF7C1FA1920FFF7D7FA1B20EE
:10B06000FFF7D4FA1A20FFF7B8FA85E03B20FFF784
:10B07000CDFA3A20FFF7B1FA3920FFF7AEFA3820BF
:10B08000FFF7C4FA1920FFF7C1FA1B20FFF7A5FA52
:10B090001A20FFF7A2FA6FE06DE03B20FFF79DFA60
:10B0A0003A20FFF7B3FA3920FFF797FA3820FFF775
:10B0B00094FA1920FFF7AAFA1B20FFF78EFA1A203C
:10B0C000FFF78BFA58E03B20FFF787FA3A20FFF7AB
:10B0D0009DFA3920FFF781FA3820FFF77EFA192010
:10B0E000FFF77BFA1B20FFF778FA1A20FFF775FAB3
:10B0F00042E03B20FFF771FA3A20FFF76EFA392061
:10B10000FFF76BFA3820FFF781FA1920FFF77EFA74
:10B110001B20FFF77BFA1A20FFF778FA2CE03B2080
:10B12000FFF75BFA3A20FFF758FA3920FFF755FA94
:10B130003820FFF752FA1920FFF74FFA1B20FFF7CC
:10B140004CFA1A20FFF749FA16E03B20FFF745FAC0
:10B150003A20FFF742FA3920FFF73FFA3820FFF78D
:10B160003CFA1920FFF752FA1B20FFF736FA1A2093
:10B17000FFF733FA00E000BF00BF5AE40A2C7CD28C
:10B18000DFE804F0051D354D657F97AFC7DFFB2075
:10B19000FFF723FAF320FFF720FAF920FFF71DFA53
:10B1A000F820FFF71AFA40F20110FFF716FA40F202
:10B1B0000310FFF712FAFA20FFF728FADAE0FB2073
:10B1C000FFF724FAF320FFF708FAF920FFF705FA52
:10B1D000F820FFF71BFA40F20110FFF717FA40F2D0
:10B1E0000310FFF713FAFA20FFF710FAC2E0FB2072
:10B1F000FFF7F3F9F320FFF7F0F9F920FFF706FA6C
:10B20000F820FFF7EAF940F20110FFF7E6F940F203
:10B210000310FFF7FBF9FA20FFF7DFF9AAE0FB20A4
:10B22000FFF7DBF9F320FFF7D8F9F920FFF7D5F99D
:10B23000F820FFF7D2F940F20110FFF7E7F940F2EA
:10B240000310FFF7E3F9FA20FFF7C7F992E0FB20BC
:10B25000FFF7DCF9F320FFF7C0F9F920FFF7BDF99C
:10B26000F820FFF7D3F940F20110FFF7CFF940F2D1
:10B270000310FFF7B2F9FA2000E07AE0FFF7ADF92A
:10B2800078E0FB20FFF7A9F9F320FFF7BFF9F920D9
:10B29000FFF7A3F9F820FFF7A0F940F20110FFF73C
:10B2A000B5F940F20310FFF798F9FA20FFF795F986
:10B2B00060E0FB20FFF791F9F320FFF7A7F9F920F1
:10B2C000FFF78BF9F820FFF788F940F20110FFF73C
:10B2D00084F940F20310FFF780F9FA20FFF77DF9B7
:10B2E00048E0FB20FFF779F9F320FFF776F9F92022
:10B2F000FFF773F9F820FFF789F940F20110FFF723
:10B3000085F940F20310FFF781F9FA20FFF77EF983
:10B3100030E0FB20FFF761F9F320FFF75EF9F92039
:10B32000FFF75BF9F820FFF758F940F20110FFF73B
:10B3300054F940F20310FFF750F9FA20FFF74DF9E6
:10B3400018E0FB20FFF749F9F320FFF746F9F92051
:10B35000FFF743F9F820FFF740F940F20110FFF73B
:10B3600055F940F20310FFF738F9FA20FFF735F9E5
:10B3700000E000BF00BF45E40A2C74D2DFE804F00F
:10B38000051B31475D748AA0B6CCEB20FFF725F989
:10B39000E220FFF722F9E120FFF71FF9E820FFF78D
:10B3A0001CF9F120FFF719F9EA20FFF716F9E92057
:10B3B000FFF72CF9C7E0EB20FFF728F9E220FFF7B1
:10B3C0000CF9E120FFF709F9E820FFF71FF9F12058
:10B3D000FFF71CF9EA20FFF719F9E920FFF716F942
:10B3E000B1E0EB20FFF7F9F8E220FFF7F6F8E120F3
:10B3F000FFF70CF9E820FFF7F0F8F120FFF7EDF880
:10B40000EA20FFF703F9E920FFF7E7F89BE0EB20DC
:10B41000FFF7E3F8E220FFF7E0F8E120FFF7DDF8BF
:10B42000E820FFF7DAF8F120FFF7F0F8EA20FFF75D
:10B43000EDF8E920FFF7D1F885E0EB20FFF7E6F81B
:10B44000E220FFF7CAF8E120FFF7C7F8E820FFF78E
:10B45000DDF8F120FFF7DAF8EA20FFF7BEF8E9207F
:10B46000FFF7BBF86FE06DE0EB20FFF7B6F8E220E6
:10B47000FFF7CCF8E120FFF7B0F8E820FFF7ADF8D0
:10B48000F120FFF7C3F8EA20FFF7A7F8E920FFF75C
:10B49000A4F858E0EB20FFF7A0F8E220FFF7B6F899
:10B4A000E120FFF79AF8E820FFF797F8F120FFF77F
:10B4B00094F8EA20FFF791F8E920FFF78EF842E0D0
:10B4C000EB20FFF78AF8E220FFF787F8E120FFF78B
:10B4D00084F8E820FFF79AF8F120FFF797F8EA20C0
:10B4E000FFF794F8E920FFF791F82CE0EB20FFF745
:10B4F00074F8E220FFF771F8E120FFF76EF8E8201A
:10B50000FFF76BF8F120FFF768F8EA20FFF765F81E
:10B51000E920FFF762F816E0EB20FFF75EF8E22083
:10B52000FFF75BF8E120FFF758F8E820FFF755F840
:10B53000F120FFF76BF8EA20FFF74FF8E920FFF75B
:10B540004CF800E000BF00BF45E40A2C74D2DFE8ED
:10B5500004F0051B31475D748AA0B6CCDB20FFF7F1
:10B560003CF8D220FFF739F8D020FFF736F8D82082
:10B57000FFF733F8D920FFF730F8DA20FFF72DF87E
:10B58000D120FFF743F8C7E0DB20FFF73FF8D220D8
:10B59000FFF723F8D020FFF720F8D820FFF736F880
:10B5A000D920FFF733F8DA20FFF730F8D120FFF782
:10B5B0002DF8B1E0DB20FFF710F8D220FFF70DF8EF
:10B5C000D020FFF723F8D820FFF707F8D920FFF79E
:10B5D00004F8DA20FFF71AF8D120FEF7FEFF9BE00F
:10B5E000DB20FEF7FAFFD220FEF7F7FFD020FEF7B0
:10B5F000F4FFD820FEF7F1FFD920FFF707F8DA2093
:10B60000FFF704F8D120FEF7E8FF85E0DB20FEF726
:10B61000FDFFD220FEF7E1FFD020FEF7DEFFD820AD
:10B62000FEF7F4FFD920FEF7F1FFDA20FEF7D5FF91
:10B63000D120FEF7D2FF6FE06DE0DB20FEF7CDFFFB
:10B64000D220FEF7E3FFD020FEF7C7FFD820FEF799
:10B65000C4FFD920FEF7DAFFDA20FEF7BEFFD120C3
:10B66000FEF7BBFF58E0DB20FEF7B7FFD220FEF766
:10B67000CDFFD020FEF7B1FFD820FEF7AEFFD920D6
:10B68000FEF7ABFFDA20FEF7A8FFD120FEF7A5FFFB
:10B6900042E0DB20FEF7A1FFD220FEF79EFFD02084
:10B6A000FEF79BFFD820FEF7B1FFD920FEF7AEFFD3
:10B6B000DA20FEF7ABFFD120FEF7A8FF2CE0DB205D
:10B6C000FEF78BFFD220FEF788FFD020FEF785FF24
:10B6D000D820FEF782FFD920FEF77FFFDA20FEF7A1
:10B6E0007CFFD120FEF779FF16E0DB20FEF775FF27
:10B6F000D220FEF772FFD020FEF76FFFD820FEF7B2
:10B700006CFFD920FEF782FFDA20FEF766FFD1201A
:10B71000FEF763FF00E000BF00BF45E40A2C74D2CF
:10B72000DFE804F0051B31475D748AA0B6CCC32066
:10B73000FEF753FFC220FEF750FFC120FEF74DFF7A
:10B74000C020FEF74AFFC920FEF747FFCB20FEF7D7
:10B7500044FFCA20FEF75AFFC7E0C320FEF756FF9A
:10B76000C220FEF73AFFC120FEF737FFC020FEF7E8
:10B770004DFFC920FEF74AFFCB20FEF747FFCA2046
:10B78000FEF744FFB1E0C320FEF727FFC220FEF71B
:10B7900024FFC120FEF73AFFC020FEF71EFFC9209C
:10B7A000FEF71BFFCB20FEF731FFCA20FEF715FF87
:10B7B0009BE0C320FEF711FFC220FEF70EFFC12061
:10B7C000FEF70BFFC020FEF708FFC920FEF71EFFA3
:10B7D000CB20FEF71BFFCA20FEF7FFFE85E0C3204B
:10B7E000FEF714FFC220FEF7F8FEC120FEF7F5FEBB
:10B7F000C020FEF70BFFC920FEF708FFCB20FEF7A5
:10B80000ECFECA20FEF7E9FE6FE06DE0C320FEF714
:10B81000E4FEC220FEF7FAFEC120FEF7DEFEC020E5
:10B82000FEF7DBFEC920FEF7F1FECB20FEF7D5FECA
:10B83000CA20FEF7D2FE58E0C320FEF7CEFEC2209B
:10B84000FEF7E4FEC120FEF7C8FEC020FEF7C5FEED
:10B85000C920FEF7C2FECB20FEF7BFFECA20FEF7CE
:10B86000BCFE42E0C320FEF7B8FEC220FEF7B5FEE4
:10B87000C120FEF7B2FEC020FEF7C8FEC920FEF7C9
:10B88000C5FECB20FEF7C2FECA20FEF7BFFE2CE0AD
:10B89000C320FEF7A2FEC220FEF79FFEC120FEF7E6
:10B8A0009CFEC020FEF799FEC920FEF796FECB2035
:10B8B000FEF793FECA20FEF790FE16E0C320FEF7C7
:10B8C0008CFEC220FEF789FEC120FEF786FEC02056
:10B8D000FEF783FEC920FEF799FECB20FEF77DFE22
:10B8E000CA20FEF77AFE00E000BF00BF45E40A2C44
:10B8F00074D2DFE804F0051B31475D748AA0B6CC32
:10B90000B320FEF76AFEAB20FEF767FEB120FEF71C
:10B9100064FEB020FEF761FEB920FEF75EFEBB209C
:10B92000FEF75BFEB220FEF771FEC7E0B320FEF724
:10B930006DFEAB20FEF751FEB120FEF74EFEB020AB
:10B94000FEF764FEB920FEF761FEBB20FEF75EFE47
:10B95000B220FEF75BFEB1E0B320FEF73EFEAB2067
:10B96000FEF73BFEB120FEF751FEB020FEF735FE9C
:10B97000B920FEF732FEBB20FEF748FEB220FEF7EC
:10B980002CFE9BE0B320FEF728FEAB20FEF725FE41
:10B99000B120FEF722FEB020FEF71FFEB920FEF711
:10B9A00035FEBB20FEF732FEB220FEF716FE85E024
:10B9B000B320FEF72BFEAB20FEF70FFEB120FEF703
:10B9C0000CFEB020FEF722FEB920FEF71FFEBB20C2
:10B9D000FEF703FEB220FEF700FE6FE06DE0B3203D
:10B9E000FEF7FBFDAB20FEF711FEB120FEF7F5FDE3
:10B9F000B020FEF7F2FDB920FEF708FEBB20FEF7EF
:10BA0000ECFDB220FEF7E9FD58E0B320FEF7E5FDBE
:10BA1000AB20FEF7FBFDB120FEF7DFFDB020FEF707
:10BA2000DCFDB920FEF7D9FDBB20FEF7D6FDB22024
:10BA3000FEF7D3FD42E0B320FEF7CFFDAB20FEF7CB
:10BA4000CCFDB120FEF7C9FDB020FEF7DFFDB92027
:10BA5000FEF7DCFDBB20FEF7D9FDB220FEF7D6FDD8
:10BA60002CE0B320FEF7B9FDAB20FEF7B6FDB12008
:10BA7000FEF7B3FDB020FEF7B0FDB920FEF7ADFD37
:10BA8000BB20FEF7AAFDB220FEF7A7FD16E0B3200B
:10BA9000FEF7A3FDAB20FEF7A0FDB120FEF79DFD54
:10BAA000B020FEF79AFDB920FEF7B0FDBB20FEF7EF
:10BAB00094FDB220FEF791FD00E000BF00BF5AE404
:10BAC0000A2C74D2DFE804F0051B31475D748AA0AC
:10BAD000B6CCA320FEF781FD9A20FEF77EFD9920CB
:10BAE000FEF77BFDA020FEF778FDA920FEF775FD8F
:10BAF000A220FEF772FDA120FEF788FDC7E0A3207B
:10BB0000FEF784FD9A20FEF768FD9920FEF765FD9B
:10BB1000A020FEF77BFDA920FEF778FDA220FEF70E
:10BB200075FDA120FEF772FDB1E0A320FEF755FDE3
:10BB30009A20FEF752FD9920FEF768FDA020FEF73F
:10BB40004CFDA920FEF749FDA220FEF75FFDA120D4
:10BB5000FEF743FD9BE0A320FEF73FFD9A20FEF792
:10BB60003CFD9920FEF739FDA020FEF736FDA92007
:10BB7000FEF74CFDA220FEF749FDA120FEF72DFDAA
:10BB800085E0A320FEF742FD9A20FEF726FD9920CE
:10BB9000FEF723FDA020FEF739FDA920FEF736FDB4
:10BBA000A220FEF71AFDA120FEF717FD6FE06DE061
:10BBB000A320FEF712FD9A20FEF728FD9920FEF73C
:10BBC0000CFDA020FEF709FDA920FEF71FFDA22015
:10BBD000FEF703FDA120FEF700FD58E0A320FEF7CD
:10BBE000FCFC9A20FEF712FD9920FEF7F6FCA0203F
:10BBF000FEF7F3FCA920FEF7F0FCA220FEF7EDFC17
:10BC0000A120FEF7EAFC42E0A320FEF7E6FC9A2022
:10BC1000FEF7E3FC9920FEF7E0FCA020FEF7F6FC1F
:10BC2000A920FEF7F3FCA220FEF7F0FCA120FEF70E
:10BC3000EDFC2CE0A320FEF7D0FC9A20FEF7CDFC13
:10BC40009920FEF7CAFCA020FEF7C7FCA920FEF74A
:10BC5000C4FCA220FEF7C1FCA120FEF7BEFC16E04A
:10BC6000A320FEF7BAFC9A20FEF7B7FC9920FEF756
:10BC7000B4FCA020FEF7B1FCA920FEF7C7FCA2206F
:10BC8000FEF7ABFCA120FEF7A8FC00E000BF00BF60
:10BC90005AE40A2C74D2DFE804F0051B31475D74C6
:10BCA0008AA0B6CC9320FEF798FC8A20FEF795FC7C
:10BCB0008820FEF792FC9020FEF78FFC9120FEF783
:10BCC0008CFC9220FEF789FC8920FEF79FFCC7E0E0
:10BCD0009320FEF79BFC8A20FEF77FFC8820FEF76E
:10BCE0007CFC9020FEF792FC9120FEF78FFC9220C6
:10BCF000FEF78CFC8920FEF789FCB1E09320FEF76B
:10BD00006CFC8A20FEF769FC8820FEF77FFC9020FF
:10BD1000FEF763FC9120FEF760FC9220FEF776FCB4
:10BD20008920FEF75AFC9BE09320FEF756FC8A2000
:10BD3000FEF753FC8820FEF750FC9020FEF74DFCE8
:10BD40009120FEF763FC9220FEF760FC8920FEF74D
:10BD500044FC85E09320FEF759FC8A20FEF73DFC69
:10BD60008820FEF73AFC9020FEF750FC9120FEF769
:10BD70004DFC9220FEF731FC8920FEF72EFC6FE08F
:10BD80006DE09320FEF729FC8A20FEF73FFC882017
:10BD9000FEF723FC9020FEF720FC9120FEF736FCF6
:10BDA0009220FEF71AFC8920FEF717FC58E093203A
:10BDB000FEF713FC8A20FEF729FC8820FEF70DFC15
:10BDC0009020FEF70AFC9120FEF707FC9220FEF778
:10BDD00004FC8920FEF701FC42E09320FEF7FDFB06
:10BDE0008A20FEF7FAFB8820FEF7F7FB9020FEF78B
:10BDF0000DFC9120FEF70AFC9220FEF707FC89203B
:10BE0000FEF704FC2CE09320FEF7E7FB8A20FEF708
:10BE1000E4FB8820FEF7E1FB9020FEF7DEFB91209B
:10BE2000FEF7DBFB9220FEF7D8FB8920FEF7D5FB5F
:10BE300016E09320FEF7D1FB8A20FEF7CEFB882088
:10BE4000FEF7CBFB9020FEF7C8FB9120FEF7DEFB50
:10BE50009220FEF7C2FB8920FEF7BFFB00E000BF87
:10BE600000BF5AE40A2C7DD2DFE804F0051E3750EB
:10BE700069849DB6CFE8FC20FEF7AFFBFD20FEF7FE
:10BE8000ACFBFE20FEF7A9FBFF20FEF7A6FB40F26D
:10BE90000710FEF7A2FB40F20510FEF79EFB4FF4E1
:10BEA0008370FEF7B3FBE3E0FC20FEF7AFFBFD2061
:10BEB000FEF793FBFE20FEF790FBFF20FEF7A6FBAC
:10BEC00040F20710FEF7A2FB40F20510FEF79EFBC2
:10BED0004FF48370FEF79AFBCAE0FC20FEF77DFB6F
:10BEE000FD20FEF77AFBFE20FEF790FBFF20FEF719
:10BEF00074FB40F20710FEF770FB40F20510FEF7EE
:10BF000085FB4FF48370FEF768FBB1E0FC20FEF781
:10BF100064FBFD20FEF761FBFE20FEF75EFBFF20C9
:10BF2000FEF75BFB40F20710FEF770FB40F20510D6
:10BF3000FEF76CFB4FF48370FEF74FFB98E0FC209C
:10BF4000FEF764FBFD20FEF748FBFE20FEF745FBF5
:10BF5000FF20FEF75BFB40F20710FEF757FB40F2B5
:10BF6000051000E083E0FEF738FB4FF48370FEF726
:10BF700034FB7DE0FC20FEF730FBFD20FEF746FBA6
:10BF8000FE20FEF72AFBFF20FEF727FB40F20710FA
:10BF9000FEF73CFB40F20510FEF71FFB4FF48370E9
:10BFA000FEF71BFB64E0FC20FEF717FBFD20FEF70D
:10BFB0002DFBFE20FEF711FBFF20FEF70EFB40F2EB
:10BFC0000710FEF70AFB40F20510FEF706FB4FF4E0
:10BFD0008370FEF702FB4BE0FC20FEF7FEFAFD202B
:10BFE000FEF7FBFAFE20FEF7F8FAFF20FEF70EFB45
:10BFF00040F20710FEF70AFB40F20510FEF706FBC1
:10C000004FF48370FEF702FB32E0FC20FEF7E5FA06
:10C01000FD20FEF7E2FAFE20FEF7DFFAFF20FEF732
:10C02000DCFA40F20710FEF7D8FA40F20510FEF7EE
:10C03000D4FA4FF48370FEF7D0FA19E0FC20FEF733
:10C04000CCFAFD20FEF7C9FAFE20FEF7C6FAFF2063
:10C05000FEF7C3FA40F20710FEF7D8FA40F20510D7
:10C06000FEF7BBFA4FF48370FEF7B7FA00E000BFAB
:10C0700000BF3BE40A2C74D2DFE804F0051B314713
:10C080005D748AA0B6CCEC20FEF7A7FAE420FEF798
:10C09000A4FAEE20FEF7A1FAEF20FEF79EFAF620B2
:10C0A000FEF79BFAF420FEF798FAED20FEF7AEFAC1
:10C0B000C7E0EC20FEF7AAFAE420FEF78EFAEE20A5
:10C0C000FEF78BFAEF20FEF7A1FAF620FEF79EFAB4
:10C0D000F420FEF79BFAED20FEF798FAB1E0EC2091
:10C0E000FEF77BFAE420FEF778FAEE20FEF78EFAF0
:10C0F000EF20FEF772FAF620FEF76FFAF420FEF753
:10C1000085FAED20FEF769FA9BE0EC20FEF765FA70
:10C11000E420FEF762FAEE20FEF75FFAEF20FEF76A
:10C120005CFAF620FEF772FAF420FEF76FFAED20C3
:10C13000FEF753FA85E0EC20FEF768FAE420FEF7FC
:10C140004CFAEE20FEF749FAEF20FEF75FFAF620F0
:10C15000FEF75CFAF420FEF740FAED20FEF73DFA18
:10C160006FE06DE0EC20FEF738FAE420FEF74EFABF
:10C17000EE20FEF732FAEF20FEF72FFAF620FEF758
:10C1800045FAF420FEF729FAED20FEF726FA58E0EA
:10C19000EC20FEF722FAE420FEF738FAEE20FEF754
:10C1A0001CFAEF20FEF719FAF620FEF716FAF42033
:10C1B000FEF713FAED20FEF710FA42E0EC20FEF74E
:10C1C0000CFAE420FEF709FAEE20FEF706FAEF205B
:10C1D000FEF71CFAF620FEF719FAF420FEF716FA1D
:10C1E000ED20FEF713FA2CE0EC20FEF7F6F9E42040
:10C1F000FEF7F3F9EE20FEF7F0F9EF20FEF7EDF988
:10C20000F620FEF7EAF9F420FEF7E7F9ED20FEF755
:10C21000E4F916E0EC20FEF7E0F9E420FEF7DDF9A2
:10C22000EE20FEF7DAF9EF20FEF7D7F9F620FEF759
:10C23000EDF9F420FEF7D1F9ED20FEF7CEF900E09C
:10C2400000BF00BF3BE40A2C74D2DFE804F0051BFA
:10C2500031475D748AA0B6CCDC20FEF7BEF9D5204C
:10C26000FEF7BBF9D620FEF7B8F9DF20FEF7B5F9E7
:10C27000E620FEF7B2F9DD20FEF7AFF9DE20FEF78B
:10C28000C5F9C7E0DC20FEF7C1F9D520FEF7A5F916
:10C29000D620FEF7A2F9DF20FEF7B8F9E620FEF778
:10C2A000B5F9DD20FEF7B2F9DE20FEF7AFF9B1E017
:10C2B000DC20FEF792F9D520FEF78FF9D620FEF7A5
:10C2C000A5F9DF20FEF789F9E620FEF786F9DD20E3
:10C2D000FEF79CF9DE20FEF780F99BE0DC20FEF7FC
:10C2E0007CF9D520FEF779F9D620FEF776F9DF2024
:10C2F000FEF773F9E620FEF789F9DD20FEF786F9EF
:10C30000DE20FEF76AF985E0DC20FEF77FF9D52014
:10C31000FEF763F9D620FEF760F9DF20FEF776F925
:10C32000E620FEF773F9DD20FEF757F9DE20FEF771
:10C3300054F96FE06DE0DC20FEF74FF9D520FEF7F1
:10C3400065F9D620FEF749F9DF20FEF746F9E62029
:10C35000FEF75CF9DD20FEF740F9DE20FEF73DF93F
:10C3600058E0DC20FEF739F9D520FEF74FF9D6204A
:10C37000FEF733F9DF20FEF730F9E620FEF72DF95E
:10C38000DD20FEF72AF9DE20FEF727F942E0DC2067
:10C39000FEF723F9D520FEF720F9D620FEF71DF988
:10C3A000DF20FEF733F9E620FEF730F9DD20FEF757
:10C3B0002DF9DE20FEF72AF92CE0DC20FEF70DF93E
:10C3C000D520FEF70AF9D620FEF707F9DF20FEF7A1
:10C3D00004F9E620FEF701F9DD20FEF7FEF8DE2085
:10C3E000FEF7FBF816E0DC20FEF7F7F8D520FEF7A5
:10C3F000F4F8D620FEF7F1F8DF20FEF7EEF8E6209D
:10C40000FEF704F9DD20FEF7E8F8DE20FEF7E5F898
:10C4100000E000BF00BFA3E30A2C74D2DFE804F001
:10C42000051B31475D748AA0B6CCCC20FEF7D5F849
:10C43000C520FEF7D2F8C720FEF7CFF8CF20FEF7D1
:10C44000CCF8CE20FEF7C9F8CD20FEF7C6F8C620FE
:10C45000FEF7DCF8C7E0CC20FEF7D8F8C520FEF7E1
:10C46000BCF8C720FEF7B9F8CF20FEF7CFF8CE20F2
:10C47000FEF7CCF8CD20FEF7C9F8C620FEF7C6F8C7
:10C48000B1E0CC20FEF7A9F8C520FEF7A6F8C7203A
:10C49000FEF7BCF8CF20FEF7A0F8CE20FEF79DF8FF
:10C4A000CD20FEF7B3F8C620FEF797F89BE0CC202E
:10C4B000FEF793F8C520FEF790F8C720FEF78DF839
:10C4C000CF20FEF78AF8CE20FEF7A0F8CD20FEF7A9
:10C4D0009DF8C620FEF781F885E0CC20FEF796F89F
:10C4E000C520FEF77AF8C720FEF777F8CF20FEF7D1
:10C4F0008DF8CE20FEF78AF8CD20FEF76EF8C62024
:10C50000FEF76BF86FE06DE0CC20FEF766F8C52013
:10C51000FEF77CF8C720FEF760F8CF20FEF75DF845
:10C52000CE20FEF773F8CD20FEF757F8C620FEF7B1
:10C5300054F858E0CC20FEF750F8C520FEF766F816
:10C54000C720FEF74AF8CF20FEF747F8CE20FEF7C7
:10C5500044F8CD20FEF741F8C620FEF73EF842E051
:10C56000CC20FEF73AF8C520FEF737F8C720FEF7D3
:10C5700034F8CF20FEF74AF8CE20FEF747F8CD205A
:10C58000FEF744F8C620FEF741F82CE0CC20FEF779
:10C5900024F8C520FEF721F8C720FEF71EF8CF20AB
:10C5A000FEF71BF8CE20FEF718F8CD20FEF715F8A1
:10C5B000C620FEF712F816E0CC20FEF70EF8C520D4
:10C5C000FEF70BF8C720FEF708F8CF20FEF705F8B6
:10C5D000CE20FEF71BF8CD20FDF7FFFFC620FDF7AC
:10C5E000FCFF00E000BF00BFBAE20A2C74D2DFE813
:10C5F00004F0051B31475D748AA0B6CCB420FDF76A
:10C60000ECFFB520FDF7E9FFB620FDF7E6FFB72008
:10C61000FDF7E3FFBE20FDF7E0FFBC20FDF7DDFFE7
:10C62000BD20FDF7F3FFC7E0B420FDF7EFFFB52015
:10C63000FDF7D3FFB620FDF7D0FFB720FDF7E6FFEB
:10C64000BE20FDF7E3FFBC20FDF7E0FFBD20FDF7B6
:10C65000DDFFB1E0B420FDF7C0FFB520FDF7BDFF61
:10C66000B620FDF7D3FFB720FDF7B7FFBE20FDF7DB
:10C67000B4FFBC20FDF7CAFFBD20FDF7AEFF9BE075
:10C68000B420FDF7AAFFB520FDF7A7FFB620FDF700
:10C69000A4FFB720FDF7A1FFBE20FDF7B7FFBC2028
:10C6A000FDF7B4FFBD20FDF798FF85E0B420FDF74E
:10C6B000ADFFB520FDF791FFB620FDF78EFFB72047
:10C6C000FDF7A4FFBE20FDF7A1FFBC20FDF785FF0D
:10C6D000BD20FDF782FF6FE06DE0B420FDF77DFF28
:10C6E000B520FDF793FFB620FDF777FFB720FDF7E4
:10C6F00074FFBE20FDF78AFFBC20FDF76EFFBD2052
:10C70000FDF76BFF58E0B420FDF767FFB520FDF79C
:10C710007DFFB620FDF761FFB720FDF75EFFBE206D
:10C72000FDF75BFFBC20FDF758FFBD20FDF755FF6F
:10C7300042E0B420FDF751FFB520FDF74EFFB620D3
:10C74000FDF74BFFB720FDF761FFBE20FDF75EFF51
:10C75000BC20FDF75BFFBD20FDF758FF2CE0B420A7
:10C76000FDF73BFFB520FDF738FFB620FDF735FF9D
:10C77000B720FDF732FFBE20FDF72FFFBC20FDF7ED
:10C780002CFFBD20FDF729FF16E0B420FDF725FFA3
:10C79000B520FDF722FFB620FDF71FFFB720FDF7FC
:10C7A0001CFFBE20FDF732FFBC20FDF716FFBD20A9
:10C7B000FDF713FF00E000BF00BFD1E10A2C74D2E7
:10C7C000DFE804F0051B31475D748AA0B6CCA420D5
:10C7D000FDF703FF9C20FDF700FFA620FDF7FDFEFF
:10C7E000A720FDF7FAFEAE20FDF7F7FEAC20FDF71F
:10C7F000F4FEA520FDF70AFFC7E0A420FDF706FF21
:10C800009C20FDF7EAFEA620FDF7E7FEA720FDF736
:10C81000FDFEAE20FDF7FAFEAC20FDF7F7FEA520E9
:10C82000FDF7F4FEB1E0A420FDF7D7FE9C20FDF754
:10C83000D4FEA620FDF7EAFEA720FDF7CEFEAE202F
:10C84000FDF7CBFEAC20FDF7E1FEA520FDF7C5FE10
:10C850009BE0A420FDF7C1FE9C20FDF7BEFEA620B4
:10C86000FDF7BBFEA720FDF7B8FEAE20FDF7CEFE1C
:10C87000AC20FDF7CBFEA520FDF7AFFE85E0A420A0
:10C88000FDF7C4FE9C20FDF7A8FEA620FDF7A5FE3F
:10C89000A720FDF7BBFEAE20FDF7B8FEAC20FDF7EC
:10C8A0009CFEA520FDF799FE6FE06DE0A420FDF74A
:10C8B00094FE9C20FDF7AAFEA620FDF78EFEA72081
:10C8C000FDF78BFEAE20FDF7A1FEAC20FDF785FE47
:10C8D000A520FDF782FE58E0A420FDF77EFE9C20F7
:10C8E000FDF794FEA620FDF778FEA720FDF775FE64
:10C8F000AE20FDF772FEAC20FDF76FFEA520FDF720
:10C900006CFE42E0A420FDF768FE9C20FDF765FE6A
:10C91000A620FDF762FEA720FDF778FEAE20FDF70A
:10C9200075FEAC20FDF772FEA520FDF76FFE2CE032
:10C93000A420FDF752FE9C20FDF74FFEA620FDF738
:10C940004CFEA720FDF749FEAE20FDF746FEAC20C9
:10C95000FDF743FEA520FDF740FE16E0A420FDF7FD
:10C960003CFE9C20FDF739FEA620FDF736FEA720F1
:10C97000FDF733FEAE20FDF749FEAC20FDF72DFE9E
:10C98000A520FDF72AFE00E000BF00BFE8E00A2C6A
:10C9900074D2DFE804F0051B31475D748AA0B6CC81
:10C9A0009420FDF71AFE8D20FDF717FE8F20FDF76E
:10C9B00014FE9720FDF711FE9E20FDF70EFE952038
:10C9C000FDF70BFE9620FDF721FEC7E09420FDF752
:10C9D0001DFE8D20FDF701FE8F20FDF7FEFD972047
:10C9E000FDF714FE9E20FDF711FE9520FDF70EFECB
:10C9F0009620FDF70BFEB1E09420FDF7EEFD8D20B3
:10CA0000FDF7EBFD8F20FDF701FE9720FDF7E5FD1B
:10CA10009E20FDF7E2FD9520FDF7F8FD9620FDF73D
:10CA2000DCFD9BE09420FDF7D8FD8D20FDF7D5FDC2
:10CA30008F20FDF7D2FD9720FDF7CFFD9E20FDF75B
:10CA4000E5FD9520FDF7E2FD9620FDF7C6FD85E0AA
:10CA50009420FDF7DBFD8D20FDF7BFFD8F20FDF756
:10CA6000BCFD9720FDF7D2FD9E20FDF7CFFD952060
:10CA7000FDF7B3FD9620FDF7B0FD6FE06DE094206B
:10CA8000FDF7ABFD8D20FDF7C1FD8F20FDF7A5FD66
:10CA90009720FDF7A2FD9E20FDF7B8FD9520FDF73C
:10CAA0009CFD9620FDF799FD58E09420FDF795FD3B
:10CAB0008D20FDF7ABFD8F20FDF78FFD9720FDF753
:10CAC0008CFD9E20FDF789FD9520FDF786FD9620C3
:10CAD000FDF783FD42E09420FDF77FFD8D20FDF7FB
:10CAE0007CFD8F20FDF779FD9720FDF78FFD9E20BF
:10CAF000FDF78CFD9520FDF789FD9620FDF786FD5D
:10CB00002CE09420FDF769FD8D20FDF766FD8F2058
:10CB1000FDF763FD9720FDF760FD9E20FDF75DFDAD
:10CB20009520FDF75AFD9620FDF757FD16E094205D
:10CB3000FDF753FD8D20FDF750FD8F20FDF74DFDD6
:10CB40009720FDF74AFD9E20FDF760FD9520FDF73B
:10CB500044FD9620FDF741FD00E000BF00BF00BF8F
:10CB600000BF30BD10B50446152C7AD2DFE804F0C2
:10CB7000790B21374D637A90A8BED4F4F2F1F0EF2F
:10CB8000EEEDECEBEA000F20FDF740FD1720FDF77E
:10CB90003DFD1520FDF73AFD0C20FDF737FD0D207A
:10CBA000FDF734FD0E20FDF731FD1620FDF72EFDBB
:10CBB000B2E11F20FDF72AFD3E20FDF727FD3D20B5
:10CBC000FDF724FD1C20FDF721FD1420FDF71EFDBF
:10CBD0001E20FDF71BFD1D20FDF718FD9CE15F20C9
:10CBE000FDF714FD5E20FDF711FD5D20FDF70EFD44
:10CBF0005C20FDF70BFD5420FDF708FD5620FDF7E6
:10CC000005FD5520FDF702FD86E15820FDF7FEFCED
:10CC10005120FDF7FBFC5320FDF7F8FC5B20FDF7EE
:10CC2000F5FC5A20FDF7F2FC5920FDF7EFFC5220ED
:10CC3000FDF7ECFC70E10B20FDF7E8FC1220FDF79E
:10CC4000E5FC1020FDF7E2FC0820FDF7DFFC0920E1
:10CC5000FDF7DCFC0A20FDF7D9FC1120FDF7D6FC1E
:10CC60005AE158E13B20FDF7D1FC3A20FDF7CEFC1C
:10CC70003920FDF7CBFC3820FDF7C8FC1920FDF763
:10CC8000C5FC1B20FDF7C2FC1A20FDF7BFFC43E1E9
:10CC9000FB20FDF7BBFCF320FDF7B8FCF920FDF706
:10CCA000B5FCF820FDF7B2FC40F20110FDF7AEFC38
:10CCB00040F20310FDF7AAFCFA20FDF7A7FC2BE1D8
:10CCC000EB20FDF7A3FCE220FDF7A0FCE120FDF73F
:10CCD0009DFCE820FDF79AFCF120FDF797FCEA2087
:10CCE000FDF794FCE920FDF791FC15E1DB20FDF751
:10CCF0008DFCD220FDF78AFCD020FDF787FCD820E0
:10CD0000FDF784FCD920FDF781FCDA20FDF77EFCDD
:10CD1000D120FDF77BFCFFE0C320FDF777FCC220AC
:10CD2000FDF774FCC120FDF771FCC020FDF76EFC1F
:10CD3000C920FDF76BFCCB20FDF768FCCA20FDF78E
:10CD400065FCE9E0D1E0BAE0A3E08CE075E05EE0EC
:10CD500044E02DE016E0FFE7B320FDF757FCAB20E1
:10CD6000FDF754FCB120FDF751FCB020FDF74EFC5F
:10CD7000B920FDF74BFCBB20FDF748FCB220FDF7C6
:10CD800045FCC9E0A320FDF741FC9A20FDF73EFCDD
:10CD90009920FDF73BFCA020FDF738FCA920FDF70A
:10CDA00035FCA220FDF732FCA120FDF72FFCB3E0FB
:10CDB0009320FDF72BFC8A20FDF728FC8820FDF747
:10CDC00025FC9020FDF722FC9120FDF71FFC92200E
:10CDD000FDF71CFC8920FDF719FC9DE0FC20FDF708
:10CDE00015FCFD20FDF712FCFE20FDF70FFCFF20D7
:10CDF000FDF70CFC40F20710FDF708FC40F20510AF
:10CE0000FDF704FC4FF48370FDF700FC84E0EC2098
:10CE1000FDF7FCFBE420FDF7F9FBEE20FDF7F6FB48
:10CE2000EF20FDF7F3FBF620FDF7F0FBF420FDF714
:10CE3000EDFBED20FDF7EAFB6EE0DC20FDF7E6FB05
:10CE4000D520FDF7E3FBD620FDF7E0FBDF20FDF763
:10CE5000DDFBE620FDF7DAFBDD20FDF7D7FBDE206A
:10CE6000FDF7D4FB58E0CC20FDF7D0FBC520FDF743
:10CE7000CDFBC720FDF7CAFBCF20FDF7C7FBCE20B7
:10CE8000FDF7C4FBCD20FDF7C1FBC620FDF7BEFBBF
:10CE900042E0B420FDF7BAFBB520FDF7B7FBB620A2
:10CEA000FDF7B4FBB720FDF7B1FBBE20FDF7AEFBED
:10CEB000BC20FDF7ABFBBD20FDF7A8FB2CE0A420B8
:10CEC000FDF7A4FB9C20FDF7A1FBA620FDF79EFB30
:10CED000A720FDF79BFBAE20FDF798FBAC20FDF7EC
:10CEE00095FBA520FDF792FB16E09420FDF78EFB45
:10CEF0008D20FDF78BFB8F20FDF788FB9720FDF73A
:10CF000085FB9E20FDF782FB9520FDF77FFB962099
:10CF1000FDF77CFB00E000BF00BF10BD0246F948F2
:10CF200012B1012A22D110E0012904D0022904D033
:10CF3000032906D103E0F44805E0F24803E0F34892
:10CF400001E0F04800BF00BF10E0012904D0022931
:10CF500004D0032906D103E0EA4805E0EB4803E0EA
:10CF6000EB4801E0E74800BF00BF00BF00BF7047CB
:10CF70002DE9FF5F90B0824600200D900E900F903B
:10CF8000E4A00B9000200A90DDF878900022134670
:10CF9000DDE912013AF00EFE09D201200A900020CC
:10CFA0000146DDE912233AF029FCCDE912014FF0E8
:10CFB000000B0AF102003AF016FD02460B46CDE9DD
:10CFC00002010020D4493BF0DBFACDE90401DDE9A0
:10CFD00012233AF019FCCDE906013AF09BFD074611
:10CFE000884664220023384641463AF001FA63211C
:10CFF0004A401A4302D17F1C48F100080AF102009E
:10D000003AF0F1FC02460B46CDE900010020C2498E
:10D010003BF0B6FACDE90401384641463AF001FD4D
:10D02000CDE90201DDE904233AF060FCCDE9060117
:10D030003AF070FD04460D4651460A98FFF76EFF20
:10D04000201A75F100012CDBB448807AC0F340004F
:10D05000F8B1B348407C012826D00120B04948747B
:10D0600006210A2030F008F9AE4890F87D00022829
:10D0700002DA0120AB49C877AA4890F87D00FA2867
:10D0800012DAA84890F87D00401CA64981F87D007E
:10D090000AE00020A2494874A249C87781F87D00BF
:10D0A00002E000209E4948740A98012803D1A9F1A2
:10D0B000010000F0FF09BAF1010F06D0BAF1020F2A
:10D0C00008D0BAF1030F4BD11FE0A9EB0A0000F022
:10D0D000FF094AE00A9810B1012810D107E09249EF
:10D0E0000020091BA84101DA4FF0010A07E08F492F
:10D0F0000020091BA84101DA4FF0010A00BF00BF60
:10D10000A9EB0A0000F0FF092FE00A9810B10128EE
:10D1100020D10FE084490020091BA84102DA4FF01A
:10D12000010A06E081490020091BA84101DA4FF0FD
:10D13000020A0FE07D490020091BA84102DA4FF0E6
:10D14000010A06E07A490020091BA84101DA4FF0E4
:10D15000020A00BF00BFA9EB0A0000F0FF0904E0CB
:10D16000A9F1020000F0FF0900BF00BFBAF1010FF2
:10D1700006D0BAF1020F07D0BAF1030F0CD107E0C5
:10D180009820FDF72AFA0BE0A820FDF726FA07E021
:10D19000B820FDF722FA03E0A820FDF71EFA00BF31
:10D1A00000BF1CE048463AF02FFC02460B46CDE992
:10D1B0000001002058493BF0E3F9CDE90401204685
:10D1C00029463AF02EFCCDE90201DDE904233AF0CC
:10D1D00015FBCDE906013AF09DFC04460D46484694
:10D1E0003AF012FC02460B46CDE9000100204A4904
:10D1F0003BF0C6F9CDE90401204629463AF011FC7E
:10D20000CDE90201DDE904233AF0F8FA00221346E1
:10D21000CDE906013AF0E6FCC4D90A2200232046F3
:10D2200029463AF0E5F8D0B20C900A2200232046B5
:10D2300029463AF0DDF804460D461AE0A9F101014D
:10D24000A1EB0B010DAA0C9850540BF1010000F05A
:10D25000FF0B0A220023204629463AF0C9F8D0B233
:10D260000C900A220023204629463AF0C1F80446D1
:10D270000D4600210846091BA841DFDBA9F1010189
:10D28000A1EB0B010DAA0C9850540BF1010000F01A
:10D29000FF0B00224FF0804310461F493BF070F90E
:10D2A000CDE90401384641463AF0BBFBCDE9020125
:10D2B000DDE904233AF01AFBCDE906013AF02AFC35
:10D2C00004460D46002618E00A220023204629467F
:10D2D0003AF08EF8D0B20C900A220023204629465C
:10D2E0003AF086F804460D4609EB0A01491E891BEF
:10D2F0000DAA0C985054701CC6B25645E4DB0026AB
:10D300001FE0000040548900804A5D05A0BB0D006D
:10D31000905F01002E00000000002440EA2D002054
:10D32000581D0020901900207F9698003F420F0062
:10D330009F8601001F993144C8B2FFF713FC701C8F
:10D34000C6B2A9EB0B00B042F4DC0A98012841D127
:10D35000A9EB0B00C0B209901E98401EC0B21E90EF
:10D360000998072821D2DFE800F004080C101418EF
:10D370001C001120FDF731F91BE01A20FDF72DF9F3
:10D3800017E0FA20FDF729F913E0E920FDF725F968
:10D390000FE0D120FDF721F90BE0CA20FDF71DF9C0
:10D3A00007E0B220FDF719F903E01120FDF715F9A8
:10D3B00000BF00BF099E09E00DAA915D1F9A32448B
:10D3C000521CD0B2FDF746F9701CC6B21E988642B8
:10D3D000F2DB0FE0A9EB0B00C6B208E00DAA915DED
:10D3E0001F9A3244D0B2FDF735F9701CC6B21E98B0
:10D3F0008642F3DB14B0BDE8F09F2DE9FF5F90B0EB
:10D40000824600200D900E900F90AFF2F8000B9026
:10D4100000200A90DDF8789000221346DDE9120121
:10D420003AF0C8FB09D201200A9000200146DDE94C
:10D4300012233AF0E3F9CDE912014FF0000B0AF1A3
:10D4400002003AF0D0FA02460B46CDE90201002074
:10D45000FE493BF095F8CDE90401DDE912233AF0ED
:10D46000D3F9CDE906013AF055FB07468846642218
:10D4700000233846414639F0BBFF63214A401A4336
:10D4800002D17F1C48F100080AF102003AF0ABFA21
:10D4900002460B46CDE900010020EC493BF070F854
:10D4A000CDE90401384641463AF0BBFACDE9020124
:10D4B000DDE904233AF01AFACDE906013AF02AFB35
:10D4C00004460D460A98012803D1A9F1010000F095
:10D4D000FF09BAF1010F06D0BAF1020F08D0BAF174
:10D4E000030F4FD120E0A9EB0A0000F0FF094EE046
:10D4F0000A9810B1012811D107E0D5490020091B75
:10D50000A84101DA4FF0010A08E042F20F71002051
:10D51000091BA84101DA4FF0010A00BF00BFA9EBC7
:10D520000A0000F0FF0932E00A9810B1012823D167
:10D5300010E0C7490020091BA84102DA4FF0010A98
:10D5400007E042F20F710020091BA84101DA4FF0F9
:10D55000020A11E042F20F710020091BA84102DA11
:10D560004FF0010A07E040F2E7310020091BA84113
:10D5700001DA4FF0020A00BF00BFA9EB0A0000F079
:10D58000FF0904E0A9F1020000F0FF0900BF00BF9D
:10D59000BAF1010F06D0BAF1020F07D0BAF1030FAA
:10D5A0000CD107E09F20FDF718F80BE0AF20FDF746
:10D5B00014F807E0BF20FDF710F803E0AF20FDF7F7
:10D5C0000CF800BF00BF1CE048463AF01DFA0246C6
:10D5D0000B46CDE9000100209C493AF0D1FFCDE98E
:10D5E0000401204629463AF01CFACDE90201DDE9A2
:10D5F00004233AF003F9CDE906013AF08BFA044628
:10D600000D4648463AF000FA02460B46CDE90001C5
:10D6100000208E493AF0B4FFCDE9040120462946A6
:10D620003AF0FFF9CDE90201DDE904233AF0E6F82A
:10D6300000221346CDE906013AF0D4FAC4D90A22F1
:10D6400000232046294639F0D3FED0B20C900A229E
:10D6500000232046294639F0CBFE04460D461AE049
:10D66000A9F10101A1EB0B010DAA0C9850540BF18B
:10D67000010000F0FF0B0A2200232046294639F062
:10D68000B7FED0B20C900A2200232046294639F07A
:10D69000AFFE04460D4600210846091BA841DFDB0A
:10D6A000A9F10101A1EB0B010DAA0C9850540BF14B
:10D6B000010000F0FF0B00224FF080431046634949
:10D6C0003AF05EFFCDE90401384641463AF0A9F947
:10D6D000CDE90201DDE904233AF008F9CDE90601BC
:10D6E0003AF018FA04460D46002618E00A220023F4
:10D6F0002046294639F07CFED0B20C900A22002345
:10D700002046294639F074FE04460D4609EB0A010D
:10D71000491E891B0DAA0C985054701CC6B2564560
:10D72000E4DB002606E01F993144C8B2FFF71AFA7D
:10D73000701CC6B2A9EB0B00B042F4DC0A980128B9
:10D7400037D1A9EB0B00C0B209901E98401EC0B2A1
:10D750001E90099830B1012809D002280BD0032867
:10D7600011D10CE04FF48370FCF737FF10E0ED208F
:10D77000FCF733FF0CE0DE20FCF72FFF08E0C620AB
:10D78000FCF72BFF04E04FF48370FCF726FF00BF8B
:10D7900000BF099E09E00DAA915D1F9A3244521CF8
:10D7A000D0B2FCF757FF701CC6B21E988642F2DB5F
:10D7B0000FE0A9EB0B00C6B208E00DAA915D1F9A1D
:10D7C0003244D0B2FCF746FF701CC6B21E988642A7
:10D7D000F3DB14B0BDE8F09F2DE9FF5F86B017467C
:10D7E00098464FF0000B00221346384641463AF067
:10D7F000E1F909D24FF0010B3A46434600200146B9
:10D8000039F0FCFF074688460698002879D1BBF11D
:10D81000000F47D10F49611A75F100003EDB0E4839
:10D82000807AC0F3400080B30C48407C012874D05B
:10D8300001200A49487406210A202FF01DFD0648E0
:10D84000807AC0F34000002867D009E0000024403F
:10D850009F86010040548900EA2D0020581D0020B9
:10D86000F84890F87D00022802DA0120F549C877CF
:10D87000F44890F87D00FA284FDAF24890F87D00DD
:10D88000401CF04981F87D0047E0FFE70020EE49A9
:10D890004874EC49C87781F87D003EE00020EA49F1
:10D8A00048743AE0E9490020091BA84132DBE84806
:10D8B000807AC0F3400028B3E348407C01282CD094
:10D8C0000120E149487406210A202FF0D5FCE048E8
:10D8D000807AC0F3400000B3DA4890F87D00022857
:10D8E00002DA0120D749C877D64890F87D00FA2897
:10D8F00013DAD44890F87D00401CD24981F87D00AD
:10D900000BE029E10020D0494874CE49C87781F85E
:10D910007D0002E00020CC494874BBF1000F71D1BA
:10D9200003E0CC4AA41A65F10005CA49631A65F1FF
:10D93000000000221146D21A8141F2DB0A220023A4
:10D940002046294639F054FD02F0FF0A0A2200233E
:10D950002046294639F04CFD04460D4618E0C9F131
:10D96000060003A901F800A009F1010000F0FF0979
:10D970000A2200232046294639F03AFD02F0FF0A28
:10D980000A2200232046294639F032FD04460D467E
:10D9900000210846091BA841E1DBC9F1060003A9E3
:10D9A00001F800A009F1010000F0FF090022AA4BD4
:10D9B0003846414639F028FFCDE900013AF0AAF88F
:10D9C00004460D460A2200232046294639F010FD60
:10D9D000D0B28DF813000022A04B3846414639F0F2
:10D9E00013FFCDE900013AF095F804460D460A22EE
:10D9F00000232046294639F0FBFCD0B28DF81400F4
:10DA0000002606E018E0311DC8B2FFF7ABF8701C25
:10DA1000C6B2C9F10700B042F5DCC9F10700C6B2D1
:10DA200007E003AA915D321DD0B2FCF713FE701C13
:10DA3000C6B2092EF5DB8BE05220FCF7CEFD03E0E9
:10DA4000874AA41A65F100058549621A65F100004C
:10DA500000239A1A73EB0001F2DB0A2220462946C2
:10DA600039F0C6FC02F0FF0A0A22002320462946AC
:10DA700039F0BEFC04460D4618E0C9F1050003A9C3
:10DA800001F800A009F1010000F0FF090A220023BB
:10DA90002046294639F0ACFC02F0FF0A0A22002396
:10DAA0002046294639F0A4FC04460D4600210846CC
:10DAB000091BA841E1DBC9F1050003A901F800A099
:10DAC00009F1010000F0FF090022634B384641468E
:10DAD00039F09AFECDE900013AF01CF804460D46F3
:10DAE0000A2200232046294639F082FCD0B28DF864
:10DAF00012000022594B3846414639F085FECDE9E7
:10DB000000013AF007F804460D460A220023204699
:10DB1000294639F06DFCD0B28DF81300002605E0DF
:10DB2000711DC8B2FFF71EF8701CC6B2C9F106001D
:10DB3000B042F5DCC9F10600C6B207E003AA915D68
:10DB4000721DD0B2FCF786FD701CC6B2082EF5DB44
:10DB5000A820FCF742FDD2E1BBF1000F3AD13B49CE
:10DB6000611A75F1000031DB3948807AC0F340005A
:10DB700020B33548407C012879D0012032494874CF
:10DB800006210A202FF078FB3148807AC0F340004C
:10DB9000F8B12C4890F87D00022802DA01202949CA
:10DBA000C877284890F87D00FA2860DA254890F870
:10DBB0007D00401C234981F87D0058E00020224967
:10DBC00048742049C87781F87D0050E000201E4944
:10DBD00048744CE023490020091BA84144DB1C4841
:10DBE000807AC0F3400020B31748407C01283ED023
:10DBF00001201549487406210A202FF03DFB1448E6
:10DC0000807AC0F34000E0B10E4890F87D00022811
:10DC100002DA01200B49C8770A4890F87D00FA28FB
:10DC200025DA084890F87D00401C064981F87D00FF
:10DC30001DE00020044948740249C87781F87D003E
:10DC400015E014E090190020581D0020A0BB0D0025
:10DC5000EA2D0020809698000000244000005940E2
:10DC600040420F00905F01000020FB494874BBF167
:10DC7000000F7DD103E0F949641A65F10005F74909
:10DC8000621A65F1000000239A1A73EB0001F2DBBF
:10DC90000A222046294639F0ABFB02F0FF0A0A228D
:10DCA00000232046294639F0A3FB04460D4618E020
:10DCB000C9F1050003A901F800A009F1010000F075
:10DCC000FF090A2200232046294639F091FB02F081
:10DCD000FF0A0A2200232046294639F089FB044620
:10DCE0000D4600210846091BA841E1DBC9F10500EA
:10DCF00003A901F800A009F1010000F0FF090022CA
:10DD0000D74B3846414639F07FFDCDE9000139F067
:10DD100001FF04460D460A2200232046294639F019
:10DD200067FBD0B28DF812000022CE4B3846414638
:10DD300039F06AFDCDE9000139F0ECFE04460D46EC
:10DD40000A2200232046294639F052FBD0B28DF832
:10DD500013000022C44B3846414639F055FDCDE949
:10DD6000000139F0D7FE04460D460A22002300E0E8
:10DD700021E02046294639F03BFBD0B28DF8140053
:10DD8000002605E0311DC8B2FEF7ECFE701CC6B2DD
:10DD9000C9F10600B042F5DCC9F10600C6B207E0E1
:10DDA00003AA915D321DD0B2FCF754FC701CC6B2C0
:10DDB000092EF5DBA0E05220FCF70FFC03E0AB4A94
:10DDC000A41A65F10005A949621A65F10001002352
:10DDD0009A1A73EB0100F2DB0A222046294639F039
:10DDE00007FB02F0FF0A0A2200232046294639F0E9
:10DDF000FFFA04460D4618E0C9F1040003A901F832
:10DE000000A009F1010000F0FF090A2200232046CA
:10DE1000294639F0EDFA02F0FF0A0A2200232046D3
:10DE2000294639F0E5FA04460D4600210846091B4B
:10DE3000A841E1DBC9F1040003A901F800A009F140
:10DE4000010000F0FF090022854B3846414639F0B9
:10DE5000DBFCCDE9000139F05DFE04460D460A22E7
:10DE600000232046294639F0C3FAD0B28DF81100BC
:10DE700000227C4B3846414639F0C6FCCDE9000112
:10DE800039F048FE04460D460A2200232046294662
:10DE900039F0AEFAD0B28DF812000022724B38463B
:10DEA000414639F0B1FCCDE9000139F033FE0446BA
:10DEB0000D460A2200232046294639F099FAD0B2AD
:10DEC0008DF81300002605E0711DC8B2FEF74AFE6A
:10DED000701CC6B2C9F10500B042F5DCC9F10500FD
:10DEE000C6B207E003AA915D721DD0B2FCF7B2FB87
:10DEF000701CC6B2082EF5DBB820FCF76EFB0AB02A
:10DF0000BDE8F09F2DE9F04F87B08346174698464D
:10DF10004FF000093846414639F0FCFD04460D46F5
:10DF2000BBF1020F78D104E042F21072A41A65F13D
:10DF3000000542F21071621A65F1000000239A1A7E
:10DF400073EB0001F0DB0A222046294639F050FA33
:10DF500002F0FF0A0A2200232046294639F048FA37
:10DF600004460D4618E0C9F1030004A901F800A019
:10DF700009F1010000F0FF090A220023204629468A
:10DF800039F036FA02F0FF0A0A2200232046294619
:10DF900039F02EFA04460D4600210846091BA84117
:10DFA000E1DBC9F1030004A901F800A009F10100B7
:10DFB00000F0FF0900222A4B3846414639F024FC84
:10DFC000CDE9020139F0A6FD04460D460A220023E0
:10DFD0002046294639F00CFAD0B28DF81400002200
:10DFE000214B3846414639F00FFC00221C4BCDE94D
:10DFF000000139F07BFCCDE9020139F08BFD0446CC
:10E000000D460A2200232046294639F0F1F9D0B204
:10E010008DF81500002607E02AE006F10D01C8B2D0
:10E02000FEF7A0FD701CC6B2C9F10400B042F4DCDA
:10E03000C9F10400C6B208E004AA915D06F10D0220
:10E04000D0B2FCF707FB701CC6B2062EF4DBBF2073
:10E05000FCF7C3FABDE00000581D002040420F004D
:10E06000000024400000594000408F40A08601007D
:10E0700004E04FF47A72A41A65F100054FF47A7146
:10E08000621A65F1000100239A1A73EB0100F0DBBC
:10E090000A222046294639F0ABF902F0FF0A0A228B
:10E0A00000232046294639F0A3F904460D4618E01E
:10E0B000C9F1020004A901F800A009F1010000F073
:10E0C000FF090A2200232046294639F091F902F07F
:10E0D000FF0A0A2200232046294639F089F904461E
:10E0E0000D4600210846091BA841E1DBC9F10200E9
:10E0F00004A901F800A009F1010000F0FF090022C5
:10E10000FC4B3846414639F07FFBCDE9020139F03E
:10E1100001FD04460D460A2200232046294639F017
:10E1200067F9D0B28DF813000022F34B3846414610
:10E1300039F06AFB0022EF4BCDE9000139F0D6FB44
:10E14000CDE9020139F0E6FC04460D460A2200231F
:10E150002046294639F04CF9D0B28DF8140000223F
:10E16000E64B3846414639F04FFB0022E14BCDE902
:10E17000000139F0BBFBCDE9020139F0CBFC0446CC
:10E180000D460A2200232046294639F031F9D0B243
:10E190008DF81500002606E006F10D01C8B2FEF765
:10E1A000E1FC701CC6B2C9F10300B042F4DCC9F155
:10E1B0000300C6B208E004AA915D06F10D02D0B2D8
:10E1C000FCF748FA701CC6B2062EF4DBD720FCF729
:10E1D00004FA07B0BDE8F08F2DE9FC4782460E46F1
:10E1E0000024A0460025002000900190BAF1090FFC
:10E1F0002ED2DFE80AF0052E4CBCFD4DBDFCFB0025
:10E2000005210846FCF726FA1320FCF7E6F918204A
:10E21000FCF7E3F9F020FCF7E0F9C820FCF7DDF9A2
:10E22000A820FCF7DAF9002410E0325D1109620041
:10E23000921DD0B2FCF70EFA325D02F00F016200BF
:10E24000D21DD0B2FCF706FA601CC4B2042CECDB81
:10E2500082E1E920FCF7C1F9B220FCF7BEF9002405
:10E2600012E0325D110904EB4402921DD0B2FCF7BA
:10E27000F1F9325D02F00F0104EB4402D21DD0B27D
:10E28000FCF7E8F9601CC4B2032CEADB64E100BFD0
:10E290001220FCF7A2F91020FCF79FF93B20FCF7B5
:10E2A0009CF93A20FCF799F91920FCF796F91B2004
:10E2B000FCF793F91A20FCF790F94FF48170FCF702
:10E2C0008CF94FF48070FCF788F9C820FCF785F9C9
:10E2D000002449E0375D0A2097FBF0F100FB117044
:10E2E00000F0FF090A2097FBF0F700250FE0C5F1C9
:10E2F00002000DF80090681CC5B20A2097FBF0F1EF
:10E3000000FB117000F0FF090A2097FBF0F7002FC7
:10E31000EDDCC5F102000DF80090681CC5B2012DBE
:10E3200002D0022D08D103E000208DF8010000BFCB
:10E3300000208DF8000000E000BF00BF4FF0000893
:10E340000DE01DF8081008F10702032303FB042267
:10E35000D0B2FCF77FF908F1010000F0FF08B8F136
:10E36000030FEEDB601CC4B2022CB3DBF4E000BF91
:10E370000B20FCF732F91220FCF72FF90920FCF7EB
:10E380002CF90A20FCF729F91120FCF726F91320B3
:10E39000FCF723F91820FCF720F93178707801EBAD
:10E3A00000270A2097FBF0F100FB117000F0FF0935
:10E3B0000A2097FBF0F70FE0C5F104000DF800907C
:10E3C000681CC5B20A2097FBF0F100FB117000F049
:10E3D000FF090A2097FBF0F7002FEDDCC5F10400E0
:10E3E0000DF80090681CC5B2012D02E04EE02FE050
:10E3F0002DE006D0022D08D0032D0AD0042D10D117
:10E400000BE000208DF8030000BF00208DF8020013
:10E4100000BF00208DF8010000BF00208DF8000033
:10E4200000E000BF00BFC5F1050000F0FF080AE0F2
:10E430001DF8081008F10602D0B2FCF70BF908F13C
:10E44000010000F0FF08B8F1050FF1DB84E000BF28
:10E45000307800F00F010520FCF7FCF8002412E0F2
:10E46000621CB25C11096200921DD0B2FCF7F2F896
:10E47000621CB25C02F00F016200D21DD0B2FCF748
:10E48000E9F8601CC4B2042CEADB65E00821052031
:10E49000FCF7E0F83B20FCF7A0F83A20FCF79DF8E9
:10E4A0001920FCF79AF81B20FCF797F81A20FCF7C4
:10E4B00094F805210720FCF7CDF8F220FCF78DF841
:10E4C000F020FCF78AF8F0780006B17840EA0140C5
:10E4D000717840EA0120317840EA01070A2097FB71
:10E4E000F0F100FB117000F0FF090A2097FBF0F734
:10E4F00016E000000000244000408F400088C34028
:10E50000C5F105000DF80090681CC5B20A2097FB04
:10E51000F0F100FB117000F0FF090A2097FBF0F703
:10E52000002FEDDCC5F105000DF80090681CC5B2A8
:10E53000C5F1060000F0FF080AE01DF8081008F118
:10E540000802D0B2FCF786F808F1010000F0FF08DD
:10E55000B8F1060FF1DB00BF00BFBDE8FC872DE975
:10E56000FC4782460D460024A0460026002000906D
:10E570000190BAF1090F3BD2DFE80AF0053B5DB02C
:10E58000B25EB1B3C900FD20FCF727F8FE20FCF70E
:10E5900024F840F20710FCF720F840F20510FCF7D1
:10E5A0001CF84FF48370FCF718F8F520FCF715F809
:10E5B000F720FCF712F8D720FCF70FF8002410E042
:10E5C0002A5D110962000F32D0B2FCF743F82A5DD0
:10E5D00002F00F0162001032D0B2FCF73BF8601C71
:10E5E000C4B2022CECDB285D01091320FCF732F8E1
:10E5F000DCE0E520FBF7F1FFE720FBF7EEFFC420AE
:10E60000FBF7EBFFBF20FBF7E8FF002410E02A5DDB
:10E61000110962000E32D0B2FCF71CF82A5D02F03C
:10E620000F0162000F32D0B2FCF714F8601CC4B2C4
:10E63000032CECDBBAE000BFD720FBF7CEFF0024B1
:10E6400049E02F5D0A2097FBF0F100FB117000F00C
:10E65000FF090A2097FBF0F700260FE0C6F1020041
:10E660000DF80090701CC6B20A2097FBF0F100FB79
:10E67000117000F0FF090A2097FBF0F7002FEDDC86
:10E68000C6F102000DF80090701CC6B2012E02D037
:10E69000022E08D103E000208DF8010000BF002009
:10E6A0008DF8000000E000BF00BF4FF000080DE053
:10E6B0001DF8081008F10E02032303FB0422D0B258
:10E6C000FBF7C8FF08F1010000F0FF08B8F1030FE5
:10E6D000EEDB601CC4B2022CB3DB67E000BF65E078
:10E6E00000BF002410E02A5D110962000E32D0B292
:10E6F000FBF7B0FF2A5D02F00F0162000F32D0B2CB
:10E70000FBF7A8FF601CC4B2042CECDB4EE0052133
:10E710000E20FBF79FFFF520FBF75FFFF720FBF7CD
:10E720005CFF2F780A2097FBF0F100FB117000F0DE
:10E73000FF090A2097FBF0F70FE0C6F102000DF881
:10E740000090701CC6B20A2097FBF0F100FB11701C
:10E7500000F0FF090A2097FBF0F7002FEDDCC6F16F
:10E7600002000DF80090701CC6B2012E02D0022EDD
:10E7700008D103E000208DF8010000BF00208DF8D3
:10E78000000000E000BF00BF4FF000080AE01DF8E5
:10E79000081008F10F02D0B2FBF75CFF08F101008E
:10E7A00000F0FF08B8F1030FF1DB00BF00BFBDE8C8
:10E7B000FC8702460B4600207047704738B5054677
:10E7C000992D1FDC55B9002405E0611CC8B2FEF785
:10E7D000C9F9601CC4B2022CF7DB13E005F00F008E
:10E7E0008DF80100C5F307108DF80000002407E044
:10E7F0001DF80410621CD0B2FBF72CFF601CC4B2E1
:10E80000022CF5DB38BD38B5054655B9002405E0C6
:10E81000A11CC8B2FEF7A6F9601CC4B2022CF7DB3B
:10E8200012E005F00F008DF8010028118DF80000AE
:10E83000002407E01DF80410E21CD0B2FBF70AFF29
:10E84000601CC4B2022CF5DB38BD10B5044634B1EF
:10E85000012C09D0022C0BD0032C0ED109E04FF46F
:10E860008A70FBF7BAFE09E03F20FBF7B6FE05E031
:10E8700004E05720FBF7B1FE00E000BF00BF10BD71
:10E8800010B5044634B1012C09D0022C0BD0032C56
:10E890000ED109E04FF48A70FBF7B8FE09E03F2083
:10E8A000FBF7B4FE05E004E05720FBF7AFFE00E005
:10E8B00000BF00BF10BD10B504462046FBF78DFE1B
:10E8C000FE48FBF74AFE10BD10B5002404E0FF200F
:10E8D000FA490855601C84B2232CF8DBF748FBF793
:10E8E0003CFE10BD10B504462046FBF78FFEF348F2
:10E8F000FBF733FE10BD10B500244FF48A70FBF710
:10E900006CFE3C20FBF769FE4320FBF766FE4420CB
:10E91000FBF763FEEA4890F86300012803D1422028
:10E92000FBF75BFE07E0E64890F86300022802D19F
:10E930004920FBF752FEE34890F8090110B140204E
:10E94000FBF74BFEE0488079C0F3401018B14FF45C
:10E950008970FBF742FEDC48C0790221B1EB901FC1
:10E9600003D140F21110FBF738FED548007C012896
:10E9700003D14820FBF731FE02E04820FBF746FEBA
:10E98000D248007B00F00400042804D140F20D10AE
:10E99000FBF723FE03E04FF48670FBF71EFE40F208
:10E9A0001510FBF71AFEC648407E462810DD4FF4CE
:10E9B0008770FBF712FE40F20F10FBF70EFE40F2DD
:10E9C0001710FBF70AFE4FF48B70FBF706FE25E0ED
:10E9D000BB48407E28280CDD4FF48770FBF7FDFD17
:10E9E00040F20F10FBF7F9FD40F21710FBF7F5FDB1
:10E9F00014E0B348407E142808DD4FF48770FBF71D
:10EA0000ECFD40F20F10FBF7E8FD07E0AC48407E5C
:10EA1000002803DD4FF48770FBF7DFFDAC488078FA
:10EA200010B90620FBF7D9FDA948407804282FD05B
:10EA300006DC012809D002280ED0032854D117E0A3
:10EA4000052835D063284FD140E00520FBF7C5FDF0
:10EA50000720FBF7C2FD48E00520FBF7BEFD0420C0
:10EA6000FBF7BBFD9A49B1F80B00FFF7A7FE3CE0AE
:10EA70000520FBF7B2FD9548007B00F0010018B1BE
:10EA80000720FBF7AAFD02E00720FBF7BFFD2CE003
:10EA90000520FBF7A2FD8D48007B00F0010018B1B6
:10EAA0000420FBF79AFD02E00420FBF7AFFD1CE019
:10EAB0008648007B00F00200022803D10520FBF706
:10EAC0008CFD02E00520FBF7A1FD0EE07F48007BF6
:10EAD00000F00400042803D10520FBF77EFD02E0CE
:10EAE0000520FBF793FD00E000BF00BF7748C07C26
:10EAF0000A2833DA00241DE07448C17C704846308F
:10EB0000405C50B15720FBF768FD7049CA7C6C49E6
:10EB10004631885CFFF777FE0EE06C48C07C401CF5
:10EB20006A49C8740846C07C0A2801DB0020C87402
:10EB3000601CC4B20A2CDFDB00BF6448007B00F01D
:10EB40000100D0B96148C07C401C6049C8740846C7
:10EB5000C07C0A2811DB0020C8740EE000205B494D
:10EB6000C874574890F8460038B15720FBF735FD78
:10EB7000534991F84600FFF746FE4720FBF72DFD6D
:10EB80005448C07919280FDD4620FBF726FD4520A3
:10EB9000FBF723FD4D20FBF720FD4E20FBF71DFD6D
:10EBA0004F20FBF71AFD40E04A48C079152810DBDA
:10EBB0004848C07919280CDC4620FBF70EFD45209B
:10EBC000FBF70BFD4D20FBF708FD4E20FBF705FD85
:10EBD0002BE04048C07910280DDB3E48C07914284E
:10EBE00009DC4620FBF7F9FC4520FBF7F6FC4D203D
:10EBF000FBF7F3FC19E03748C0790B280ADB3548EE
:10EC0000C0790F2806DC4620FBF7E7FC4520FBF720
:10EC1000E4FC0AE02F48C079002806DD2D48C079C1
:10EC20000B2802DA4620FBF7D8FC2548007A012899
:10EC30000CD12948807800F0010018B13F20FBF783
:10EC4000CCFC0EE03F20FBF7E1FC0AE01C4890F80A
:10EC5000450018B93F20FBF7C0FC02E03F20FBF75E
:10EC6000D5FC10BD2DE9FC410446052C7ED2DFE821
:10EC700004F0450386C0FB000320FBF7AEFC8320B5
:10EC8000FBF7ABFC4FF48470FBF7A7FC8520FBF788
:10EC9000A4FC8420FBF7A1FC05200921CDE900108C
:10ECA00008488030056843682A460220FEF760F96C
:10ECB0000449D1F8880038F0A7FE0FE0D20F0020F9
:10ECC000A21600208E220020D22D0020581D0020E8
:10ECD000D94700203A1F00200C00002007460022E0
:10ECE000CE4B38F003FE05460B460E2007212A4680
:10ECF000CDE900100320FEF780FBEFE00120FBF7D9
:10ED00006CFC0020FBF769FC8B20FBF766FC822083
:10ED1000FBF763FC8E20FBF760FC8720FBF75DFCB4
:10ED20008620FBF75AFCBE4890F8090158B9052027
:10ED30000921CDE90010BA48856AC36A2A46022033
:10ED4000FEF716F90AE005200921CDE90010B449C3
:10ED50008D6CCB6C2A460220FEF70AF9B049486F49
:10ED600038F015FF05460B460E2000E0B5E0072100
:10ED70002A46CDE900100220FEF73FFBAEE001205D
:10ED8000FBF72BFC0020FBF728FC8B20FBF725FC76
:10ED90008220FBF722FC8120FBF71FFCA04890F8A3
:10EDA000090158B905200921CDE900109C48856A60
:10EDB000C36A2A460220FEF7DBF80AE00520092193
:10EDC000CDE9001096498D6CCB6C2A460220FEF7E7
:10EDD000CFF89349D1F8980038F0D9FE05460B4694
:10EDE0000E2007212A46CDE900100220FEF705FB80
:10EDF00074E00120FBF7F1FB0020FBF7EEFB8B201A
:10EE0000FBF7EBFB8220FBF7E8FB8C20FBF7E5FB35
:10EE1000834890F8090158B905200921CDE900106F
:10EE20007F48856AC36A2A460220FEF7A1F80AE0F5
:10EE300005200921CDE900107948856CC36C2A466C
:10EE40000220FEF795F87649D1F89C0038F09FFE35
:10EE500005460B460E2007212A46CDE90010022068
:10EE6000FEF7CBFA3AE0FFE70220FBF7B6FB002003
:10EE7000FBF7B3FB8220FBF7B0FB8720FBF7ADFB72
:10EE80008620FBF7AAFB664890F8090158B90520CF
:10EE90000921CDE9001062490D6A4B6A2A46022019
:10EEA000FEF766F80AE005200921CDE900105C486C
:10EEB000056C436C2A460220FEF75AF85849086F41
:10EEC00038F065FE05460B460E2007212A46CDE99F
:10EED00000100220FEF791FA00E000BF00BFBDE87D
:10EEE000FC813CB505465020FBF777FB092D7DD210
:10EEF000DFE805F0050F193C5223425C86004949C2
:10EF00000020FFF769F94749491F0020FFF727FB59
:10EF100081E045490120FFF75FF94349C91C012001
:10EF2000FFF71DFB77E041490220FFF755F93F4904
:10EF3000891C0220FFF713FB6DE03D480078012893
:10EF400009D13C490520FFF747F93A49891C0520BA
:10EF5000FFF705FB09E0374919310520FFF73CF9B8
:10EF600034491B310520FFF7FAFA54E02F49091DF7
:10EF70000320FFF731F94EE02D480078012805D134
:10EF80002C49091D0620FFF727F904E029491D3106
:10EF90000620FFF721F93EE027490420FFF71CF97E
:10EFA0002549491D0420FFF7DAFA34E022484138A8
:10EFB00090F84D003038C0B28DF80000002411E008
:10EFC0006000001D1C490A31085C30386100C91C12
:10EFD000194A0A32515C00EB0110C1B2601C0DF8F5
:10EFE0000010C4B2072CEBDB694600E012E00720FA
:10EFF000FFF7F2F80DF105010720FFF7B0FA0AE07C
:10F000000E490820FFF7E8F80C49491E0820FFF7D1
:10F01000A6FA00E000BF00BF3CBD00000088C3406E
:10F020008E22002096270020140000203D2C002076
:10F03000F04600202645002061270020E90000203E
:10F0400008B50120ADF8000010208DF80300032062
:10F050008DF802006946FE4801F0D8FD08BD08B5EC
:10F060000120ADF8000000208DF8030003208DF88A
:10F0700002006946F64801F0C9FD08BD08B5402008
:10F08000ADF8000048208DF8030003208DF8020041
:10F090006946EF4801F0BAFD08BD08B54020ADF85B
:10F0A000000000208DF8030003208DF8020069465F
:10F0B000E74801F0ABFD08BD08B50420ADF800003D
:10F0C0008DF8030003208DF802006946E04801F046
:10F0D0009DFD08BD08B50420ADF8000000208DF8A6
:10F0E000030003208DF802006946D94801F08EFD27
:10F0F00008BD08B54FF40070ADF8000010208DF881
:10F10000030003208DF802006946D24801F07EFD1D
:10F1100008BD08B54FF48060ADF8000010208DF8F0
:10F12000030003208DF802006946CA4801F06EFD15
:10F1300008BD08B54FF40070ADF8000000208DF850
:10F14000030003208DF802006946C24801F05EFD0D
:10F1500008BD08B54FF48060ADF8000000208DF8C0
:10F16000030003208DF802006946BA4801F04EFD05
:10F1700008BD10B5FFF7BDFF0120B74908604FF487
:10F18000FA70F9F798F90020B449C1F8A40110BD4C
:10F1900010B5FFF7AEFF0120AF49086010BD10B5F4
:10F1A000FFF7A7FF0020AC49086010BD10B5FFF7BE
:10F1B000B0FF0120A849091D08604FF4FA70F9F763
:10F1C0007AF90020A549C1F8A80110BD10B5FFF7D4
:10F1D000A0FF0120A049091D086010BD10B5FFF770
:10F1E00098FF00209C49091D086010BD9848806860
:10F1F00000F00401890809B9002070470120FCE7EC
:10F2000010B59748807A012802D19549087402E028
:10F210000020934908749248407A01280FD1904801
:10F22000408A30B901208E49C8734FF4616048822A
:10F2300008E08B48408A401E8949488202E000204D
:10F24000874948828648007C012802D1FFF7A0FF49
:10F2500005E00020834981F83400FFF7A0FF8048D3
:10F26000C07B012826D17F4890F835000F2807DAA7
:10F270007C4890F83500401C7A4981F8350006E05A
:10F2800000207749C8730F20764981F8350075480A
:10F2900090F83500032802DAFFF7A0FF10E071486C
:10F2A00090F835000D2802DAFFF790FF08E0FFF72D
:10F2B00095FF05E000206B4981F83500FFF78EFFD0
:10F2C00010BD2DE9F05F6648807A012803D1002047
:10F2D0006449487685E06248407A012861D16048F7
:10F2E0008079012816D15F49498E46F2A862501AEA
:10F2F00038F079FB804600225B4B38F085FA0646F1
:10F3000000225A4B38F0F2FA044638F0EAFB55492D
:10F31000487637E052484079012833D15148B0F857
:10F3200017005349097801EB8101B0EB410F26DC4E
:10F330004F4909784E4A5278891A01EB81014800F9
:10F3400038F051FB04460D464649B1F81710484ABB
:10F35000527802EB8202A1EB420038F044FB0646F1
:10F360000022444B38F050FA804622462B4638F0B3
:10F37000BDFA824638F0B5FB3A49487602E01420DF
:10F38000384948763748407E142802DD1420354934
:10F3900048763448407E002823DA002031494876F8
:10F3A0001FE03048408E46F2A861884216DA2D49A7
:10F3B000498E46F2A862501A38F015FB80460022AA
:10F3C000294B38F021FA06460022284B38F08EFAF5
:10F3D000044638F086FB2349487602E000202149A4
:10F3E00048762048407E642802DD64201D49487626
:10F3F000BDE8F09F70B52048007817280AD11E4854
:10F400004078392806D11C488078022802DA012089
:10F410001349087012480078012807D01048407836
:10F42000012803D00E48007B012806D101200C4999
:10F430008870002008704870087309488078012897
:10F4400030D10748C0780A281BD10020044915E0B4
:10F450000010014000180140A40123420000234293
:10F46000F60F0020A21600200000594000AAD94043
:10F47000F2000020000034400C0000208870C870AA
:10F4800004E0F848C078401CF649C870F548C078D8
:10F49000012808D1FFF7D4FD0120F9F70CF801206D
:10F4A000F14908609EE0EF48C0780228FAD1EF48A1
:10F4B000B0F81700EE49097801EB8101B0EB410F7C
:10F4C0000EDB04F013F8E948B0F81700E8490978B2
:10F4D00001EB8101B0EB410F04DA04F007F801E021
:10F4E00004F004F80020E0490860DE48407B022870
:10F4F00036D10020DB494873DC48B0F81700DC49FE
:10F50000497801EB8101B0EB410F21DDD548807BCB
:10F51000012867D00120D3498873122102202DF0E1
:10F52000ABFE06F094FBD34890F86D00022802DA97
:10F530000120D049C873CF4890F86D00FA2851DAFD
:10F54000CC4890F86D00401CCA4981F86D0049E034
:10F550000020C4498873C749C87381F86D0041E031
:10F56000C048407B012823D10020BE494873C248CF
:10F570000079C0F38000A8B3BC48B0F81700BC49BC
:10F58000497801EB8101322202EB4101884229DDF9
:10F59000B448807B012825D10020B2498873B54941
:10F5A000C87381F86D00012102202DF065FE19E07D
:10F5B000FFF764FDAC4868380068012812D1A948FB
:10F5C000807B01280ED10A20F8F775FFA64868381D
:10F5D0000068012806D10020A2498873A549C87394
:10F5E00081F86D009F48C07A01281FD100209D49F5
:10F5F000C8729E49B1F8170038F006FA0446002296
:10F600009E4B38F0EFFA11D8002142F66400FAF769
:10F6100012FA002142F66800FAF70DFA0020934929
:10F6200008864886012102202DF026FE8F48007CA6
:10F63000E8BB8E48008E401C8C4908860846008E28
:10F64000B0F5616F1BDB002008860846408E401C29
:10F6500048860846408E4FF6FA71884202DD002047
:10F66000824948868148018E42F66400FAF7E3F940
:10F670007E48418E42F66800FAF7DDF90EE07B48DD
:10F68000008E4FF4167190FBF1F201FB120028B9C5
:10F690007648018E42F66400FAF7CDF97348408E41
:10F6A0004FF6FA71884202DD0020704948866F48A3
:10F6B000B0F817006E49097801EB8101B0EB410FFA
:10F6C00003DA0120674948710EE06848B0F8170076
:10F6D0006749097801EB8101142202EB410188425C
:10F6E00002DD00205F4948716048B0F817006049AA
:10F6F000497801EB8101B0EB410F03DA0120594950
:10F70000C8710EE05948B0F817005949497801EB23
:10F710008101142202EB4101884202DD002051499F
:10F72000C8715248408E46F2A861884203DB01202E
:10F730004C49087211E04D49488E38F065F904468D
:10F7400000224F4B38F04EFA03D80120454988710A
:10F7500003E00020434908728871424880790128FB
:10F7600003D04048407901282CD14348007900F06B
:10F770000100F8B13B48407A01282ED001203949D8
:10F780004872102102202DF077FD3A4890F8610070
:10F79000022802DA01203749C870364890F8610023
:10F7A000FA281ADA334890F86100401C314981F890
:10F7B000610012E000202B4948722E49C87081F880
:10F7C00061000AE02748407A38B100202549487294
:10F7D00041F2100102202DF04FFD2248C07901288E
:10F7E00003D02048007A01282ED106F030FA2248B2
:10F7F0000079C0F34000F8B11A48807A01282ED071
:10F80000012018498872112102202DF035FD194878
:10F8100090F86200022802DA0120164908711548A2
:10F8200090F86200FA281ADA124890F86200401C38
:10F83000104981F8620012E000200A4988720D49DF
:10F84000087181F862000AE00648807A38B1002029
:10F850000449887241F2110102202DF00DFDFFF7DD
:10F8600030FD70BDF60F002080012242A21600205C
:10F87000F200002090190020EA2D002000001C401A
:10F880000088D44010B500215D4803F048F84FF4DB
:10F890007A715B4803F058F80121594803F03FF8AA
:10F8A00010BD704710B590B004460121880401F0E6
:10F8B00076FC0121084601F058FC524802F05EFD3A
:10F8C0000C940020ADF83400ADF83600ADF83800E7
:10F8D000ADF83C000C20ADF83A000CA9494802F004
:10F8E00090FD474802F04EFF4648001D01904648F3
:10F8F0000290002003904FF47A700490002005904D
:10F9000080200690002007900890202009904FF456
:10F9100040500A9000200B9001A9394802F0D4FF12
:10F9200001224021374802F029FE0121344802F02B
:10F93000F6FF0121334802F0F0FD40F22661314824
:10F9400002F006FF10B010BD10B500212C4802F0E7
:10F95000E6FF4FF47A712A4802F0F6FF01212848A9
:10F9600002F0DDFF4FF47A71274837F09EFD4FF427
:10F970008071264837F099FD10BD2DE9F04104460D
:10F980000D46274600260DE039781E4802F032FE6B
:10F990007F1C00BF40211B4802F09AFE0028F9D0CE
:10F9A000701C86B2AE42EFDBBDE8F0812DE9F0417C
:10F9B00005460E462F461648C079012804D001207E
:10F9C00014490860F8F777FD40210E4802F08DFEDB
:10F9D00000240DE039780B4802F00CFE7F1C00BFBC
:10F9E0004021084802F074FE0028F9D0601C84B25F
:10F9F000B442EFDB002007490860BDE8F081000059
:10FA000030000240004800400C1000200448002054
:10FA1000A2160020880123420146FE48405C704740
:10FA20000146FD48405C7047F8B5002429E00020FD
:10FA300000EB8400F9490968085C002101EB8401AE
:10FA4000F74A5054012000EB8400F4490968085C2F
:10FA5000012101EB84015054022000EB8400EF49A6
:10FA60000968085C022101EB84015054032000EB7B
:10FA70008400EA490968085C032101EB84015054C1
:10FA8000641C042CD3D378E0002507E0601E05EB4E
:10FA90008000E349085C0DF805006D1C042DF5D3CA
:10FAA00004F0030088BB9DF800609DF801008DF80C
:10FAB00000009DF802008DF801009DF803008DF80C
:10FAC00002008DF803609DF80000FFF7A5FF8DF898
:10FAD00000009DF80100FFF79FFF8DF801009DF8E1
:10FAE0000200FFF799FF8DF802009DF80300FFF771
:10FAF00093FF8DF803009DF80000CA4901EB9401C3
:10FB0000097848408DF8000001E0FFE700BF201FA2
:10FB1000002101EB8000C249085C9DF800104840BC
:10FB2000002101EB8401BE4A5054201F012101EB4A
:10FB300080001146085C9DF801104840012101EB4E
:10FB400084015054201F022101EB80001146085C03
:10FB50009DF802104840022101EB84015054201FFF
:10FB6000032101EB80001146085C9DF8031048401A
:10FB7000032101EB84015054641C2C2C84D3F8BD68
:10FB800010B50246002018E0002112E0130103EB3B
:10FB900080030B44A24CE35CA34C246804EB800478
:10FBA000645C6340A04C246804EB800463544B1CE9
:10FBB000D9B20429EADB431CD8B20428E4DB10BD27
:10FBC00070B5002413E000250DE09749096801EBAA
:10FBD0008501085DFFF720FF9349096801EB850166
:10FBE0000855681CC5B2042DEFDB601CC4B2042CA0
:10FBF000E9DB70BD8C49096848788B490968497907
:10FC0000894A12685170884909684A7A86490968A0
:10FC10004A71854909684A7B834909684A72824961
:10FC2000096848738049096888787F490968897A32
:10FC30007D4A126891707C49096888727A4909681E
:10FC40008879794909688A7B774909688A71764990
:10FC50000968887374490968C87873490968C97B59
:10FC6000714A1268D17070490968CA7A6E49096888
:10FC7000CA736D490968CA796B490968CA726A49C9
:10FC80000968C87170470146C80900EBC00000EB65
:10FC9000400080EA4100C0B270472DE9F0410024E5
:10FCA00088E06148006810F824705F48006810F828
:10FCB00024005D49096801EB8401497848405A49AC
:10FCC000096801EB8401897848405749096801EBCC
:10FCD0008401C97880EA01055348006810F82400BF
:10FCE0005149096801EB8401497880EA01063046F0
:10FCF000FFF7C9FF06464C48006810F8240086EA62
:10FD0000050148404849096801F824004648006850
:10FD100000EB840040784449096801EB840189784C
:10FD200080EA01063046FFF7AEFF06463E4800680F
:10FD300000EB8400407886EA050148403A490968AA
:10FD400001EB840148703848006800EB840080783B
:10FD50003549096801EB8401C97880EA010630461B
:10FD6000FFF791FF06463048006800EB840080787A
:10FD700086EA050148402C49096801EB8401887036
:10FD80002948006800EB8400C07880EA0706304606
:10FD9000FFF779FF06462448006800EB8400C0782E
:10FDA00086EA050148402049096801EB8401C870D2
:10FDB000601CC4B2042CFFF674AFBDE8F08130B50E
:10FDC00089B00020089059E217480168089811F896
:10FDD0002000079014480168089801EB80004078E3
:10FDE000069011480168089801EB80008078059022
:10FDF0000D480168089801EB8000C07804900798CE
:10FE0000FFF741FF04460798FFF73DFF0390FFF718
:10FE10003AFF0BE054450508544605082C00002025
:10FE20001415002054470508280000204440079876
:10FE3000FFF729FF0290FFF726FF0390FFF723FF4C
:10FE400044400798FFF71FFF0190FFF71CFF029047
:10FE5000FFF719FF0390FFF716FF0698FFF713FF50
:10FE6000054606984540FFF70EFF0390FFF70BFF8E
:10FE70000698FFF708FF0290FFF705FF0390FFF7D2
:10FE800002FF45400698FFF7FEFE0190FFF7FBFEDC
:10FE90000290FFF7F8FE0390FFF7F5FE6C4005981F
:10FEA000FFF7F1FE05980546FFF7EDFE0390FFF71B
:10FEB000EAFE45400598FFF7E6FE0290FFF7E3FEF5
:10FEC0000390FFF7E0FE45400598FFF7DCFE019048
:10FED000FFF7D9FE0290FFF7D6FE0390FFF7D3FE9F
:10FEE0006C400498FFF7CFFE04980546FFF7CBFE61
:10FEF0000390FFF7C8FE0498FFF7C5FE0290FFF7D6
:10FF0000C2FE0390FFF7BFFE45400498FFF7BBFE1B
:10FF10000190FFF7B8FE0290FFF7B5FE0390FFF7E0
:10FF2000B2FE6C40FE480168089801F8204007982E
:10FF3000FFF7A9FE07980446FFF7A5FE0390FFF719
:10FF4000A2FE0798FFF79FFE0290FFF79CFE03902A
:10FF5000FFF799FE44400798FFF795FE0190FFF7E1
:10FF600092FE0290FFF78FFE0390FFF78CFE06983B
:10FF7000FFF789FE05460698FFF785FE0390FFF719
:10FF800082FE45400698FFF77EFE0290FFF77BFE5B
:10FF90000390FFF778FE45400698FFF774FE019046
:10FFA000FFF771FE0290FFF76EFE0390FFF76BFE06
:10FFB0006C400598FFF767FE054605984540FFF73A
:10FFC00062FE0390FFF75FFE0598FFF75CFE02906C
:10FFD000FFF759FE0390FFF756FE45400598FFF7DF
:10FFE00052FE0190FFF74FFE0290FFF74CFE039088
:10FFF000FFF749FE6C400498FFF745FE049805465C
:020000040801F1
:10000000FFF741FE0390FFF73EFE45400498FFF7DF
:100010003AFE0290FFF737FE0390FFF734FE4540AB
:100020000498FFF730FE0190FFF72DFE0290FFF7D6
:100030002AFE0390FFF727FE6C40B9480168089834
:1000400001EB800044700798FFF71DFE07980446F7
:10005000FFF719FE0390FFF716FE44400798FFF7DD
:1000600012FE0290FFF70FFE0390FFF70CFE4440D4
:100070000798FFF708FE0190FFF705FE0290FFF7D3
:1000800002FE0390FFF7FFFD0698FFF7FCFD0698C0
:100090000546FFF7F8FD0390FFF7F5FD0698FFF71B
:1000A000F2FD0290FFF7EFFD0390FFF7ECFD4540F6
:1000B0000698FFF7E8FD0190FFF7E5FD0290FFF7D6
:1000C000E2FD0390FFF7DFFD6C400598FFF7DBFDD5
:1000D00005460598FFF7D7FD0390FFF7D4FD45408F
:1000E0000598FFF7D0FD0290FFF7CDFD0390FFF7D5
:1000F000CAFD45400598FFF7C6FD0190FFF7C3FD17
:100100000290FFF7C0FD0390FFF7BDFD6C4004981F
:10011000FFF7B9FD054604984540FFF7B4FD03908D
:10012000FFF7B1FD0498FFF7AEFD0290FFF7ABFDBE
:100130000390FFF7A8FD45400498FFF7A4FD019048
:10014000FFF7A1FD0290FFF79EFD0390FFF79BFDD7
:100150006C4073480268089802EB8000847007982E
:10016000FFF791FD044607984440FFF78CFD03908C
:10017000FFF789FD0798FFF786FD0290FFF783FDE3
:100180000390FFF780FD44400798FFF77CFD019046
:10019000FFF779FD0290FFF776FD0390FFF773FDFF
:1001A0000698FFF770FD06980546FFF76CFD039073
:1001B000FFF769FD45400698FFF765FD0290FFF7E0
:1001C00062FD0390FFF75FFD45400698FFF75BFD7A
:1001D0000190FFF758FD0290FFF755FD0390FFF7E0
:1001E00052FD6C400598FFF74EFD05980546FFF758
:1001F0004AFD0390FFF747FD0598FFF744FD029085
:10020000FFF741FD0390FFF73EFD45400598FFF7DE
:100210003AFD0190FFF737FD0290FFF734FD0390A0
:10022000FFF731FD6C400498FFF72DFD054604985B
:10023000FFF729FD0390FFF726FD45400498FFF7DF
:1002400022FD0290FFF71FFD0390FFF71CFD4540C4
:100250000498FFF718FD0190FFF715FD0290FFF7D6
:1002600012FD0390FFF70FFD6C402D4802680898BF
:1002700002EB8000C4700898401C0890089804287D
:10028000FFF6A2AD09B030BD70B5002413E0002523
:100290000DE02349096801EB8501085DFFF7C0FB0C
:1002A0001F49096801EB85010855681CC5B2042D7A
:1002B000EFDB601CC4B2042CE9DB70BD184909688F
:1002C000487B174909684A7A154909684A731449ED
:1002D00009684A79124909684A72114909684A78D5
:1002E0000F4909684A710E49096848700C49096844
:1002F00088780B490968897A094A12689170084917
:1003000009688872064909688879054909688A7BFD
:10031000034909688A71024909688873004901E044
:10032000280000200968C8783C490968C9793B4A17
:100330001268D17039490968CA7A38490968CA719E
:1003400036490968CA7B35490968CA723349096860
:10035000C873704710B500240020FFF711FC01247A
:100360000AE0FFF72DFCFFF745FCFFF796FC20465F
:10037000FFF706FC601CC4B20A2CF2DBFFF720FC7E
:10038000FFF738FC0A20FFF7FBFB10BD10B5002477
:100390000A20FFF7F5FB09240AE0FFF78FFFFFF7BC
:1003A00073FF2046FFF7ECFBFFF709FD601EC4B2A8
:1003B000002CF2DCFFF782FFFFF766FF0020FFF75B
:1003C000DFFB10BD0246002003E00B5C1354431C0E
:1003D000D8B21028F9DB704770B505460E461446B2
:1003E00029462046FFF7EEFF0C4804600C480660E3
:1003F000FFF71AFBFFF7AEFF70BD70B505460E465E
:10040000144629462046FFF7DDFF044804600448EF
:100410000660FFF709FBFFF7B9FF70BD2800002059
:100420002C00002010B54FF4A06000F0F9F810BDCA
:10043000704700BFFEE700BFFEE700BFFEE700BF5A
:10044000FEE7704770477047704700000CB500200A
:10045000019000905E48006840F480305C4908607C
:1004600000BF5B48006800F4003000900198401C19
:100470000190009818B90198B0F5A06FF1D15448D7
:10048000006800F4003010B10120009001E000206D
:1004900000900098012828D14E48006840F01000D4
:1004A0004C4908600846006820F0030008600846D0
:1004B000006808604648406845494860084640680A
:1004C00048600846406848600846406820F00300DD
:1004D00048600846406840F00100486000BF3C4862
:1004E000406800F00C000428F9D10CBD10B5FFF7EE
:1004F000ADFF10BD10B53648006840F0010034492A
:100500000860084640683449084031494860084658
:100510000068324908402E4908600846006820F407
:10052000802008600846406820F4FE0048604FF4D0
:100530001F008860FFF7DAFF4FF00060284908606D
:1005400010BD10B5002100200022214B5B6803F094
:100550000C0121B1042906D0082928D107E0214B3C
:10056000214C236027E0214B1F4C236023E0184BD4
:100570005B6803F47010164B5B6803F4803202234F
:1005800003EB904022B91A4B4343174C23600DE014
:100590000F4B5B6803F4003323B1164B4343124CFB
:1005A000236003E0114B43430F4C236003E00D4BEA
:1005B0000D4C236000BF00BF054B5B68C3F3031302
:1005C0000D4CE15C084B1B68CB40074C236010BD11
:1005D00000100240002002400000FFF8FFFFF6FE7E
:1005E00008ED00E000127A0030000020001BB70088
:1005F00000093D00808D5B003400002006488047E4
:1006000006480047FEE7FEE7FEE7FEE7FEE7FEE7F7
:10061000FEE7FEE7FEE7FEE7F5040108318100088A
:1006200031490143314A1160704770B50021002300
:100630000F22C47804B32D4C246804F4E064C4F59C
:10064000E064210AC1F10403CA40447804FA03F1CA
:100650008478144021430901254C0678A15504787B
:1006600004F01F050124AC4005786D11AD0005F1C3
:10067000E025C5F8004109E0047804F01F050124D5
:10068000AC401C4D0678761145F8264070BD1A4ADC
:100690000A400243154B1B1F1A60704739B1134AB9
:1006A000121D12680243114B1B1D1A6006E00F4A0F
:1006B000121D126882430D4B1B1D1A6070470428DF
:1006C00008D14FF0E021096941F004014FF0E02228
:1006D000116107E04FF0E021096921F004014FF0BA
:1006E000E0221161704700000000FA050CED00E007
:1006F00000E400E080E100E080FFFF1F10B5044649
:10070000FA48844208D10121401500F055FD00212E
:10071000601500F051FD17E0F548844208D1012131
:10072000001500F049FD0021201500F045FD0BE00B
:10073000F048844208D10121C80300F03DFD0021AA
:100740004FF4004000F038FD10BD30B502460020E7
:1007500000235068E84C20400D790C6844EA0524D9
:10076000204350609068E54C2040D1E902542C436E
:100770004D7944EA450420439060D06A20F470002B
:100780000C7C641EE4B2234340EA0350D06230BDC7
:1007900000210160017141718160C160012101741A
:1007A000704721B1826842F00102826003E08268F2
:1007B00022F001028260704721B1826842F48072A7
:1007C000826003E0826822F480728260704710B514
:1007D0000023CBB21AB144681C43446002E0446871
:1007E0009C43446010BD816841F0080181607047FE
:1007F000014600208A6802F008020AB1012000E0E8
:1008000000207047816841F0040181607047014613
:1008100000208A6802F004020AB1012000E00020F2
:10082000704721B1826842F4A002826003E08268CE
:1008300022F4A00282607047014600208A6802F418
:1008400080020AB1012000E00020704710B50A467E
:1008500000210023416821F46041531E41EA4331E5
:10086000416010BD21B1426842F40062426003E081
:10087000426822F4006242607047F0B504460D46BB
:1008800000200021092D11DDE068A5F10A0606EB24
:100890004607072606FA07F18843A5F10A0606EB84
:1008A000460603FA06F10843E0600CE0206905EB18
:1008B0004507072606FA07F1884305EB450603FAC4
:1008C00006F108432061072A0FDA606B561E06EB1B
:1008D00086071F2606FA07F18843561E06EB860692
:1008E00005FA06F10843606322E00D2A0FDA206B57
:1008F000D61F06EB86071F2606FA07F18843D61F88
:1009000006EB860605FA06F10843206310E0E06A6C
:10091000A2F10D0606EB86071F2606FA07F18843AB
:10092000A2F10D0606EB860605FA06F10843E06221
:10093000F0BD21B1826842F48012826003E08268D7
:1009400022F48012826070470146C86C80B2704702
:1009500066484C300068704721B1426842F48062BA
:10096000426003E0426822F480624260704721B135
:10097000426842F48052426003E0426822F48052AE
:10098000426070470A460021816821F4E04111432A
:100990008160704721B1826842F40042826003E0C6
:1009A000826822F400428260704721B1826842F47A
:1009B0000212826003E0826822F4021282607047B1
:1009C000014600208A6802F400120AB1012000E00A
:1009D00000207047F0B5044615460020002200268E
:1009E000092911DDE068A1F10A0707EB470C072789
:1009F00007FA0CF29043A1F10A0707EB470703FA45
:100A000007F21043E0600CE0206901EB410C07277E
:100A100007FA0CF2904301EB410703FA07F2104387
:100A20002061A06BC0F30156EF1C06F1010CA7EB8F
:100A30000C0707EB870C1F2707FA0CF29043EF1CFB
:100A400006F1010CA7EB0C0707EB870701FA07F289
:100A50001043A063F0BD10B50A4600210023816B4E
:100A600021F44011531E41EA0351816310BD08B5C2
:100A7000002300930090009B0B440093009B1A609E
:100A800008BD08B5024600200090009201F1280040
:100A9000009B184400900098006880B208BD0A4688
:100AA00000214168164B1940114341607047416273
:100AB000826270470A460021416821F01F011143FC
:100AC0004160704740B109490831096841F40001AB
:100AD000064A0832116007E004490831096821F428
:100AE0000001024A083211607047000000240140F2
:100AF00000280140003C0140FFFEF0FFFDF7F1FF40
:100B0000FFFD3FFF0246002013680B400BB10120A0
:100B100000E000207047CA430260704770B502468B
:100B20000020002300240B125568CEB205EA06040B
:100B300015681D4015B10CB1012000E0002070BD0A
:100B400000220A12D34303607047000010B5044628
:100B5000CC48844208D10121042000F02DFB002163
:100B6000042000F029FB46E0C748844208D1012157
:100B7000082000F021FB0021082000F01DFB3AE0D6
:100B8000C248844208D10121102000F015FB002149
:100B9000102000F011FB2EE0BD48844208D1012155
:100BA000202000F009FB0021202000F005FB22E0BE
:100BB000B848844208D10121402000F0FDFA00210C
:100BC000402000F0F9FA16E0B348844208D1012130
:100BD000802000F0F1FA0021802000F0EDFA0AE018
:100BE000AE48844207D10121801500F0E5FA0021CA
:100BF000A01500F0E1FA10BD10B50121084600F083
:100C0000DBFA0021012000F0D7FA10BD2DE9F041F8
:100C1000024600250026002000230024002791F82A
:100C200003C00CF00F0591F803C00CF0100CBCF1E0
:100C3000000F03D091F802C04CEA050591F800C0FE
:100C4000BCF1000F31D0146800202BE04FF0010CF4
:100C50000CFA00F3B1F800C00CEA03069E4220D162
:100C600083004FF00F0C0CFA03F7BC4305FA03FCAA
:100C70004CEA040491F803C0BCF1280F06D14FF0F0
:100C8000010C0CFA00FCC2F814C00AE091F803C091
:100C9000BCF1480F05D14FF0010C0CFA00FCC2F872
:100CA00010C0401C0828D1D31460B1F800C0BCF1BA
:100CB000FF0F34DD546800202EE000F1080C4FF0E7
:100CC000010808FA0CF3B1F800C00CEA03069E42D2
:100CD00021D183004FF00F0C0CFA03F7BC4305FA47
:100CE00003FC4CEA040491F803C0BCF1280F05D1C1
:100CF00000F1080C08FA0CF8C2F8148091F803C04F
:100D0000BCF1480F07D100F1080C4FF0010808FAB8
:100D10000CF8C2F81080401C0828CED35460BDE8FF
:100D2000F0814FF6FF710180022181700421C170B2
:100D300070470246002093680B400BB1012000E091
:100D4000002070470146886880B270470246002044
:100D5000D3680B400BB1012000E000207047014632
:100D6000C86880B2704701617047416170470AB13D
:100D7000016100E041617047C16070474FF480320B
:100D80000A43826181618261826982697047024699
:100D90000020434B18684FF68073184040EA021059
:100DA00008433F4B186070473E49C8617047F0B533
:100DB0000A46002300240021002500F00046B6F179
:100DC000004F02D1364EF16901E0354E7168C0F333
:100DD000034583B200F44016B6F5401F08D121F058
:100DE00070612F4E766826F070662D4F7E6012E09F
:100DF00000F48016B6F5801F06D1032606FA05F426
:100E0000A14341F0706106E0460D360103FA06F693
:100E1000B14341F0706122B1460D360103FA06F686
:100E2000314300F00046B6F1004F02D11C4EF16193
:100E300001E01B4E7160F0BD30B500228B071C0F26
:100E40000F2303FA04F2164B08338C1053F82430A6
:100E50009343134C08348D1044F8253023468C10EE
:100E600053F824308C07240F00FA04F423430C4C6D
:100E700008348D1044F8253030BD0A49DC31086053
:100E80007047000000080140000C014000100140C4
:100E90000014014000180140001C014000200140E6
:100EA0000000014000002042DF48006840F00100DF
:100EB000DD49086008464068DC490840DA49486076
:100EC00008460068DA490840D749086008460068C3
:100ED00020F4802008600846406820F4FE00486046
:100EE0004FF41F0088607047CF49096821F48031B2
:100EF000CD4A11601146096821F480211160B0F5D6
:100F0000803F03D0B0F5802F0ED106E0C6490968B6
:100F100041F48031C44A116007E0C349096841F4D3
:100F2000A021C14A116000E000BF00BF704710B5AA
:100F300001460022002300204A11012A02D1BA4CA6
:100F4000236806E0022A02D1B74C236A01E0B64CBE
:100F5000636A01F01F02012494401C400CB101207F
:100F600000E0002010BD38B50020009000240025CE
:100F700000BF3120FFF7DBFF05460098401C0090C2
:100F80000098B0F5A06F01D0002DF2D03120FFF70E
:100F9000CEFF08B1012400E00024204638BD014600
:100FA0000020A14A106820F0F80040EAC10010605B
:100FB0007047A04908607047024600209A4B586865
:100FC00020F47C1042EA01031843974B58607047A5
:100FD00098490866704701460020934A506820F0FF
:100FE00003000843506070478F48406800F00C00D1
:100FF0007047014600208C4A506820F0F0000843FA
:101000005060704701460020874A506820F4E06035
:1010100008435060704701460020834A506820F41E
:10102000605040EAC1005060704729B17E4A527A50
:1010300002437D4B5A7204E07B4A527A82437A4BD8
:101040005A7270477B49D8310860704701460020CA
:10105000754A506820F440400843506070470021B2
:10106000714A20321170704A82F82010012802D093
:1010700004280AD104E001216B4A2032117005E0F6
:101080000521694A2032117000E000BF00BF70479F
:101090006949086070476449096A0143624A1162FC
:1010A0007047654944390860704730B50021002217
:1010B000002400235C4D6D6805F00C0121B104296A
:1010C00005D0082923D105E05C4D056022E05C4D88
:1010D00005601FE0544D6D6805F47012524D6D6847
:1010E00005F48034022505EB92421CB9554D554359
:1010F00005600BE04C4D6D6805F400351DB1524D97
:101100005543056002E04E4D5543056002E04B4DEE
:10111000056000BF00BF444D6D6805F0F00109098E
:101120004A4D6B5C0568DD4045603F4D6D6805F4D8
:10113000E061090A454D6B5C4568DD4085603A4DCC
:101140006D6805F46051C90A404D6B5C4568DD402F
:10115000C560354D6D6805F44041890B3C4D6B5CB5
:10116000C568B5FBF3F5056130BD29B12E4A52695A
:1011700002432D4B5A6104E02B4A526982432A4BA9
:101180005A61704729B1284A92690243264B9A61F5
:1011900004E0254A92698243234B9A61704729B142
:1011A000214AD2690243204BDA6104E01E4AD26927
:1011B00082431D4BDA61704729B11B4AD268024352
:1011C000194BDA6004E0184AD2688243164BDA60A1
:1011D000704729B1144A12690243134B1A6104E0A3
:1011E000114A12698243104B1A6170471249403903
:1011F000086070470F49C86470470B49C871704751
:101200000948406A40F080700749486270470146CB
:101210000020054A92680A400AB1012000E000203F
:101220007047014988727047001002400000FFF8C3
:10123000FFFFF6FE000042428004424200127A00A4
:10124000001BB70000093D00808D5B0044000020BA
:101250005400002010B50446FE48844208D1012104
:10126000C014FFF7A9FF0021E014FFF7A5FFC4E0B9
:10127000B4F1804F08D101210846FFF7AAFF0021F1
:101280000120FFF7A6FFB8E0F348844208D101210E
:101290000220FFF79EFF00210220FFF79AFFACE03B
:1012A000EE48844208D101210420FFF792FF00217B
:1012B0000420FFF78EFFA0E0E948844208D1012115
:1012C0000820FFF786FF00210820FFF782FF94E047
:1012D000E448844208D101211020FFF77AFF002161
:1012E0001020FFF776FF88E0DF48844208D1012113
:1012F0002020FFF76EFF00212020FFF76AFF7CE02F
:10130000DA48844208D101214014FFF755FF00213B
:101310006014FFF751FF70E0D548844209D10121E4
:10132000C804FFF749FF00214FF40020FFF744FFF6
:1013300063E0D048844209D101210805FFF73CFF52
:1013400000214FF48010FFF737FF56E0CA4884426F
:1013500009D101214805FFF72FFF00214FF40010AC
:10136000FFF72AFF49E0C548844208D10121402007
:10137000FFF72FFF00214020FFF72BFF3DE0C04883
:10138000844208D101218020FFF723FF0021802023
:10139000FFF71FFF31E0BB48844208D101218015CF
:1013A000FFF717FF0021A015FFF713FF25E0B64850
:1013B000844209D101210804FFF7FEFE00214FF409
:1013C0008030FFF7F9FE18E0B048844209D10121CE
:1013D0004804FFF7F1FE00214FF40030FFF7ECFE68
:1013E0000BE0AB48844208D101218804FFF7E4FEFA
:1013F00000214FF48020FFF7DFFE10BD002202889D
:10140000944B98420ED0994B98420BD0B0F1804F3C
:1014100008D0914B984205D0904B984202D0904B07
:10142000984204D14FF68F731A404B881A438D4B64
:10143000984207D08C4B984204D04FF6FF431A4095
:10144000CB881A4302808B8883850B880385814B68
:1014500098420BD0854B984208D08B4B984205D0D0
:101460008A4B984202D08A4B984201D10B7A03866C
:1014700001238382704770B5002400220023058C6D
:101480004FF6FE7635400584028C8388048B4FF638
:101490008F752C40B51E2C400D882C43751E2A409C
:1014A0000D892A434D882A436A4DA8420BD06F4DBF
:1014B000A84208D0744DA84205D0744DA84202D06D
:1014C000734DA84213D14FF6F7752A404D892A4330
:1014D0004FF6FB752A408D882A434FF6FF652B4057
:1014E0004FF6FF552B408D892B43CD892B438380AD
:1014F0000483CD888586028470BD70B500240022E7
:101500000023058C4FF6EF7635400584028C8388E6
:10151000048B48F6FF752C404FF6FF452C400D8894
:101520004FF6FF7606EA05252C434FF6DF752A4075
:101530000D8906EA05152A434D8806EA05152A4352
:10154000444DA84202D0494DA8421DD14FF67F75A7
:101550002A404D894FF6FF7606EA05152A434FF6D5
:10156000BF752A408D8806EA05152A434FF6FF35D8
:101570002B404FF2FF752B408D8906EA85052B43E2
:10158000CD8906EA85052B4383800483CD880587B2
:10159000028470BD70B5002400220023058C4FF634
:1015A000FF6635400584028C8388848B4FF68F75E7
:1015B0002C404FF6FC752C400D882C434FF6FF5500
:1015C0002A400D894FF6FF7606EA05252A434D8805
:1015D00006EA05252A431F4DA84202D0234DA84202
:1015E0001DD14FF2FF752A404D894FF6FF7606EA6E
:1015F00005252A434FF6FF352A408D8806EA052542
:101600002A434EF6FF752B404DF6FF752B408D8912
:1016100006EA05152B43CD8906EA05152B43838081
:101620008483CD888587028470BD70B50022002335
:101630000024058C4EF6FF7635400584038C8488A3
:10164000828B48F6FF752A404FF6FF452A400D88E9
:1016500020E00000002C0140000400400008004091
:10166000000C004000100040001400400034014015
:10167000004C01400050014000540140001800405F
:10168000001C004000200040004001400044014098
:10169000004801404FF6FF7606EA05252A434DF63D
:1016A000FF752B400D8906EA05352B434D8806EA68
:1016B00005352B43FA4DA84202D0FA4DA84208D175
:1016C0004BF6FF752C408D894FF6FF7606EA85159F
:1016D0002C4384808283CD88A0F84050038470BD61
:1016E000828B4FF2FF331A408283828B4FF6FF7357
:1016F00003EA01231A4382837047F0B50C4615466E
:10170000002200210026078C4EF6FF7C07EA0C071A
:101710000784828B018C4FF6FF7707EA043640F688
:10172000FF473A404FF6FF7707EA05273A434FF65F
:10173000FF7707EA03373A43D94FB8420ED0D94F63
:10174000B8420BD0B0F1804F08D0D74FB84205D087
:10175000D64FB84202D0D64FB84206D14DF6FF77E9
:10176000394046F48057394305E047F6FF57394082
:1017700044F48057394382830184F0BD828B4FF655
:10178000F3731A408283828B0A4382837047F0B5D9
:101790000C461546002200210026078C4FF6FF6CF0
:1017A00007EA0C070784828B018C4FF6FF7707EA64
:1017B00004264FF60C773A404FF6FF7707EA0317F7
:1017C0002F433A43B64FB8420ED0B64FB8420BD073
:1017D000B0F1804F08D0B44FB84205D0B34FB842F3
:1017E00002D0B34FB84206D14FF6FF57394046F406
:1017F0008077394305E04FF2FF57394044F4807752
:10180000394382830184F0BD028B4FF2FF331A40CB
:101810000283028B4FF6FF7303EA01231A4302830C
:101820007047F0B50C461546002200210026078CB3
:101830004FF6EF7C07EA0C070784028B018C4FF60A
:10184000FF7707EA041640F6FF473A404FF6FF7766
:1018500007EA03373A434FF6FF7707EA05273A438B
:101860008F4FB8420ED08F4FB8420BD0B0F1804F9F
:1018700008D08D4FB84205D08C4FB84202D08C4F63
:10188000B84206D14FF6DF77394046F010073943AA
:1018900005E04FF65F77394044F010073943028383
:1018A0000184F0BD028B4FF6F3731A400283028B62
:1018B0000A4302837047F0B50C461546002200210A
:1018C000068C4FF6FE773E400684028B018C4FF665
:1018D0000C7632407E1C06EA03162E433243704ECD
:1018E000B0420ED06F4EB0420BD0B0F1804F08D056
:1018F0006D4EB04205D06D4EB04202D06C4EB0423B
:1019000006D14FF6FD76314044F00106314305E043
:101910004FF6F576314044F00106314302830184ED
:10192000F0BD70B505460C465D4885420ED05D4859
:1019300085420BD0B5F1804F08D05B48854205D079
:101940005A48854202D05A48854200D100E000BF83
:10195000208850B92389A28861882846FFF7ABFF09
:10196000E1882846FFF79EFF25E0208804280AD159
:101970002389A28861882846FFF753FFE18828461B
:10198000FFF742FF17E0208808280AD12389A288A0
:1019900061882846FFF7FBFEE1882846FFF7EEFE48
:1019A00009E02389A28861882846FFF7A6FEE1881E
:1019B0002846FFF795FE70BD2DE9F04105460C461F
:1019C00000260127608808B9022600E00026A088CA
:1019D000012801D1022700E001272088A0B923892E
:1019E000A28861882846FFF766FFE1882846FFF74E
:1019F00059FF23893A4631462846FFF712FFE1880E
:101A00002846FFF701FF13E02389A2886188284652
:101A1000FFF707FFE1882846FFF7F6FE23893A46DD
:101A200031462846FFF747FFE1882846FFF73AFF8F
:101A3000BDE8F0810A884B881A438B881A43CB880B
:101A40001A430B891A434B891A438B891A43A0F80E
:101A5000442070474FF6FF71818000210180C180D2
:101A60004180017270470021018041808180C180E6
:101A7000018141818181C1817047002101804180C4
:101A8000012181800021C1800181704700210180F6
:101A900041808180C1800181418181817047000046
:101AA000002C0140003401400004004000080040C8
:101AB000000C004021B1028842F00102028004E0E3
:101AC00002884FF6FE731A400280704731B1B0F8B9
:101AD000442042F40042A0F8442005E0B0F844203D
:101AE000C2F30E02A0F8442070471AB183890B4359
:101AF000838102E083898B438381704781827047B1
:101B000041EA0203A0F8483070471AB183890B43B9
:101B1000838102E083898B438381704701894FF67B
:101B2000F8721140018170470A46002101894FF681
:101B30008F73194011430181704730B504460D463B
:101B400029462046FFF7F0FF208940F0070020815A
:101B500030BD2DE9F04104460D4616461F46602D66
:101B600006D13B46012231462046FFF75AFE05E0EA
:101B70003B46012231462046FFF79DFE294620467E
:101B8000FFF7D2FF208940F007002081BDE8F081F7
:101B900030B50C4600210189C9B24FF6FF7505EA40
:101BA0000325154325432943018130BD2DE9F0412B
:101BB00005460E4617469846002443463A463146A7
:101BC0002846FFF7E5FF2C894FF6F870044044F0F3
:101BD00007044FF68F70044044F070042C81BDE878
:101BE000F081F0B504460D4616461F463B46324688
:101BF00029462046FFF7CCFF208940F48040208111
:101C0000F0BD0185828270470A46002101884FF6A7
:101C10008F731940114301807047F0B50C4615468B
:101C20001E460021002200230189028B038C4FF6FF
:101C3000F877394021434FF6FC473A4040F201170C
:101C40003A434FF6DD773B404FF6FF7707EA06173A
:101C50002F433B43018102830384F0BD0A460021E8
:101C6000018B4FF68F7319401143018370470A4669
:101C70000021018B48F6FF7319404FF6FF7303EA0A
:101C800002231943018370470A460021818B4FF6D6
:101C90008F7319401143818370470A460021818B5D
:101CA00048F6FF7319404FF6FF7303EA0223194306
:101CB0008183704721B1028842F08002028004E0F3
:101CC00002884FF67F731A400280704721B18288E4
:101CD00042F00402828004E082884FF6FB731A40CF
:101CE0008280704721B1828842F00802828004E03D
:101CF00082884FF6F7731A408280704721B182883C
:101D000042F00102828004E082884FF6FE731A409E
:101D1000828070470A460021018B4FF6F773194005
:101D20001143018370470A460021018B4FF2FF7374
:101D300019404FF6FF7303EA0223194301837047EA
:101D40000A460021818B4FF6F773194011438183B6
:101D500070470A460021818B4FF2FF7319404FF6FE
:101D6000FF7303EA02231943818370470A46002167
:101D7000018B4FF6FB7319401143018370470A46EC
:101D80000021018B4FF6FF3319404FF6FF7303EA32
:101D900002231943018370470A460021818B4FF6C5
:101DA000FB7319401143818370470A460021818BE0
:101DB0004FF6FF3319404FF6FF7303EA022319432E
:101DC000818370470A460021018B4FF67F731940CB
:101DD0001143018370470A460021018BC1F30E01B4
:101DE0004FF6FF7303EA02231943018370470A4643
:101DF0000021818B4FF67F73194011438183704717
:101E00000A460021818BC1F30E014FF6FF7303EAEE
:101E100002231943818370470A460021018C4FF643
:101E2000FD7319401143018470470A460021018C5B
:101E30004FF6F77319401143018470470A46002199
:101E4000018C4FF6DF7319404FF6FF7303EA02135C
:101E50001943018470470A460021018C4FF67F73B5
:101E600019404FF6FF7303EA0213194301847047C8
:101E70000A460021018C4FF6FF5319404FF6FF73BD
:101E800003EA02231943018470470A460021018CAA
:101E90004FF2FF7319404FF6FF7303EA0223194311
:101EA000018470470A460021018C4DF6FF731940EA
:101EB0004FF6FF7303EA023319430184704730B5CC
:101EC000002301248C40A3B2048C9C430484048C22
:101ED00002FA01F5ADB22C43048430BD30B50023C5
:101EE00004248C40A3B2048C9C430484048C02FA26
:101EF00001F5ADB22C43048430BD70B5034600201B
:101F000000241846183001258D40ACB21D8CA54325
:101F10001D8409B1082909D100EB6100056825F08D
:101F2000700505600568154305600EE00D1FC5F3DB
:101F30004E052844056825F4E045056005684FF620
:101F4000FF7606EA02263543056070BD21B102889E
:101F500042F00202028004E002884FF6FD731A404C
:101F60000280704721B1028842F00402028004E03E
:101F700002884FF6FB731A400280704721B18288B5
:101F800042F08002828004E082884FF67F731A401C
:101F90008280704702884FF6F7731A4002800288E9
:101FA0000A430280704782884FF68F731A408280FE
:101FB00082880A438280704702894FF6F8731A407C
:101FC000028102890A430281704702894FF67F73BA
:101FD0001A40028102890A43028170478184704756
:101FE0008185704781867047018770478187704778
:101FF000A0F84010704702884FF6FF431A40028055
:1020000002880A43028070470146888E7047014665
:10201000088F70470146888F70470146B1F840002D
:1020200070470146888C70470146088D704702460C
:102030000020138A0B400BB1012000E00020704704
:10204000CA430282704730B50246002000230024B4
:10205000158A05EA0103958905EA010413B10CB15B
:10206000012000E0002030BDCA430282704700001A
:1020700010B50446BE48844208D101218014FFF700
:102080009BF80021A014FFF797F816E0B9488442A6
:1020900008D101210014FFF79CF800212014FFF75C
:1020A00098F80AE0B448844207D10121C013FFF731
:1020B00090F80021E013FFF78CF810BD10B5002256
:1020C000028802F441520B884C8823438C882343B6
:1020D000CC8823430C8923434C8923438C89234395
:1020E000CC8923431A430280838B4FF2FF74234031
:1020F00083830B8A038210BD2DE9F04F85B005461E
:102100000C464FF0000902274FF000084FF0010B7A
:102110000026B246A88B4FF240010840A883022057
:102120002884B5F81C90A068022801D100BF38E0CF
:10213000A08810B94FF0010B01E04FF0020B8D4861
:10214000854200D100E000BF6846FEF7AEFFDDF833
:1021500000A0E088B0F5007F0AD14FEA1A2000EB1A
:1021600080004000A168B0FBF1F0401D86B20BE09A
:102170004FEA4B10BAFBF0F000EB80004000A16882
:10218000B0FBF1F0401D86B20A20B6FBF0F606F077
:102190000108A6EB0800C0F34F074FF6FF7000EAF6
:1021A0000828022F01DBFF2F02DD02274FF0000875
:1021B000E08840EA080038432884A088A1890843C1
:1021C000618808432188084340F4006040EA090917
:1021D000A5F81C9005B0BDE8F08F0021018041807A
:1021E0008180C180018141818181C181072101827A
:1021F00070470021018041808180C180022181607F
:1022000000218181704721B1028842F040020280A2
:1022100004E002884FF6BF731A400280704721B174
:10222000828B42F48062828304E0828B4FF6FF331C
:102230001A408283704730B5002400230C11012519
:10224000A540ABB21AB185881D43858002E0858820
:102250009D43858030BD1AB183880B43838002E0A3
:1022600083888B43838070478181704701468889CA
:1022700070474FF6FF62914204D0028842F48072A8
:10228000028004E002884FF6FF631A400280704724
:1022900021B1828842F00402828004E082884FF6F5
:1022A000FB731A408280704702884FF2FF731A4016
:1022B000028002880A4302807047018841F48051FD
:1022C0000180704721B1028842F40052028004E08C
:1022D00002884DF6FF731A400280704702460020C4
:1022E000012901D0108B00E0908A70470146088ACE
:1022F0007047B1F5804F04D1028842F480420280D9
:1023000004E002884BF6FF731A40028070470246D1
:10231000002013890B400BB1012000E00020704722
:10232000CA4302817047F0B5024600200024002312
:10233000002501F00F070126BE40B4B20B110126A3
:102340009E40B3B2968806EA03051689264016B168
:102350000DB1012000E00020F0BD10B5002201F019
:102360000F040123A3409AB2D343038110BD0000A0
:102370000030014000380040003C004010B50446E9
:10238000FB48844209D101218803FEF715FF002193
:102390004FF48040FEF710FF32E0F648844209D146
:1023A00001214804FEF715FF00214FF40030FEF72D
:1023B00010FF25E0F048844209D101218804FEF78E
:1023C00008FF00214FF48020FEF703FF18E0EB48E0
:1023D000844209D10121C804FEF7FBFE00214FF41D
:1023E0000020FEF7F6FE0BE0E548844208D101210B
:1023F0000805FEF7EEFE00214FF48010FEF7E9FE1F
:1024000010BD2DE9F04786B005460E460024A246D1
:1024100000BFA1460027B08900B100BF2F462C8A1B
:102420004CF6FF700440F08804432C82AC894EF6D1
:10243000F3100440B088318908437189084304438C
:10244000AC81AC8A4FF6FF400440B0890443AC82B3
:1024500001A8FEF72AFEC648874202D1DDF810A087
:1024600001E0DDF80CA0A88900F4004040B10AEBBF
:10247000CA0000EB0A1031684900B0FBF1F807E030
:102480000AEBCA0000EB0A1031688900B0FBF1F8D2
:102490006420B8FBF0F004012009642101FB1089DD
:1024A000A88900F4004040B1322000EBC900B0FB25
:1024B000F1F000F00700044308E0322000EB0910BF
:1024C0006421B0FBF1F000F00F0004432C8106B052
:1024D000BDE8F0874FF41651016000218180C18072
:1024E00001810C21418100218181704710B5024694
:1024F0000020108A4FF2FF0318400B884C882343BA
:102500008C882343CC8823431843108210BD0021BC
:10251000018041808180C180704721B1828942F46D
:102520000052828104E082894DF6FF731A40828155
:102530007047F0B50346002400260025002040F631
:102540006A17B94200D100BF1846C1F3421401F026
:102550001F06012707FA06F5012C01D10C3004E013
:10256000022C01D1103000E014301AB107682F435B
:10257000076002E00768AF430760F0BD1AB1838AC5
:102580000B43838202E0838A8B4383827047028AF3
:102590004FF6F0731A400282028A0A4302827047A1
:1025A00082894FF2FF731A40828182890A438281B5
:1025B000704721B1828942F00202828104E082895F
:1025C0004FF6FD731A4082817047028A4FF6DF731F
:1025D0001A400282028A0A430282704721B1028AAB
:1025E00042F48042028204E0028A4BF6FF731A40F2
:1025F00002827047C1F308028280704701468888D2
:10260000C0F308007047818941F001018181704762
:10261000028BD2B20283028B42EA0122028370470C
:10262000028B02F47F420283028B0A4302837047CB
:1026300021B1828A42F02002828204E0828A4FF62F
:10264000DF731A408282704721B1828A42F0100201
:10265000828204E0828A4FF6EF731A4082827047CA
:1026600021B1828A42F00802828204E0828A4FF617
:10267000F7731A408282704721B1828942F4004286
:10268000828103E08289C2F30E028281704721B108
:10269000828A42F40062828204E0828A4FF2FF73EF
:1026A0001A4082827047828A4FF6FB731A408282F8
:1026B000828A0A438282704721B1828A42F00202F2
:1026C000828204E0828A4FF6FD731A40828270474C
:1026D00002460020B1F5007F00D100BF13880B40F7
:1026E0000BB1012000E00020704701F40072B2F548
:1026F000007F00D100BFCA430280704770B5024618
:10270000002400230025002040F66A16B14200D1C3
:1027100000BFC1F3421501F01F03012606FA03F3BF
:10272000012D02D19689334006E0022D02D1168A8E
:10273000334001E0968A33400C12012606FA04F475
:102740001688344013B10CB1012000E0002070BDA8
:1027500010B50022002340F66A14A14200D100BF48
:102760000A1201249440A3B2DC43048010BD00008F
:10277000003801400044004000480040004C004048
:102780000050004001684FF6FE72114001600021C8
:10279000016041608160C1608D49884208D18C49E7
:1027A0000839496841F00F01894A083A51608AE0C6
:1027B00087491431884208D185490839496841F070
:1027C000F001834A083A51607DE08149283188420E
:1027D00008D17F490839496841F470617C4A083A58
:1027E000516070E07A493C31884208D17849083913
:1027F000496841F47041764A083A516063E074498F
:102800005031884208D172490839496841F4702131
:102810006F4A083A516056E06D496431884208D1E8
:102820006B490839496841F47001694A083A5160B6
:1028300049E067497831884208D1654908394968D3
:1028400041F07061624A083A51603CE06149884257
:1028500006D1011F096841F00F01021F116032E02B
:102860005C491431884208D15A49091F096841F06E
:10287000F001584A121F116025E05649283188425C
:1028800008D15449091F096841F47061514A121F67
:10289000116018E04F493C31884208D14D49091F69
:1028A000096841F470414B4A121F11600BE049491D
:1028B0005031884207D14749091F096841F4702106
:1028C000444A121F1160704710B50022026847F693
:1028D000F0739A430C6A8B6823430C6923434C6959
:1028E00023438C692343CC6923434C6A23438C6A7A
:1028F00023431A430260CB6843600B6883604B68D4
:10290000C36010BD0021016041608160C160016150
:1029100041618161C161016241628162704721B19F
:10292000026842F00102026004E002684FF6FE73A2
:102930001A40026070471AB103680B43036002E05B
:1029400003688B43036070474160704701464868E5
:1029500080B2704701460020002201F080531BB175
:102960001C4B083B1A6802E0194B083B1A6802EA44
:1029700001030BB1012000E00020704700F08051FE
:1029800019B11449091F086002E01149083948606B
:10299000704701460020002201F080531BB10D4B0F
:1029A000083B1A6802E00A4B083B1A6802EA010376
:1029B0000BB1012000E00020704700F0805119B1F8
:1029C0000449091F086002E001490839486070475E
:1029D000080002400804024010B501210807FEF774
:1029E000F8FB00214FF08050FEF7F3FB10BD2A49A1
:1029F0000862704728490861704701460020274A4D
:102A0000106820F0E0000843106070472249A031B0
:102A10000860704710B502460020204B186820F06F
:102A20000300104318601E4B1B6843F004031C4C4A
:102A30002360012901D130BF00E020BF184B1B6883
:102A400023F00403164C236010BD1448006840F0C6
:102A50000400124908600846006840F0020008605F
:102A60000F48006840F004000D49086000BF00BF37
:102A700030BF704701460020084A52680A400AB138
:102A8000012000E0002070470449096841EA800104
:102A9000024A11607047000000000E4200700040C2
:102AA00010ED00E001460020FE4A106800F03800FA
:102AB000084310607047FB49096821F00801F94A92
:102AC000116011460968014311607047F5490968B2
:102AD00021F01001F34A11601146096801431160A9
:102AE0007047F148EF494860F04848607047EE4849
:102AF000EC494860ED4848607047EA48006940F09A
:102B00008000E84908617047E648006940F08000AD
:102B1000E449086170470420E249C96801F00101F5
:102B200009B101200EE0DF49C96801F0040109B1D3
:102B3000022007E0DB49C96801F0100109B1032058
:102B400000E00420704700B502460423FFF7E3FFCE
:102B5000034603E0FFF7DFFF0346521E012B01D1BE
:102B6000002AF7D102B90523184600BD30B5044646
:102B700004254FF43020FFF7E6FF0546042D17D15A
:102B8000C848006940F00200C6490861084644612F
:102B9000006940F0400008614FF43020FFF7D3FF98
:102BA0000546C048006941F6FD710840BD4908610D
:102BB000284630BD10B504244FF43020FFF7C3FF82
:102BC0000446042C16D1B748006940F00400B5490A
:102BD00008610846006940F0400008614FF4302069
:102BE000FFF7B1FF0446AF48006941F6FB710840AA
:102BF000AC490861204610BD00B502460423FFF72A
:102C00008AFF034603E0FFF786FF0346521E012BAF
:102C100001D1002AF7D102B90523184600BD10B52D
:102C200004244FF43020FFF7E7FF0446042C16D1AC
:102C30009C48006940F004009A4908610846006910
:102C400040F0400008614FF43020FFF7D5FF044604
:102C50009448006941F6FB7108409249086120469A
:102C600010BD00208F49C96901F0020109B101209E
:102C700000E00020704730B5A5250424FFF7F1FFE0
:102C800000B100254FF43020FFF75DFF0446042C0F
:102C90003AD185488349886084488860084600693D
:102CA00040F0200008610846006940F040000861DB
:102CB0004FF43020FFF747FF0446042C1BD179481E
:102CC000006941F6DF7108407649086108460069ED
:102CD00040F01000086176480580E002FFF733FFFE
:102CE0000446052C10D06F48006941F6EF7108408A
:102CF0006C49086108E0052C06D06A48006941F675
:102D0000EF71084067490861204630BD78B5064636
:102D10000C46042500200090E802FFF714FF05464A
:102D2000042D24D15F48006940F001005D4908612D
:102D30003480E802FFF707FF0546042D10D1B01CD0
:102D40000090200C00990880E802FFF7FCFE054681
:102D50005448006941F6FE7108405249086106E096
:102D60005048006941F6FE7108404E490861284606
:102D700078BD70B504460D460426F002FFF7E3FE69
:102D80000646042E11D14748006940F0010045492C
:102D900008612580F002FFF7D6FE0646414800692B
:102DA00041F6FE7108403F490861304670BD70B57C
:102DB00005460E460424E002FFF7C5FE0446042C37
:102DC00017D1394837498860384888600846006913
:102DD00040F0100008612E80E002FFF7B4FE0446C8
:102DE000052C06D02F48006941F6EF7108402D49A7
:102DF0000861204670BD2DE9F04304464FF6FF768A
:102E00003746B046B1460425E443E6B2C4F307278B
:102E1000C4F307484FEA1469E802FFF794FE054639
:102E2000042D49D120481F49886020488860084601
:102E3000006940F010000861FF2E06D01C480830E1
:102E40000680E802FFF77FFE0546042D08D1FF2F1C
:102E500006D017480A300780E802FFF774FE0546DF
:102E6000042D0AD1B8F1FF0F07D011480C30A0F89B
:102E70000080E802FFF767FE0546042D0AD1B9F18C
:102E8000FF0F07D00A480E30A0F80090E802FFF7C5
:102E90005AFE0546052D0FD00248006941F6EF7134
:102EA000084007E00020024023016745AB89EFCDD1
:102EB00000F8FF1F664908612846BDE8F08330B579
:102EC000054604244FF43020FFF73DFE0446042C51
:102ED00041D160485E4988605F4888600846006963
:102EE00040F0200008610846006940F04000086199
:102EF0004FF43020FFF727FE0446042C22D154481B
:102F0000006941F6DF7108405149086108460069CF
:102F100040F0100008611DB100205049088002E017
:102F2000A5204E4908804FF43020FFF70CFE0446E0
:102F3000052C10D04648006941F6EF71084044491D
:102F4000086108E0052C06D04148006941F6DF71B0
:102F500008403F490861204630BDF0B505460E46A1
:102F6000174604243B483A4988603B488860E002A1
:102F7000FFF7E9FD0446042C19D13548006940F0FB
:102F800010003349086147F0F800304328433349C3
:102F9000891C0880E002FFF7D6FD0446052C06D008
:102FA0002B48006941F6EF71084029490861204625
:102FB000F0BD2748C069800870472548006A7047FF
:102FC00000202349096801F0200109B1012000E037
:102FD0000020704729B11E4A126902431C4B1A6136
:102FE00004E01B4A12698243194B1A61704701467B
:102FF0000020012908D1164AD26902F001020AB163
:10300000012008E0002006E0114AD2680A400AB117
:10301000012000E0002070470D49C860704704207F
:103020000B49C96801F0010109B101200EE008490E
:10303000C96801F0040109B1022007E00449C96828
:1030400001F0100109B1032000E0042070470000E6
:103050000020024023016745AB89EFCD00F8FF1F38
:10306000002044490860091D0860091D0860091D09
:10307000086041483F4914310860704700213D49CC
:103080008279002A3AD00A46126803689A430B46AE
:103090001A600A1D126803689A430B1D1A600279B0
:1030A00011440A6803681A430A60324A08321268F7
:1030B00003689A432F4B08331A601A1D126803687D
:1030C0009A432C4B0C331A604279102A0ED11A1FE6
:1030D000126803681A43274B08331A601A1D1268D6
:1030E00003681A43234B0C331A600DE021494279DF
:1030F00011440A6803681A430A6005E00279114422
:103100000A6803689A430A607047002101600171F0
:103110000C214171002181717047164910310968F5
:103120000143144A10321160704701460020114AD1
:10313000143212680A400AB1012000E000207047F2
:103140000C49143108607047014600200022094BE9
:103150001B6803EA0102074B14331B680B4013B1D1
:103160000AB1012000E000207047024914310860D4
:103170007047000000040140FFFF0F000E49086087
:1031800070470D49486070470B49886070474AF6A0
:10319000AA200949086070474CF6CC4006490860EF
:1031A000704701460020044AD2680A400AB1012053
:1031B00000E000207047000000300040F0B50346FA
:1031C00000201C460D4608E026782F78F61B301E9E
:1031D00000D004E0641C6D1C521E002AF4D800BF0D
:1031E000F0BD70B504460D46002305E026782E702C
:1031F0006D1C641C5E1CB3B29342F7DB70BDF0B56E
:1032000005460E46144663B929463246002005E0BD
:103210000F781770521C491C471CB8B2A042F7DB4C
:103220000EE0012B0CD12F19791E3246002005E04B
:103230000F781770521C491E471CB8B2A042F7DB2A
:10324000F0BD10B50346002204E000241C705B1C96
:10325000541CE2B28A42F8DB10BD10B502460023CE
:103260001078992812DC507880B1507812280DDC43
:10327000907858B19078312808DCD078232805DC84
:103280001079592802DC5079592801DD002010BD41
:103290000878992812DC487880B1487812280DDC2B
:1032A000887858B18878312808DCC878232805DC6C
:1032B0000879592802DC4879592801DD0020E6E721
:1032C00010780C78A04201DD002342E010780C78E1
:1032D000A0423DD150784C78A04201DD002338E077
:1032E00050784C78A04231D190788C78A04201DDA2
:1032F00000232EE090788C78A04225D1D078CC782D
:10330000A04201DD002324E0D078CC78A04219D17E
:1033100010790C79A04201DD00231AE010790C79B4
:10332000A0420DD150794C79A04201DD002310E07C
:1033300050794C79A04201D101230AE0022308E030
:10334000022306E0022304E0022302E0022300E05D
:10335000022318469BE701460878992812DC487832
:1033600080B1487812280DDC887858B188783128E7
:1033700008DCC878232805DC0879592802DC48795C
:10338000592801DD002070470120FCE7704730B567
:1033900001460846CC1701EB14742411A1EB041468
:1033A0000A46CD1701EB15752D1105EB850504EBCC
:1033B0004504E3B2184630BD01460A2291FBF2F300
:1033C00002FB131391FBF2F203EB0212D0B270472F
:1033D0002DE9FC4704460D4616464FF00009002231
:1033E00013462046294634F0E5FB03D24FF001098D
:1033F00085F000452046294634F073FB0190019882
:1034000034F002FB074622462B4634F0FAF9044614
:103410000D460022FE4B2046294634F0F5F90446BD
:103420000D462046294634F05CFB80B20090B9F18D
:10343000010F03D1019840F0004001900222314673
:103440006846FFF7CEFE0422B11C01A8FFF7C9FEB3
:10345000BDE8FC872DE9F04104460D46164622469C
:103460002B463046F6F7AAFA3046F6F757FA0746E3
:1034700088463A4643462046294634F09BFB02D113
:103480000020BDE8F0810120FBE770B504460D4641
:1034900021462846F6F738FA2846F6F780F9064618
:1034A0003146204634F0D2FB01D1002070BD01200E
:1034B000FCE770B504460D4621462846F6F7A2FA09
:1034C0002846F6F787FA0646A64201D1002070BDCD
:1034D0000120FCE710B5F5F797FAF4F7ADFFF5F723
:1034E00012FCF5F7A2FC07F0A5FD10BD2DE9F04197
:1034F00000210D20F5F742F9054634F06FFA044635
:10350000204634F044FB0546C24AC34B34F07CF9F4
:10351000074634F07FFB0446204634F0AFFAC1B2D0
:10352000BE4881750146887D34F058FA0746214629
:1035300034F050F80646BA4934F04FF8054634F0F6
:103540009DFAB64948750846807DA1F817000846DF
:10355000B0F8170000EBC00101EB00104FF6FF714F
:1035600001EA8000AD49A1F817000846B0F817003D
:10357000497D0844A949A1F81700BDE8F08170B55C
:10358000FBF79AFD0120F4F796FFFBF72FFE0446A8
:10359000FBF7A0FDFBF754FD0120F4F78CFF0120A1
:1035A000A04908604FF4FA70F4F785FF4FF400610A
:1035B0009D48FDF7CBFB08B9012000E0002005463F
:1035C0002A464FF400619848FDF7D1FB4FF4FA709A
:1035D000F4F771FF4FF400619348FDF7B7FB08B9AA
:1035E000012000E0002005462A464FF400618E4885
:1035F000FDF7BDFBFFF77AFF00208A4908604CB950
:10360000012086490874082048740620887001202B
:10361000087008E006208149C87000200874022064
:1036200008700120487400207C49887007F0A0FBD6
:1036300007F0BEFB7D480068012812D17C48407825
:10364000C0F3C00038B17B48407801280DD001207C
:103650007849487009E00020764948704870087041
:1036600003E0002073494870087070481C380068F7
:10367000012814D16E484078C0F3001038B16D486D
:10368000C07801280FD001206A49C8700BE00020E3
:103690006849C8706849487481F86F0003E00020E9
:1036A0006449C870887007F073FB07F090FB70BD29
:1036B00010B529F031FC07216048FCF777F90120AB
:1036C000F4F7F9FE00205E490860FFF758FF10BDCF
:1036D00000205C4908704870C87088700871C87311
:1036E00008744882888270470020574981F8680032
:1036F00081F8690081F86B0081F86A0081F86C003C
:1037000081F86D0081F86F0081F8700008667047DD
:1037100070472DE9FF5F4D4908684D4933F05DFF63
:103720004C49C1F81A0049494868494933F055FFE6
:103730004849C1F81E0045498868454933F04DFFA6
:103740004449C1F822004FF47A703449A1F81F00AF
:1037500001200870002040498870404A1060506085
:1037600000219160D160114681F809013C4908703F
:1037700001204871002088713A49487003201146A1
:1037800081F8A00001203849087048703748C08887
:1037900048803648C1883448A0F80D103348C178B5
:1037A000314801713148C1782F48C1731046026A0F
:1037B000416A104634F02EFA2B49C1F8050027491A
:1037C0008A6AC96A104634F025FA2749C1F8090007
:1037D0002248026A416A104634F01CFA2249086104
:1037E0001E48826AC16A104634F014FA1E494861C4
:1037F0001E48C07808761D48C1781B4880F8221002
:103800001A480179184841761848017916482FE07E
:103810000088C340B6BE4868CBB9643FA2160020FA
:103820000000C842800122420008014030012342CA
:10383000EA2D002067000020901900205348050859
:1038400084812242F60F00201F190020912D0020B4
:1038500000007A44D91800205F1A00208E22002030
:10386000581D002070000020E31700200C000020ED
:1038700080F82310F8490A6A496A104634F0CAF9F8
:10388000F649C1F81A00F448826AC16A104634F059
:10389000C1F9F249C1F81E00EF48026A416A1046B8
:1038A00034F0B8F9ED494862EB48826AC16A1046C3
:1038B00034F0B0F9E94988620A20E94988740020A7
:1038C000E8490872C871E849088834F087F8E74980
:1038D000C1F81600E449488834F080F8E349C1F89B
:1038E0001A00E149888834F079F8E049C1F80E00FF
:1038F000DD49C88834F072F8DC49C1F82200DA49A1
:10390000088934F06BF8D949C1F81200D6494889C2
:1039100034F064F8D549C1F81E0016F00DF816F021
:10392000DBF816F007F916F0DCF9D1490869D1493E
:1039300033F085FED049C1F842000020CF49C8715C
:1039400016F077FD0120C64981F85500FFF7E0FE2B
:10395000DFF82CB34FF0000A08E000208BF80000DD
:103960000BF1010B0AF1010000F0FF0ABAF1030F9D
:10397000F3D3BE49D1F8060034F009F904460D46E8
:10398000BA49D1F8060034F002F90646BD4ABE4BEA
:1039900033F03AFF22462B46CDE9000133F034FFE5
:1039A00080460022B94B33F0A1FFCDE9020134F08B
:1039B00031F9AE49C1F80A000020A9494872C8711E
:1039C0000872012008750020A64908714FF40061B3
:1039D000AF48FDF7BBF908B9012000E0002004461C
:1039E00022464FF40061AA48FDF7C1F94FF07E501E
:1039F000A149C8630220A74908700020984981F8AE
:103A00003600A5490870FFF76FFEFFF761FE0DF065
:103A1000B2FF16F02FFE2FF0C0FEBDE8FF9F10B5DD
:103A20000BF00DFF10BD10B5FFF754FD4FF4006112
:103A30009748FDF78BF908B9012000E00020044603
:103A400022464FF400619248FDF791F94FF4FA7065
:103A5000F4F731FD4FF400618D48FDF777F908B9AF
:103A6000012000E00020044622464FF4006188480F
:103A7000FDF77DF94FF4FA70F4F71DFDF6F76EFBD4
:103A80004FF400618248FDF761F908B9012000E0B8
:103A90000020044622464FF400617D48FDF767F997
:103AA00015F0ECFA4FF400617948FDF74FF908B9C9
:103AB000012000E00020044622464FF400617448D3
:103AC000FDF755F915F021FD16F0F0FA29F0BFFACF
:103AD0004FF400616E48FDF739F908B9012000E0A4
:103AE0000020044622464FF400616948FDF73FF983
:103AF00029F0BFFE4FF400616548FDF727F908B9CA
:103B0000012000E00020044622464FF40061604896
:103B1000FDF72DF94FF400615D48FDF717F908B97D
:103B2000012000E00020044622464FF4006158487E
:103B3000FDF71DF9FFF773FF4FF400615448FDF7DF
:103B400005F908B9012000E00020044622464FF4A0
:103B500000614F48FDF70BF9FFF7DBFD4FF4006103
:103B60004B48FDF7F3F808B9012000E000200446B7
:103B700022464FF400614648FDF7F9F8FFF798FD3B
:103B80004FF400614248FDF7E1F808B9012000E078
:103B90000020044622464FF400613D48FDF7E7F857
:103BA00000203E49087010BD70472E4880792D498D
:103BB0004871084640793C2803DD0120C871002087
:103BC0008871704727488079FA2804DC2548807975
:103BD000401C2449887170472DE9F0470646894604
:103BE000154600270024A046C8212D4833F05DFC6F
:103BF000C82D02D90120BDE8F087002724E04FF04E
:103C00000008C821264833F050FC2A464946304671
:103C100012F061FD2A464946214812F067FD002452
:103C200009E0305D1E49095D884202D04FF001086D
:103C300003E0601C84B2AC42F3DB00BFB8F1010FBB
:103C400000D003E0781C87B2032FD8DB00BFB8F1A7
:103C5000010F27D10120CEE78E220020E31700209C
:103C6000A21600209D180020BA2D002098230020C5
:103C7000DB2B002000006145D91800207C1D0020AE
:103C8000FE0000206F1283C0CA21094000001040CE
:103C900000080140FB000020660000200601002013
:103CA000FE1A00200020A6E700B59BB0002101917C
:103CB0000291039104910591069107910891099150
:103CC0000A9100200B900C900D910E910F90109086
:103CD0001190129013911491FE48CDE9151042F203
:103CE0001070179000201890FB481990FB481A900C
:103CF0000120FB4908700020C1F80100012240F6B4
:103D00003E51F748FFF768FF012240F63F51F44863
:103D1000FFF762FF01224FF45461F148FFF75CFFA7
:103D200068224FF47F7101A812F0D5FC682240F29E
:103D3000924101A812F0CFFC68224FF4A56101A8BE
:103D400012F0C9FC042240F2BE51E548401C12F0BA
:103D5000C2FC682240F2D65101A812F0BCFC6822D5
:103D600040F26C6101A812F0B6FC682240F20271C8
:103D700001A812F0B0FC04224FF4F361D848401CB3
:103D800012F0A9FC68224FF4F66101A812F0A3FC1E
:103D9000682240F6460101A812F09DFC682240F618
:103DA000DC0101A812F097FC042240F67211CC4805
:103DB000401C12F090FC682240F68A1101A812F013
:103DC0008AFC68224FF4226101A812F084FC682268
:103DD00040F6B62101A812F07EFC042240F64C31D8
:103DE000BF48401C12F077FC682240F6643101A8FD
:103DF00012F071FC682240F6FA3101A812F06BFC57
:103E000068224FF4496101A812F065FC042240F6D3
:103E10002651B348401C12F05EFCB24ADDE90110A5
:103E20009162D062DDE9031011625062DDE90501A3
:103E30009063D163DDE9071011635063DDE9090187
:103E40009064D164DDE90B0110645164DDE90D017A
:103E50009065D165DDE90F1011655065DDE911014F
:103E60009066D166DDE91301106651668032DDE9A6
:103E70001510116050609B491798C1F88800189878
:103E8000C1F8940098481999416697491A98C1F861
:103E90002E001BB000BD2DE9F05F81460F46904615
:103EA0001C464FF0000A4846F5F779FC05463846AF
:103EB000F5F775FC06464046F5F771FC834631463A
:103EC000284633F0C3FE06D15946304633F0BEFED5
:103ED00001D1256015E03146284633F0B7FE04D005
:103EE0005946284633F0B2FE01D1256009E0594613
:103EF000304633F0ABFE01D1266002E025604FF082
:103F0000010A5046BDE8F09F2DE9F05F82468846E1
:103F100091461D464FF0000B5046F5F75BFD0446F9
:103F20004046F5F757FD06464846F5F753FD074668
:103F3000B44203D1BE4201D12C600CE0B44201D0A6
:103F4000BC4201D12C6006E0BE4201D12E6002E0ED
:103F50002C604FF0010B5846BDE8F09F2DE9FF4F54
:103F600081B08B469A46002000900198F5F7D6FC68
:103F700004460D465846F5F7D1FC06460F46039811
:103F8000F5F7CCFC8046894632463B46204629461A
:103F900033F010FE09D142464B463046394633F0E5
:103FA00009FE02D1CAE900451EE032463B462046E2
:103FB000294633F0FFFD06D042464B4620462946AF
:103FC00033F0F8FD02D1CAE900450DE042464B4608
:103FD0003046394633F0EEFD02D1CAE9006703E00E
:103FE000CAE9004501200090009805B0BDE8F08FB7
:103FF00000B59FB01CAB4FF4A56240F292414FF464
:104000007F70FFF7ABFF012818D11CAB4FF4A562FE
:1040100040F292414FF47F70FFF7A0FF012808D1D2
:10402000324890F8500040F00100304981F85000CB
:1040300008E0DDE91C01CDE9000103E0DDE91C0138
:10404000CDE900011CAB4FF4A66240F29A4140F268
:104050000440FFF783FF012818D11CAB4FF4A66280
:1040600040F29A4140F20440FFF778FF012808D15E
:104070001E4890F8500040F002001C4981F85000A2
:1040800008E0DDE91C01CDE9020103E0DDE91C01E6
:10409000CDE902011CAB4FF4A76240F2A24140F20D
:1040A0000C40FFF75BFF012827D11CAB4FF4A76240
:1040B00040F2A24140F20C40FFF750FF012817D117
:1040C0000A4890F8500040F00400084981F8500078
:1040D00017E00000000059400000A0419A99CA4230
:1040E000D50000208E220020F6150020A216002008
:1040F000DDE91C01CDE9040103E0DDE91C01CDE9A6
:1041000004011CAB4FF4A86240F2AA4140F21440F3
:10411000FFF724FF012818D11CAB4FF4A86240F22E
:10412000AA4140F21440FFF719FF012808D1FC48CA
:1041300090F8500040F00800F94981F8500008E07C
:10414000DDE91C01CDE9060103E0DDE91C01CDE953
:1041500006011CAB4FF4A96240F2B24140F21C4090
:10416000FFF7FCFE012818D11CAB4FF4A96240F206
:10417000B24140F21C40FFF7F1FE012808D1E848A7
:1041800090F8500040F01000E54981F8500008E038
:10419000DDE91C01CDE9080103E0DDE91C01CDE901
:1041A00008011CAB4FF4AA6240F2BA4140F224402D
:1041B000FFF7D4FE012818D11CAB4FF4AA6240F2DD
:1041C000BA4140F22440FFF7C9FE012808D1D44883
:1041D00090F8500040F01000D14981F8500008E0FC
:1041E000DDE91C01CDE90A0103E0DDE91C01CDE9AF
:1041F0000A011CAB4FF4AB6240F2C24140F22C40CA
:10420000FFF7ACFE012818D11CAB4FF4AB6240F2B3
:10421000C24140F22C40FFF7A1FE012808D1C0485E
:1042200090F8500040F01000BD4981F8500008E0BF
:10423000DDE91C01CDE90C0103E0DDE91C01CDE95C
:104240000C011CAB4FF4AC6240F2CA4140F2344066
:10425000FFF784FE012818D11CAB4FF4AC6240F28A
:10426000CA4140F23440FFF779FE012808D1AC483A
:1042700090F8500040F01000A94981F8500008E083
:10428000DDE91C01CDE90E0103E0DDE91C01CDE90A
:104290000E011CAB4FF4AD6240F2D24140F23C4003
:1042A000FFF75CFE012818D11CAB4FF4AD6240F261
:1042B000D24140F23C40FFF751FE012808D1984816
:1042C00090F8500040F01000954981F8500008E047
:1042D000DDE91C01CDE9100103E0DDE91C01CDE9B8
:1042E00010011CAB4FF4AE6240F2DA4140F24440A0
:1042F000FFF734FE012818D11CAB4FF4AE6240F238
:10430000DA4140F24440FFF729FE012808D18448F1
:1043100090F8500040F01000814981F8500008E00A
:10432000DDE91C01CDE9120103E0DDE91C01CDE965
:1043300012011CAB4FF4AF6240F2E24140F24C403C
:10434000FFF70CFE012818D11CAB4FF4AF6240F20E
:10435000E24140F24C40FFF701FE012808D17048CD
:1043600090F8500040F020006D4981F8500008E0BE
:10437000DDE91C01CDE9140103E0DDE91C01CDE913
:1043800014011AAB4FF4B06240F2EA4140F25440DB
:10439000FFF7BAFD012816D11AAB4FF4B06240F214
:1043A000EA4140F25440FFF7AFFD012808D15C48D4
:1043B00090F8500040F02000594981F8500004E086
:1043C0001A98169001E01A9816901BAB40F284528E
:1043D00040F2EE414FF48B60FFF75DFD012816D1EE
:1043E0001BAB40F2845240F2EE414FF48B60FFF77A
:1043F00052FD012808D14A4890F8500040F0400092
:10440000474981F8500004E01B98179001E01B9881
:1044100017901BAB4FF4B16240F2F24140F25C40A6
:10442000FFF739FD012816D11BAB4FF4B16240F202
:10443000F24140F25C40FFF72EFD012808D13848D8
:1044400090F8500040F08000354981F8500004E0B9
:104450001B98189001E01B9818901BAB40F28C52EF
:1044600040F2F6414FF48C60FFF715FD012816D19C
:104470001BAB40F28C5240F2F6414FF48C60FFF7D8
:104480000AFD012808D1264890F8500040F080002D
:10449000234981F8500004E01B98199001E01B9813
:1044A0001990204ADDE900019062D162DDE9020144
:1044B00010625162DDE904109163D063DDE90610FA
:1044C00011635063DDE908019064D164DDE90A10ED
:1044D00011645064DDE90C109165D065DDE90E10C2
:1044E00011655065DDE910109166D066DDE91201B5
:1044F000106651668032DDE9141011605060094980
:104500001698C1F888001798C1F8940006481899C1
:10451000416605491998C1F82E001FB000BD000082
:10452000A21600208E220020F61500202DE9FE4F55
:1045300005468B4616461F460C9C4FF0000800208F
:1045400002908146824601900090C821F74832F0DF
:10455000ACFFC821F64832F0A8FFC821F54832F078
:10456000A4FFC82C01D800D802D90120BDE8FE8FD5
:104570004FF0000861E04FF00009CA4600200190AA
:10458000009022465946E94812F0B0F822463146DA
:10459000E74812F0ABF822463946E64812F0A6F892
:1045A0002246E349E14832F0A4FF08B1012000E0CF
:1045B000002081462246DF49DC4832F09AFF08B1EC
:1045C000012000E0002082462246DA49D84832F035
:1045D00090FF08B1012000E000200190B9F1000F28
:1045E00009D1BAF1000F06D1002322462946CF484F
:1045F000FEF705FE24E0B9F1000F02D0BAF1000F7A
:1046000006D1002322462946C848FEF7F8FD17E0E8
:10461000019830B9002322462946C548FEF7EFFD30
:104620000EE0002322462946C048FEF7E8FD01209F
:10463000009008F101001FFA80F8B8F1030F9ADB2F
:1046400000BF0098012800D190E700208EE7F0B568
:104650009BB001204FF454635A1E511E0090B6487F
:10466000FFF764FFB448007818B1B3480078052814
:1046700014DD0120B0490870012240F63E51AE48D9
:10468000FFF7AAFA012240F63F51AB48FFF7A4FA20
:1046900001224FF45461A848FFF79EFAA64800781B
:1046A000062831D2DFE800F030030C151E274FF446
:1046B0007F7440F292454FF4A56640F2BE5724E065
:1046C00040F2D65440F26C6540F202764FF4F36744
:1046D0001BE04FF4F66440F6460540F6DC0640F673
:1046E000721712E040F68A144FF4226540F6B6269F
:1046F00040F64C3709E040F6643440F6FA354FF4A2
:10470000496640F6265700E000BF00BF0422394644
:104710008948401C11F0EAFF8748D0F8010087491A
:10472000884209D900208449C1F801000422394691
:104730008148401C11F0CFFF682033462A462146AD
:10474000009001A8FFF7F2FE7D4ADDE901109162B9
:10475000D062DDE9031011625062DDE9051091635A
:10476000D063DDE9071011635063DDE9090190644E
:10477000D164DDE90B1011645064DDE90D01906531
:10478000D165DDE90F1011655065DDE91110916605
:10479000D066DDE91310116650668032DDE9151030
:1047A0001160506066491798C1F888001898C1F8E0
:1047B000940064481999416662491A98C1F82E001C
:1047C0001BB0F0BD10B500215F4A116051609160CF
:1047D000D160116151619161D1610020106250621C
:1047E0009162D162116351639163D1631164516429
:1047F0009164D164116551659065D065106650660D
:104800009066D066106750679167D16780321160FB
:1048100051600832106050600832116051600832F7
:1048200010605060083210605060083211605160B2
:104830000832116051600832116051600832116015
:1048400051600832116051600832116051600832C5
:104850001060506008321060506008321160516082
:10486000083211605160083210605060F83AC2F8A6
:104870000011C2F80411C2F80811C2F80C11C2F8F4
:104880001011C2F81411C2F81811C2F81C114FF41B
:1048900090724FF45C612C4811F01DFF10BD10B5F3
:1048A0004FF490724FF45C61274811F01FFF10BD68
:1048B0002DE9F047804689469246DDE908670025E4
:1048C000002406E0601CC4B2032C02DB681CC5B2E5
:1048D00006E0424630463946FEF7BCFD0128F1D0DD
:1048E00000BF002406E0601CC4B2032C02DB681C7D
:1048F000C5B206E04A4630463946FEF7ABFD012810
:10490000F1D000BF002406E0601CC4B2032C02DB1F
:10491000681CC5B206E0524630463946FEF79AFD9D
:104920000128F1D000BF2846BDE8F087FE1A00201C
:10493000C61B00208E1C0020D50000208096980009
:104940008E220020F6150020232800202DE9F047B4
:1049500006468946174698460025002406E0601C56
:10496000C4B2032C02DB681CC5B205E031464046E8
:10497000FEF78BFD0128F2D000BF002406E0601C8A
:10498000C4B2032C02DB681CC5B205E049464046B0
:10499000FEF77BFD0128F2D000BF002406E0601C7A
:1049A000C4B2032C02DB681CC5B205E039464046A0
:1049B000FEF76BFD0128F2D000BF2846BDE8F08766
:1049C0002DE9F047064689461746984600250024FB
:1049D00006E0601CC4B2032C02DB681CC5B205E013
:1049E00031464046FEF765FD0128F2D000BF06E0E3
:1049F000601CC4B2032C02DB681CC5B205E049464A
:104A00004046FEF756FD0128F2D000BF06E0601CCC
:104A1000C4B2032C02DB681CC5B205E0394640462F
:104A2000FEF747FD0128F2D000BF2846BDE8F08719
:104A30002DE9F0439BB04FF46168F84800780628F0
:104A400031D2DFE800F030030C151E274FF47F74DD
:104A500040F292454FF4A56640F2BE5724E040F282
:104A6000D65440F26C6540F202764FF4F3671BE0D7
:104A70004FF4F66440F6460540F6DC0640F6721741
:104A800012E040F68A144FF4226540F6B62640F64E
:104A90004C3709E040F6643440F6FA354FF4496685
:104AA00040F6265700E000BF00BFDD48816AC06ABB
:104AB000CDE90110DA49086A496ACDE90301D8480D
:104AC000816BC06BCDE90510D548016B406BCDE91A
:104AD0000710D348816CC06CCDE90910D049086C2F
:104AE000496CCDE90B01CE48816DC06DCDE90D104B
:104AF000CB48016D406DCDE90F10C949886EC96E74
:104B0000CDE91101C649086E496ECDE91301C448CB
:104B1000803001684068CDE91510C148D0F88800A0
:104B20001790BF48D0F894001890BE48406E199076
:104B3000BC48D0F82E001A906822214601A8FFF741
:104B40004BF86822294601A8FFF746F8682231464B
:104B500001A8FFF741F8B148D0F80100401CAF4967
:104B6000C1F8010004223946AC48401C11F0B3FDE5
:104B7000AA48D0F8010040457ED3F4F777F94FF406
:104B80000061A948FCF7E2F808B9012000E0002024
:104B900081464A464FF40061A348FCF7E8F89F4875
:104BA0000078401C9D49087008460078052801DD02
:104BB0000120087099480078062831D2DFE800F01B
:104BC00030030C151E274FF47F7440F292454FF4CA
:104BD000A56640F2BE5724E040F2D65440F26C6520
:104BE00040F202764FF4F3671BE04FF4F66440F6B0
:104BF000460540F6DC0640F6721712E040F68A14CD
:104C00004FF4226540F6B62640F64C3709E040F6F0
:104C1000643440F6FA354FF4496640F6265700E012
:104C200000BF00BF7E49886AC96ACDE901017C489E
:104C3000016A406ACDE903107949886BC96BCDE9F7
:104C400005017749086B496BCDE907017449886C08
:104C5000C96CCDE909017248016C406CCDE90B10BB
:104C60006F48816DC06DCDE90D106D48016D406DCF
:104C7000CDE90F106A4800E048E0816EC06ECDE9D2
:104C800011106748016E406ECDE913106448803002
:104C900001684068CDE915106148D0F88800179088
:104CA0005F48D0F8940018905E48406E19905D48B7
:104CB000D0F82E001A906822214601A8FEF78CFF3A
:104CC0006822294601A8FEF787FF6822314601A81D
:104CD000FEF782FF01205149C1F801000422394644
:104CE0004E48401C11F0F7FC012240F63E514B4863
:104CF000FEF772FF012240F63F514848FEF76CFF75
:104D000001224FF454614548FEF766FF6420F3F733
:104D1000D2FB1BB0BDE8F08338B54448407908B9F0
:104D200000240CE041484079012801D1012406E02B
:104D30003E484079022801D1022400E000243B488B
:104D40000094D0F8013001780022104631F068FB61
:104D500031F02BFC38BD36480078012806D10420FC
:104D60003449087000203249087015E03248007854
:104D7000012803D103202F4908700DE02E48007848
:104D8000022809D12B48007C012802D1294908704A
:104D900002E0022027490870704710B52748407884
:104DA000042813DB254800783C280FDC2148C07913
:104DB00018B901201F49C87105E0002011F08EF8D4
:104DC00000201C49C87100201C4948701948C0794E
:104DD00001280AD100201A49086001201949C1F8A8
:104DE0009C01002011F0E2F805E000201449086061
:104DF0001449C1F89C0110BD10B510484078042832
:104E00002BDB0E4800783C2827DC15F033FC0948E2
:104E1000C079C8B901200749C8711BE0D50000203E
:104E20008E220020F615002000080140E800002036
:104E3000FE000020A2160020FB000020581D0020CC
:104E40008481224200002342012011F047F8002013
:104E5000FE49C8710020FE494870FC48C07901280D
:104E600009D10020FB4908600120FB49C1F89C01E1
:104E700011F09CF808E00120F64908600020F6498E
:104E8000C1F89C0128F053F8F048007B022805DBAC
:104E90004FF46160ED49A1F80D000BE0EB48B0F86C
:104EA0000D00002806DDE948B0F80D00401EE74976
:104EB000A1F80D00E548007B092829DD4620E749D7
:104EC000087060204870672088708921E348C170AD
:104ED0004320E24908718621E04841716820DF499A
:104EE00088716821DD48C1715220DC490872862131
:104EF000DA4841727520D94988729721D748C17222
:104F00000C2242F2300111F0E6FB0020CF49087379
:104F100010BD10B505F02CFF05F04AFFD048006821
:104F2000012834D1CF48007802282ADDCE484078C5
:104F3000C0F3C000F8B1CB48407801282BD0012045
:104F4000C84948700321072028F096F9C74890F80F
:104F50006E00022802DA0120C4490874C34890F8A0
:104F60006E00FA2817DAC14890F86E00401CBF495D
:104F700081F86E000FE00020BA4948704870087050
:104F800009E0B8480078401CB649087003E00020EA
:104F9000B44948700870B2481C380068012836D1FE
:104FA000B048807802282CDDAF484078C0F300106C
:104FB000F8B1AC48C07801282DD00120A949C870AB
:104FC0000421072028F058F9A84890F86F0002281B
:104FD00002DA0120A5494874A44890F86F00FA2825
:104FE00019DAA24890F86F00401CA04981F86F00C0
:104FF00011E000209B49C8709C49487481F86F00FB
:1050000009E098488078401C9649887003E00020A9
:105010009449C870887005F0BBFE05F0D8FE10BD3D
:1050200010B5FAF749F80120F3F745FAFAF7DEF878
:105030000446FAF74FF8A4BB00208449C87008461C
:105040008078052825DD012008700846007C0128AD
:1050500024D00120087484484078C0F34000E8B1AF
:105060000221062028F008F9804890F86000042802
:1050700002DA01207D4988707C4890F86000FA28A7
:105080000CDA7A4890F86000401C784981F860009A
:1050900004E06E488078401C6C4988706B488078CA
:1050A00033E0FFE70020694988700846C07805288A
:1050B00024DD022008700846007C20B3002008741C
:1050C00069484078C0F34000E8B10221062028F08A
:1050D000D3F8664890F86000042802DA0220634999
:1050E0008870624890F86000FA280CDA5F4890F8FF
:1050F0006000401C5D4981F8600004E05348C078BE
:10510000401C5249C8705148C078FFF702FF10BDDB
:105110002DE9F041044656498979A1F5FA61C8B2F2
:10512000FEF74AF920705249C878FEF745F96070D9
:105130004F490879FEF740F9A0704D490878FEF70D
:105140003BF9E0704A494878FEF736F92071484942
:105150008878FEF731F96071A41C4649886AC96AEB
:105160006060A1604348016A406AE1602061414893
:105170008568C1680022404B284632F045FB07464F
:1051800032F048FD60613B480568416800223A4BB7
:10519000284632F039FB074632F03CFDA061354825
:1051A000D0F89800E0613348D0F89C002062314884
:1051B000D0F8880060622F49803108684968A06291
:1051C000E162A41EBDE8F0812DE9F04104462849C2
:1051D0008979A1F5FA61C8B2FEF7EEF8207024498A
:1051E000C878FEF7E9F8607021490879FEF7E4F81D
:1051F000A0701F490878FEF7DFF8E0701C49487876
:10520000FEF7DAF820711A498878FEF7D5F8607150
:105210001848826AC16A104632F063FCC4F806007E
:105220001448026A416A104632F05BFCC4F80A0076
:105230001048826BC16B104632F053FCC4F80E006C
:105240000C48026B416B104618E00000A2160020CB
:10525000581D00208481224200002342312C00206E
:105260003001234267000020EA2D00209019002021
:105270000C0000208E2200200020AC4032F031FCD7
:10528000C4F81200FE480569416900221346284609
:1052900032F0A8FC1AD2FA488569C1690022F94B9C
:1052A000284632F0B1FA074632F0B4FCC4F81600D2
:1052B000F348056941690022F24B284632F0A4FA0E
:1052C000074632F0A7FCC4F81A0019E0EC488568DC
:1052D000C1680022EC4B284632F096FA074632F0BD
:1052E00099FCC4F81600E648056841680022E64BC0
:1052F000284632F089FA074632F08CFCC4F81A00CE
:10530000DF48D0F89800C4F81E00DD48D0F89C00B3
:10531000C4F82200DD48B0F817000A2190FBF1F034
:1053200084F82600D948B0F8170090FBF1F084F813
:105330002700D7480168A1624168E1628068206364
:10534000BDE8F0812DE9F05F81464C46D14989796D
:10535000A1F5FA61C8B2FEF72FF82070CD49C878E0
:10536000FEF72AF86070CB490879FEF725F8A0709F
:10537000C8490878FEF720F8E070C6494878FEF77B
:105380001BF82071C3498878FEF716F86071A41CD9
:10539000BB48876AC16A0022BF4B384632F034FAF4
:1053A000054632F0DCFB6060A160B548056A416AE1
:1053B0000022B94B284632F027FA074632F0CFFBDD
:1053C000E0602161AE48856BC16B0022B24B28467C
:1053D00032F01AFA074632F0C2FB6061A161A848B8
:1053E000056B416B0022AC4B284632F00DFA0746A4
:1053F00032F0B5FBE0612162A41EA84800780121CB
:10540000B1EBD01F53D19E48056941690022134674
:10541000284632F0E7FB25D29948D0F818A0C16998
:105420000022984B504632F0EFF9074600229A4B83
:1054300032F0EAF9054632F035FBC4F82600904810
:105440000569416900228F4B284632F0DDF982461A
:105450000022914B32F0D8F9074632F023FBC4F812
:105460002A0048E086498D68C9680022864B284694
:1054700032F0CAF907460022874B32F0C5F982465E
:1054800032F010FBC4F826007D480768416800220E
:105490007D4B384632F0B8F9824600227E4B32F01E
:1054A000B3F9054632F0FEFAC4F82A0023E0744945
:1054B0008D68C9680022744B284632F0A5F907466A
:1054C0000022754B32F0A0F9824632F0EBFAC4F8B4
:1054D00026006B490D68496800226B4B284632F064
:1054E00093F9074600226C4B32F08EF9824632F077
:1054F000D9FAC4F82A006248D0F898002E346060C7
:105500005F48D0F89C0020605D48D0F8B100A060F2
:105510005B48D0F888006061594980310D6849685E
:1055200000225F4B284632F06FF9074632F0F2FA5C
:10553000E0600E34C4F802105449B1F8170032F09C
:1055400063FA0746574A584B32F05EF9054632F087
:10555000C8FAA0724D48407EE0724C49B1F817007D
:1055600032F052FA07464F4A4F4B32F04DF905469A
:1055700032F0B7FA20734548407E60734B4890F88C
:105580003000A073494890F83200E073474890F823
:1055900034002074454890F836006074434890F811
:1055A0003800A074414890F83A00E0743F4890F801
:1055B0003C0020753D4890F83D0060753B4890F8F0
:1055C0003E00A075394890F83F00E075374890F8E4
:1055D00040002076354890F841006076334890F8D6
:1055E0004200A076314890F84300E0762F4890F8CA
:1055F000440020772D4890F8450060772B4890F8BC
:105600004600A077294890F84700E07727480068CF
:10561000206226484068606224488068A06223486F
:10562000C068E062214800692063204840696063E7
:105630001E48406AA0631D48806AE0631B48C06A38
:1056400020641A48806C60641848C06CA0641748D5
:10565000006DE0640E480088A4F850003C3C0C4803
:10566000418804F18C00A4F88E100948818804F167
:105670008C00A4F890100648C18804F18C0017E053
:105680008E2200200020ACC00020AC40A2160020DA
:10569000C62D00200C0000200088C340D22D002021
:1056A00000408F409A9999999999B93F062E002008
:1056B000A4F89210FE48018904F18C00A4F894101B
:1056C000FB48418904F18C00A4F89610BDE8F09FD6
:1056D0002DE9F041F7498979A1F5FA61C8B2FDF7E2
:1056E0006BFEF5490870F349C878FDF765FEF2498D
:1056F0004870F0490879FDF75FFEEF498870ED4981
:105700000878FDF759FEEC49C870EA494878FDF77A
:1057100053FEE9490871E7498878FDF74DFEE649EF
:105720004871E6480088C880E4484188E248018121
:10573000E2488188E0484181E048C188DE488181B3
:10574000DE480189DC48C181DC484189DA480182B0
:10575000DA488189D8484182D948836AC16AD64AE1
:1057600014321846FDF734FED548036A416AD24A1E
:105770001A321846FDF72CFED148836BC16BCE4A16
:1057800020321846FDF724FECD48036B416BCA4A10
:1057900026321846FDF71CFECA4800780121B1EBFD
:1057A000D01F3ED1C64804694169002213462046F5
:1057B00032F018FA1AD2C2488669C1690022C24B77
:1057C000304632F021F8044632F024FABA49C86271
:1057D000BB490E6949690022BB4B304632F014F8D0
:1057E000044632F017FAB449086334E0B4498E68CD
:1057F000C9680022B54B304632F006F8044632F054
:1058000009FAAD49C862AE48066841680022AF4B4C
:10581000304631F0F9FF044632F0FCF9A64908633E
:1058200019E0A7488668C1680022A84B304631F0CD
:10583000EBFF044632F0EEF99F49C862A0480668C3
:1058400041680022A14B304631F0DEFF044632F0C1
:10585000E1F9994908639A48D0F898009649486355
:105860009748D0F89C0088639548D0F8B100C86389
:105870009748407D81F840009548807D81F841003F
:105880009348407D81F842009148807D81F8430033
:10589000904890F8300081F844008E4890F832002B
:1058A00081F845008B4890F8340081F8460089481B
:1058B00090F8360081F84700864890F8380081F863
:1058C0004800844890F83A0081F84900814890F8EF
:1058D0003C0081F84A007F4890F83D0081F84B0079
:1058E0007C4890F83E0081F84C007A4890F83F00E0
:1058F00081F84D00774890F8400081F84E007548D7
:1059000090F8410081F84F00724890F8420081F809
:105910005000704890F8430081F851006D4890F8AD
:10592000440081F852006B4890F8450081F853001C
:10593000684890F8460081F85400664890F847009F
:1059400081F8550063480068C1F856006148406816
:10595000C1F85A005F488068C1F85E005D48C068C1
:10596000C1F862005B480069C1F8660059484069A7
:10597000C1F86A005748406AC1F86E005548806A0D
:10598000C1F872005348C06AC1F876005148806C73
:10599000C1F87A004F48C06CC1F87E004D48006DD8
:1059A000C1F8820042480088A1F88600404841883A
:1059B0004148A0F888103E4881883F48A0F88A10E6
:1059C0003B48C1883C48A0F88C10394801893A48C6
:1059D000A0F88E10364841893748A0F89010BDE8ED
:1059E000F0812DE9F041044632498979A1F5FA6147
:1059F000C8B2FDF7E1FC384908702E49C878FDF7B8
:105A0000DBFC354948702B490879FDF7D5FC324954
:105A1000887028490878FDF7CFFC2F49C8702549C0
:105A20004878FDF7C9FC2C49087122498878FDF7B0
:105A3000C3FC294948712248856AC16A264A921DD9
:105A40002846FDF7C5FC1E48056A416A224A0C3209
:105A50002846FDF7BDFC1A498D68C96800221B4B1A
:105A6000284631F0D1FE07461B4A1832FDF7B0FC3C
:105A700013490D6849680022144B284631F0C4FED2
:105A80000746154A1E32FDF7A3FC0D48D0F89800D2
:105A9000114948620A48D0F89C0088620C48407D51
:105AA00081F82C000A48807D81F82D00094815E016
:105AB000C62D00200C000020531E0020DC2D0020ED
:105AC0008E220020D22D00200020ACC00020AC404F
:105AD000A2160020062E00202B18002090F830007F
:105AE00081F82E00FE4890F8340081F82F00FC4821
:105AF00090F8320081F83000F94890F8360081F8CB
:105B00003100F74890F83C0081F83200F44890F8F2
:105B10003E0081F83300F24890F83D0081F83400EF
:105B2000EF4890F83F0081F83500ED48406AC1F831
:105B30003600EB48806AC1F83A00E948806CC1F849
:105B40003E00E748C06CC1F8420046222146E548C5
:105B5000FDF747FBBDE8F081F0B59BB000240027BE
:105B600000250026E048407820B9DF48807808B951
:105B7000012700E00027DC48007838B9DA4840788F
:105B800020B9D948807808B9012500E00025D64819
:105B9000007901280AD1D448007838B9D248407831
:105BA00020B9D148807808B9012600E00026CF4806
:105BB000008860B1CC484078CC49098890FBF1F26C
:105BC00001FB120018B9C848807800B901240024EC
:105BD000002700250026C648407900F00F00032862
:105BE0000BD0C348407900F00F00062805D0C0480C
:105BF000407900F00F00092803D101240127012575
:105C00000126012F06D10EA8FFF782FA0EA9012066
:105C100013F08DFD012D06D10EA8FFF779FA0EA91C
:105C2000022013F084FD012E06D10EA8FFF770FAB2
:105C30000EA9032013F07BFD012C06D101A8FFF76C
:105C4000C3FA01A9042013F034FD1BB0F0BD10B558
:105C5000FEF7EEFE10BD10B50024FDF7B3FFA5481A
:105C6000C079012803D0A348007A01280CD1002074
:105C7000A049C8710872012C02D0FEF7D9FE012498
:105C800000209D49A1F821009B48B0F82100B0F503
:105C9000967F09DB012C02D0FEF7CAFE012400200A
:105CA0009549A1F8210006E09348B0F82100401C76
:105CB0009149A1F8210010BD2DE9F0418A484078B2
:105CC00000287DD1884880780028FAD18B48046864
:105CD00043688B48066A416A2246304631F08EFDA1
:105CE000864AC03A1061516102F1C80004684368F5
:105CF00083498E6AC96A2246304631F07FFD7F4A69
:105D0000C03A9061D16102F1F000046843687C48B8
:105D1000066B416B2246304631F070FD774AC03A3F
:105D20001067516702F1F800046843687448866B95
:105D3000C16B2246304631F061FD704AC03A90672F
:105D4000D16702F1D000046843686D490E6A496A60
:105D50002246304631F052FD684AC03A1062516224
:105D600002F1D8010C684B6865498E6AC96A2246FF
:105D7000304631F043FD614AC03A9062D16210462C
:105D8000D0F80041D0F804315D490E6B496B2246D2
:105D9000304631F033FD594A403A10605160A2F16B
:105DA0008000D0F80841D0F80C3155498E6BC96B92
:105DB0002246304631F022FD504A383A106000E069
:105DC0004EE1516002F158010C684B684C490E6A73
:105DD000496A2246304631F011FD484AC03A106403
:105DE000516402F1E800046843684548866AC16A64
:105DF0002246304631F002FD404AC03A9064D164F8
:105E00001046D0F81041D0F814313D490E6B496B63
:105E10002246304631F0F2FC384A203A1060516098
:105E2000A2F1A001D1F81841D1F81C313448866B99
:105E3000C16B2246304631F0E1FC304A183A10601E
:105E400051602F48016A406A1832116050602C4836
:105E5000816AC06A0832116050602949086B496B39
:105E60002832106051602648816BC06B0832116087
:105E7000506008224FF46861204810F02CFC082282
:105E800040F688611D48083010F025FC08224FF4C8
:105E90006B611A48303010F01EFC082240F6B861E1
:105EA0001648383010F017FC0F480078002870D1E1
:105EB0001248C038016A406A104AC03A1163506300
:105EC0001146886AC96A9063D16302F1800108684B
:105ED0004968903210605160A2F10800016811E039
:105EE000062E00202B1800200C000020EE000020C1
:105EF000140000209D180020A2160020E328002096
:105F00008E22002040680832116050600021983ACB
:105F1000116251629162D162002080321060506043
:105F2000083210605060FE49086A496A48321060C1
:105F30005160FB49886AC96A083210605160F848AC
:105F4000016B406BD83AC2F80011C2F80401F44862
:105F5000816BC06BC2F80811C2F80C0108224FF423
:105F60006961F04810F0B7FB082240F69861ED48EF
:105F7000083010F0B0FB08224FF46C61E948303073
:105F800010F0A9FB082240F6C861E648383010F04E
:105F9000A2FBE5480079012862D1E3480078002897
:105FA0005ED1E048D038016C406CDE4AD03A1165D1
:105FB00050651046816CC06C9165D06502F1A000FF
:105FC00001684068B03211605060A2F108000168B9
:105FD00040680832116050600021B83A1164516481
:105FE0009164D1640020A0321060506008321160CA
:105FF0005160CB48016A406A383211605060C8482D
:10600000816AC06A083211605060C548016B406BFC
:10601000E83AC2F81011C2F81401C148816BC06B94
:10602000C2F81811C2F81C0108224FF46A61BD4879
:10603000103010F050FB082240F6A861B948183023
:1060400010F049FB08224FF46D61B648403010F063
:1060500042FB082240F6D861B248483010F03BFBC2
:10606000B148407850B9B0488078032806D1C022A2
:106070004FF45C61AB48D03810F02DFBBDE8F081E7
:106080002DE9FF478146A9490868A94931F0D7FAA7
:106090000546494631F0DAFD31D8A648807AC0F38A
:1060A000C00010B3A44890F86E0001282BD0012046
:1060B000A14981F86E006021052027F0DDF89F4896
:1060C00090F87E00022803DA01209C4981F8200024
:1060D0009A4890F87E00FA2815DA984890F87E00E1
:1060E000401C964981F87E000DE00020924981F81D
:1060F0006E00924981F8200081F87E0003E00020C4
:106100008D4981F86E008C4890F868008A4901EB4F
:106110008000C0F80090084690F86800401C81F8A4
:106120006800084690F86800142802D1002081F821
:106130006800814890F8690014286FD14FF0000A78
:10614000002409E07C4800EB84000168504631F0EF
:10615000ECF98246601CC4B2142CF3DB784950463B
:1061600031F06DFA7449C86570494868704931F07A
:1061700066FA05467048C16D284631F067FD7DD24C
:1061800000206D4981F86D00084690F86C000A28DF
:1061900075DD6349D1F8D10031F0F9FC07460022E2
:1061A000684B31F031FB0022674BCDE9000131F043
:1061B0009DFB05460E466049C86D31F0E8FC2A4655
:1061C0003346CDE9020131F00DFD32D25948807AD3
:1061D000C0F3401018B3584890F8700001281CD044
:1061E0000120554981F870006221052027F044F80C
:1061F000524890F88000022803DA01204F4981F8C4
:1062000022004E4890F88000FA2870DA4B4890F847
:106210008000401C494981F8800068E060E000206F
:10622000454981F87000454981F8220081F88000D5
:106230005DE00020404981F870003E48807AC0F35C
:10624000001020B3084690F86F0001284FD00120BD
:1062500081F86F006121052027F00EF8374890F88B
:106260007F00022803DA0120344981F821003348F5
:1062700090F87F00FA283ADA304801E019E010E09F
:1062800090F87F00401C2D4981F87F002FE000200E
:10629000294981F86F00294981F8210081F87F00A0
:1062A00025E0254890F86C00401C234981F86C00DB
:1062B0001DE00020204981F86C00084690F86D0030
:1062C0000A2805DD002081F8700081F86F000EE0DB
:1062D000194890F86D00401C174981F86D0006E0E0
:1062E000154890F86900401C134981F8690012486C
:1062F00090F86F00BDE8FF8700207047704710B529
:106300002FF0FEFF114908700846007838B10120CF
:1063100030F06DF900200D490870012010BD17E024
:106320008E220020F32800200C000020DB2B002010
:1063300000006145EA2D00201F190020901900205F
:106340000000A0410000F43F0020AC406C000020A1
:10635000002010BD1CB5694601A82FF046FFFE497C
:1063600008709DF8040001280FD10846007848B154
:10637000002030F03CF90020F74908700120F7496F
:10638000487202E00020F54948721CBD0020F44923
:106390000870087148700120C8700020C1F805001D
:1063A00070470020EF490860EF49C1F8AC01704721
:1063B00070B505460C4626460120307003207070EB
:1063C000281D81B22046F9F7F1FA70BD10B50346D9
:1063D000002009E0441C145D0C54441CA0B2441E6F
:1063E000145D0C54441CA0B29842F3DB10BDDB4892
:1063F000C079012800D17047D848007A012801D11E
:106400000220F8E7D548007C012801D10320F2E7FB
:10641000D2484079012801D10420ECE7D3488078A4
:10642000012801D10520E6E7CC488079012805D173
:1064300000BFCA4880790028FBD1DCE70020DAE7FA
:10644000C648B0F86100102803D10320C349087082
:106450007047C248B0F861005A2803D10420BF49F0
:106460000870F5E7BD48B0F86100202807D1BB48A7
:106470000078032803D10120B8490870E8E7B7483D
:106480000078E5E7704700B5B548D0F80500B0F5ED
:10649000616F02D90220B6490870FEF75CFCFFF775
:1064A000F1FF002000BD10B5F3F755FDF2F72BFC0E
:1064B000F2F7BBFC4FF4E130F2F716FE04F035FFC3
:1064C00008F047FE01200FF02DFD26F025FD14F009
:1064D000D1F809F0F7F90020A649087048709F49E3
:1064E000C871487208720846807C4874002081F8A0
:1064F000370081F8380081F8390081F83E0081F8D2
:1065000045009D490870012048710020887148703D
:10651000C87088759149A1F81D00A1F8210081F883
:10652000270081F82800A1F82500A1F82300052004
:1065300081F8290081F82A00084690F82900801E79
:10654000A1F82500084690F82A00801EA1F8230033
:1065500008F040FB00208149A1F80D00C87485496E
:106560004871012088700020C87008718349087044
:106570000FF0B2FA012007F077FF7849B1F81F0059
:10658000F2F7A9FB10BD10B5F3F7E5FCF2F7BBFB82
:1065900000207B4908607B49C1F8BC017849203163
:1065A0000860774914310860091F08607149087054
:1065B00048706A49C871487208728872012048742C
:1065C000002081F8370081F8380081F8390081F81F
:1065D0003E0081F84500684908700120487100209C
:1065E00088714870C8708875674981F809015B49EE
:1065F00081F8280081F827003C2081F8290081F8E3
:106600002A00084690F82900801EA1F825000846B7
:1066100090F82A00801EA1F8230008F0DBFA002081
:106620004E4981F82C00A1F81D00A1F82100C87482
:1066300050494871012088700020C87008710FF01F
:106640004BFA08F086FD04F070FEFCF79FFE002078
:106650000FF068FC022007F007FF4049B1F81F0067
:10666000F2F739FB6420F1F726FF10BD38B5044678
:1066700040F2754084422DD040F28D40844202D1D8
:1066800009F020F926E040F29D40844222D0801C8F
:1066900084421FD0801C84421CD13C48407908B9F8
:1066A00000250CE039484079012801D1012506E098
:1066B00036484079022801D1022500E00025334800
:1066C0000095D0F801300178002210462FF0A8FE86
:1066D0002FF06BFF38BD70477047704770477047A9
:1066E00070477047704700B5FFF7F9FFFFF7F6FFF7
:1066F000FFF7F3FFFFF7EFFFFFF7EEFFFFF7F0FF06
:10670000FFF7EFFF00BD7047002000BF06E000224A
:106710001F4901EB40010A80411CC8B20728F6DB83
:1067200070471C4800781C49097988427DD01A4876
:10673000007918490870002081F8600081F8610034
:1067400081F8620081F8630081F8640081F86500D7
:1067500081F8660022E000006B000020A2160020F5
:106760005F1A0020BC0121420000234206010020E4
:10677000FB00002004000020581D00206D000020B8
:106780008C012342000021428E220020E8000020DC
:106790001E1F0020901900200C00002081F86700C7
:1067A00081F8680081F8690081F86A0081F86B005F
:1067B00081F86C0081F86D0081F86E0081F86F003F
:1067C00081F8700081F8710081F8720081F873001F
:1067D00081F8740081F8750081F8760081F87700FF
:1067E00081F8780081F8790081F87A0081F87B00DF
:1067F00081F87C0081F87D0081F87E0081F87F00BF
:1068000081F8800081F8810081F8820081F883009E
:1068100081F8840081F8850081F8860081F887007E
:1068200081F8880081F8890000E029E081F88A0079
:1068300081F88B0081F88C0081F88D0081F88E0042
:1068400081F88F0081F8900081F8910081F8920022
:1068500081F8930081F8940081F8950081F8960002
:1068600081F8970081F8980081F8990081F89A00E2
:1068700081F89C0081F89D0081F89E0081F89B00C2
:10688000704710B50024FFF74CFF2BF0CDFF012817
:1068900007D10124FB48807820F020002030F949FE
:1068A00088702CF06EF8012807D10124F548807813
:1068B00020F040004030F34988702CF0F5F80128B2
:1068C00007D10124EF48807820F010001030ED4906
:1068D0008870ED4890F8A100B42812D1EA4890F8E9
:1068E000A100401CE84981F8A100E848407800F088
:1068F000010000B30846007B01281CD0012008736A
:1069000019E0E14890F8A100FA2806DADE4890F88C
:10691000A100401CDC4981F8A100DB4890F8A100EF
:10692000012808D1D948407800F0010018B10121B0
:10693000084626F0A1FCD448807A012822D1002004
:10694000D1498872D2480078C0F3401038B1CD48A0
:10695000007820F020002030CA4908700124CD487A
:106960000078C0F3800068B1CA480078C0F3C00066
:1069700020B1042163202DF0ABFF03E0012163204F
:106980002DF0A6FFC048007B012812D1C0484078F6
:1069900000F0010050B1BB48407820F00100401CDD
:1069A000B849487001240420BB4988730020B649C7
:1069B0000873B5488078012810D10020B24988704A
:1069C000B3484078C0F3400050B3AE48407820F060
:1069D0000200801CAB494870012426E0AA48807858
:1069E000022822D10020A8498870A9484078C0F325
:1069F000400038B1A348407820F00200801CA14933
:106A000048700124A3480078C0F3001040B1A148A9
:106A10000078C0F3401020B1042170202DF058FF01
:106A200003E0012170202DF053FF9748007C0128DE
:106A300022D100209449087495484078C0F3C000E2
:106A400038B19048407820F0080008308D494870EF
:106A500001249048407800F0010068B18D484078EA
:106A6000C0F3400020B1042103202DF031FF03E0EA
:106A7000012103202DF02CFF8348407C012822D1E6
:106A800000208149487482484078C0F3001038B132
:106A90007C48407820F0100010307A49487001247A
:106AA0007C484078C0F3800068B17A484078C0F3F1
:106AB000C00020B1042108462DF00AFF03E00121A7
:106AC00004202DF005FF704890F83F00012823D1E5
:106AD00000206D4981F83F006D48807800F001008A
:106AE00038B16848807820F00100401C6549887002
:106AF00001246848807800F0010068B1654880781A
:106B0000C0F3400020B1042170202DF0E1FE03E02D
:106B1000012170202DF0DCFE5B4890F83E0001283A
:106B20001FD10020584981F83E005948C07A00F032
:106B3000010018B101205349C87201245548007D55
:106B400000F0010068B15348007DC0F3400020B15F
:106B5000042171202DF0BCFE03E0012171202DF0F5
:106B6000B7FE494890F84000012810D1002046495E
:106B700081F8400046488078C0F3400038B1414871
:106B8000807820F00200801C3E49887001243E4835
:106B900090F83A00012810D100203B4981F83A00D2
:106BA0003B48C078C0F3C00038B13648C07820F008
:106BB000080008303349C8700124334890F83B007E
:106BC000012810D10020304981F83B003048C078BE
:106BD000C0F3001038B12B48C07820F010001030FE
:106BE0002849C8700124284890F83C00012810D199
:106BF0000020254981F83C002548C078C0F34010AA
:106C000038B12048C07820F0200020301D49C870DD
:106C100001241D4890F83D00012810D100201A4998
:106C200081F83D001A48C078C0F3801038B115488B
:106C3000C07820F0400040301249C870012412484A
:106C4000C07801282ED100200F49C8701048007963
:106C500000F0010038B10B48007920F00100401C21
:106C60000849087101240B48807900F00100C8B17F
:106C700008488079C0F3400080B1042110202DF035
:106C800027FE0FE0DC2D002090190020EA2D0020C7
:106C9000F82D002011010020921F0020012110205A
:106CA0002DF016FEFD480079012822D10020FB4975
:106CB0000871FB480079C0F3400038B1F948007909
:106CC00020F00200801CF74908710124F648807901
:106CD000C0F3800068B1F4488079C0F3C00020B1EF
:106CE000042111202DF0F4FD03E0012111202DF0ED
:106CF000EFFDEA48C07B012822D10020E749C87394
:106D0000E7480079C0F3800038B1E648007920F008
:106D10000400001DE34908710124E3488079C0F3B1
:106D2000001068B1E0488079C0F3401020B1042120
:106D300012202DF0CDFD03E0012112202DF0C8FD21
:106D4000D64890F84200012823D10020D34981F889
:106D50004200D3484079C0F3401038B1D14840795F
:106D600020F020002030CF4948710124CE48407ADD
:106D7000C0F3001068B1CC48407AC0F3401020B195
:106D8000042117202DF0A4FD03E0012117202DF090
:106D90009FFDC248807C012822D10020BF49887411
:106DA000BF48807900F0010038B1BE48807920F0FA
:106DB0000100401CBB4988710124BB48007B00F0E6
:106DC000010068B1B848007BC0F3400020B1042145
:106DD00020202DF07DFD03E0012120202DF078FD05
:106DE000AE48C07C012822D10020AC49C874AC4810
:106DF0008079C0F3400038B1AA48807920F00200C1
:106E0000801CA84988710124A748807A00F00100FD
:106E100068B1A548807AC0F3400020B10421212048
:106E20002DF056FD03E0012121202DF051FD9B485E
:106E3000007D012822D10020984908759848807962
:106E4000C0F3800038B19748807920F00400001D1D
:106E50009449887101249448807AC0F3800068B115
:106E60009148807AC0F3C00020B1042122202DF087
:106E70002FFD03E0012122202DF02AFD8748407DCF
:106E8000012822D100208549487585488079C0F3C2
:106E9000C00038B18348807920F00800083081496B
:106EA000887101248048807AC0F3001068B17E4860
:106EB000807AC0F3401020B1042123202DF008FD7A
:106EC00003E0012123202DF003FD7448807D01287B
:106ED00023D100207149887571488079C0F3001072
:106EE00038B17048807920F0100010306D498871F9
:106EF00001246D48807AC0F3801070B16A48807AAE
:106F00000121B1EBD01F04D1042124202DF0E0FC9D
:106F100003E0012124202DF0DBFC6048007E0128E5
:106F200022D100205D4908765D488079C0F3401089
:106F300038B15C48807920F02000203059498871B0
:106F400001245948007BC0F3001068B15648007B0B
:106F5000C0F3401020B1042130202DF0B9FC03E033
:106F6000012130202DF0B4FC4C48407E012823D173
:106F700000204A4948764A488079C0F3801038B1E9
:106F80004848807920F0400040304649887101240B
:106F90004548007BC0F3801070B14348007B01215D
:106FA000B1EBD01F04D1042131202DF091FC03E07E
:106FB000012131202DF08CFC3848C07D012823D1DF
:106FC00000203649C875364880790121B1EBD01FC1
:106FD00007D13448807920F08000803031498871B1
:106FE00001243148407B00F0010068B12E48407B0D
:106FF000C0F3400020B1042132202DF069FC03E0F1
:10700000012132202DF064FC2448807E012822D109
:107010000020224988762248C07900F0010038B16A
:107020002048C07920F00100401C1E49C87101248D
:107030001D48007BC0F3800068B11B48007BC0F393
:10704000C00020B1042125202DF042FC03E00121E5
:1070500025202DF03DFC1148C07E01282AD10020BA
:107060000E49C8760E48C079C0F3400038B10D48CB
:10707000C07920F00200801C0A49C87101240A4826
:10708000C07A00F00100A8B10748C07AC0F3400000
:1070900060B1042126202DF01BFC0BE0901900208C
:1070A000F82D0020DC2D00201101002001212620D8
:1070B0002DF00EFCF848007F012822D10020F6496F
:1070C0000877F648C079C0F3800038B1F448C07939
:1070D00020F00400001DF249C8710124F148C07A73
:1070E000C0F3800068B1EF48C07AC0F3C00020B19F
:1070F000042127202DF0ECFB03E0012127202DF0B7
:10710000E7FBE548407F012822D10020E24948778B
:10711000E248C079C0F3C00038B1E148C07920F03E
:1071200008000830DE49C8710124DE48C07AC0F387
:10713000001068B1DB48C07AC0F3401020B10421D0
:1071400028202DF0C5FB03E0012128202DF0C0FBF5
:10715000D148807F012823D10020CF498877CF48AC
:10716000C079C0F3001038B1CD48C07920F01000CC
:107170001030CB49C8710124CA48C07AC0F38010CE
:1071800070B1C848C07A0121B1EBD01F04D10421ED
:1071900029202DF09DFB03E0012129202DF098FBF3
:1071A000BD4890F82A0001282DD10020BA4981F865
:1071B0002A00BA48407AC0F3400060B1BA488079EA
:1071C000C0F3401038B1B648407A20F00200801C6D
:1071D000B34948720124B348007CC0F3800090B1E9
:1071E000B1488079C0F3401068B1AE48007CC0F36C
:1071F000C00020B1042149202DF06AFB03E00121E9
:1072000049202DF065FBA44890F8390001282DD1C4
:107210000020A14981F83900A048407AC0F38000DD
:1072200060B1A1488079C0F3401038B19C48407AE1
:1072300020F00400001D9A49487201249948007CFE
:10724000C0F3001090B198488079C0F3401068B145
:107250009448007CC0F3401020B1042150202DF050
:1072600037FB03E0012150202DF032FB8A4890F8D3
:10727000230018B30020884981F823008748007A4A
:1072800000F0010038B18648007A20F00100401C6F
:107290008349087201248348807B00F0010068B1B3
:1072A0008048807BC0F3400020B1042141202DF0B4
:1072B0000FFB03E0012141202DF00AFB764890F8F6
:1072C000240018B30020744981F824007348007A20
:1072D000C0F3400038B17248007A20F00200801CF0
:1072E0006F49087201246F48807BC0F3800068B149
:1072F0006C48807BC0F3C00020B1042142202DF0F7
:10730000E7FA03E0012142202DF0E2FA624890F80A
:10731000250018B30020604981F825005F48007AF5
:10732000C0F3800038B15E48007A20F00400001DF0
:107330005B49087201245B48807BC0F3001068B190
:107340005848807BC0F3401020B1042143202DF029
:10735000BFFA03E0012143202DF0BAFA4E4890F81D
:107360002700F8B100204C4981F827004B48007AEB
:10737000C0F3C00038B14A48007A20F00800083055
:107380004749087201244748807BC0F3801048B108
:107390004448807B0121B1EBD01F04D1042144205B
:1073A0002DF096FA03E0012144202DF091FA3A489D
:1073B00090F82C0018B30020374981F82C0037488A
:1073C000007AC0F3001038B13548007A20F0100080
:1073D00010303349087201243248C07B00F00100AC
:1073E00068B13048C07BC0F3400020B10421452083
:1073F0002DF06EFA03E0012145202DF069FA2648B0
:1074000090F8280018B30020234981F82800234869
:10741000007AC0F3401038B12148007A20F02000F3
:1074200020301F49087201241E48C07BC0F3800031
:1074300068B11C48C07BC0F3C00020B104214620C5
:107440002DF046FA03E0012146202DF041FA1248C2
:1074500090F82900F8B100200F4981F829000F4861
:10746000007AC0F3801038B10D48007A20F0400057
:1074700040300B49087201240A48C07BC0F3001059
:1074800048B10848C07BC0F3401078B104214720C0
:107490002DF01EFA0EE00DE090190020F82D0020CE
:1074A000DC2D002011010020D22D002001214720D9
:1074B0002DF00EFAFE4890F82B0000B30020FC4996
:1074C00081F82B00FB48007A0121B1EBD01F07D1D6
:1074D000F948007A20F080008030F74908720124D2
:1074E000F648C07BC0F3801048B1F448C07B01214E
:1074F000B1EBD01F04D1042140202DF0E9F903E0C5
:10750000012140202DF0E4F9E94890F82A0018B351
:107510000020E74981F82A00E648407AC0F340009D
:1075200038B1E548407A20F00200801CE2494872F8
:107530000124E248007CC0F3800068B1DF48007C91
:10754000C0F3C00020B1042149202DF0C1F903E0AF
:10755000012149202DF0BCF9D54890F8260080B1D2
:107560000020D34981F82600D248407AC0F30010A9
:1075700038B1D148407A20F010001030CE4948721E
:107580000124CB48C07F012822D10020C849C877F8
:10759000C848807AC0F3400038B1C748807A20F0EC
:1075A0000200801CC44988720124C448807CC0F356
:1075B000800068B1C148807CC0F3C00020B10421C4
:1075C00006202DF085F903E0012106202DF080F939
:1075D000B74890F82000012824D10020B44981F850
:1075E0002000B448807AC0F3C00038B1B248807A35
:1075F00020F008000830B04988720124AF48807C30
:10760000C0F3801070B1AD48807C0121B1EBD01F78
:1076100004D1042160202DF05BF903E001216020FA
:107620002DF056F9A24890F82100012823D100201E
:107630009F4981F821009F48807AC0F3001038B13B
:107640009D48807A20F0100010309B4988720124F8
:107650009A48C07C00F0010068B19848C07CC0F333
:10766000400020B1042161202DF032F903E0012116
:1076700061202DF02DF98E4890F82200012823D1A9
:1076800000208B4981F822008A48807AC0F340109C
:1076900038B18948807A20F02000203086498872ED
:1076A00001248648C07CC0F3800068B18348C07C58
:1076B000C0F3C00020B1042162202DF009F903E0DD
:1076C000012162202DF004F9794890F82D0001285D
:1076D00010D10020764981F82D007648007B00F01B
:1076E000010038B17448007B20F00100401C724951
:1076F000087301246E4890F83800012810D100204A
:107700006B4981F838006B48007BC0F3400038B10A
:107710006948007B20F00200801C6749087301243F
:10772000634890F82E00012810D10020604981F8AC
:107730002E006048407B00F0010038B15E48407B7D
:1077400020F00100401C5C4948730124584890F81F
:107750002F00012810D10020554981F82F005548ED
:10776000007BC0F3401038B15348007B20F020006C
:1077700020305149087301244D4890F83000012809
:1077800010D100204A4981F830004A48007BC0F3FC
:10779000C00038B14848007B20F008000830464956
:1077A00008730124424890F83100012810D10020CC
:1077B0003F4981F831003F48007BC0F3800038B179
:1077C0003D48007B20F00400001D3B490873012464
:1077D000374890F83200012810D10020344981F850
:1077E00032003448407BC0F3400038B13248407B1F
:1077F00020F00200801C3049487301242C4890F886
:107800003700012810D10020294981F83700294884
:10781000407BC0F3800038B12748407B20F0040053
:10782000001D254948730124214890F833000128A0
:1078300010D100201E4981F833001E48007BC0F3A0
:10784000801038B11C48007B20F0400040301A49BD
:1078500008730124164890F83400012810D1002044
:10786000134981F834001348407BC0F3C00038B19D
:107870001148407B20F0080008300F49487301246C
:107880000B4890F83500012810D10020084981F8F4
:1078900035000848407BC0F3001038B10648407BF3
:1078A00020F010001030044948730124004807E01C
:1078B00090190020F82D0020DC2D0020110100205F
:1078C00090F83600012810D10020FE4981F83600DA
:1078D000FD48007BC0F3001038B1FC48007B20F06D
:1078E00010001030F94908730124002C04DD012038
:1078F000F4494870F649C87410BD10B5F548007ACF
:10790000C0F30010002850D0F348407A012830D14D
:10791000EC4890F8530004281FDDEF48807A0128D6
:1079200022D00120EC498872452025F03FFDE54832
:1079300090F88A00022803DA0120E24981F82C003D
:10794000E04890F88A00FA280EDADE4890F88A00BB
:10795000401CDC4981F88A0006E0DA4890F85300C0
:10796000401CD84981F853000020D64981F85F00B7
:1079700027E0D44890F85F0004280ADDD648807AD2
:1079800070B10020D449887241F2450025F00EFD07
:1079900006E0CC4890F85F00401CCA4981F85F00BF
:1079A0000020C84981F853000BE00020CA498872C2
:1079B000C44981F82C0081F88A0081F8530081F8CD
:1079C0005F0010BD10B50446C34840792070002008
:1079D000C1494871C14890F8E600012817D1C04854
:1079E000407900F00400042800D14871BC48407977
:1079F00000F00200022801D1B7494871B848407927
:107A000000F00100A0B10120B349487110E0B44872
:107A1000407900F00400042802D1AF49487107E022
:107A2000AF48407900F00200022801D1AA4948710C
:107A3000A948407900285FD0A7484079217888423A
:107A40005AD0A548407900F00100C0B1522025F07D
:107A5000ADFC9C4890F88400022803DA0320994981
:107A600081F82600974890F88400FA2844DA95486F
:107A700090F88400401C934981F884003CE09648CB
:107A8000407900F00400042818D1522025F08EFC23
:107A90008C4890F88400022803DA0120894981F893
:107AA0002600884890F88400FA2825DA854890F85E
:107AB0008400401C834981F884001DE08648407999
:107AC00000F00200022817D1522025F06FFC7D48FB
:107AD00090F88400022803DA02207A4981F826000F
:107AE000784890F88400FA2806DA764890F88400FE
:107AF000401C744981F8840010BD2DE9F04F89B015
:107B000000BF00BF00BF00BF7248007A00F0010054
:107B100000287DD07048807A01287AD06E4840795C
:107B2000002876D16D4890F8E600012814D16D4AFE
:107B3000D16C906C2FF0F9FC01906A48016D0198AE
:107B40002FF0F3FC684902902FF079FD039030F09C
:107B50001EF804460D460EE0624AD16C906C2FF080
:107B6000E4FC4FF0804102902FF069FD039030F06B
:107B70000EF804460D465B49886C30F008F8224642
:107B80002B46CDE902012FF039FE06460F460022B2
:107B900013463046394630F00DF801D287F00047E1
:107BA0005049C86C2FF0F3FF22462B46CDE9020165
:107BB0002FF024FE8046894600221346404649465F
:107BC0002FF0F8FF01D289F000494649086D2FF0E7
:107BD000DEFF22462B46CDE902012FF00FFE824642
:107BE0008B4600221346504659462FF0E3FF02D23F
:107BF00087F0004BB24600221346204629462FF05C
:107C0000D9FF01D285F000453849D1F80A0001E0DA
:107C10008BE196E1002130F019F816D02F49D1F808
:107C2000CD0033492FF0D9FC324901902FF007FDE8
:107C300002902E48D0F80A1002982FF000FD039011
:107C40002FF0A5FFCDE9040114E02449D1F8CD00BF
:107C500027492FF0C2FC274900902FF0F0FC01903B
:107C60002FF095FF244A254BCDE902012FF03EFE6F
:107C7000CDE9040120462946DDE904232FF09AFFCF
:107C80000FD800221E4BDDE904012FF02FFE002249
:107C90004FF08043CDE902012FF028FECDE9060127
:107CA00038E0184908882FF0AFFE22462B46CDE970
:107CB00000012FF0A9FD144A144BCDE902012FF069
:107CC000A3FD25E090190020F82D0020DC2D0020D8
:107CD000921F0020EA2D0020321A00208E22002060
:107CE000D22D0020062E00200000404098230020C6
:107CF00000002041000061455B7C0A80F10C5A3F86
:107D000000002440872D0020FCA9F1D24D62503F95
:107D1000CDE9060130463946DDE906232FF062FF42
:107D200030D2FA4890F8480004281FDDF84840781F
:107D3000012822D00120F6494870412025F036FB69
:107D4000F24890F88100022803DA0120EF4981F817
:107D50002300EE4890F88100FA280EDAEB4890F8FC
:107D60008100401CE94981F8810006E0E74890F86D
:107D70004800401CE54981F848000020E34981F8AB
:107D80005400DEE040464946DDE906232FF02AFF95
:107D900030D2DE4890F8480004281FDDDC484078E7
:107DA000022822D00220DA494870412025F0FEFA4C
:107DB000D64890F88100022803DA0220D34981F8DE
:107DC0002300D24890F88100FA280EDACF4890F8C4
:107DD0008100401CCD4981F8810006E0CB4890F835
:107DE0004800401CC94981F848000020C74981F873
:107DF0005400A6E0C74890F8E600012866D1504636
:107E00005946DDE906232FF0EDFE30D2BF4890F849
:107E1000480004281FDDBE484078032822D00320F4
:107E2000BB494870412025F0C1FAB84890F881005C
:107E3000022803DA0320B54981F82300B34890F8FB
:107E40008100FA280EDAB14890F88100401CAF4951
:107E500081F8810006E0AD4890F84800401CAB492D
:107E600081F848000020A94981F8540069E0A7483A
:107E700090F8540004281DDDA5484078012804D15D
:107E800041F2410025F092FA10E0A1484078022822
:107E900004D141F2410025F089FA07E09C4840787E
:107EA000032803D141F2410025F080FA00209849CF
:107EB000487006E0954890F85400401C934981F8BA
:107EC00054000020914981F848003AE08F4890F82A
:107ED000540004281DDD8E484078012804D141F269
:107EE000410025F063FA10E089484078022804D167
:107EF00041F2410025F05AFA07E08548407803280E
:107F000003D141F2410025F051FA00208049487028
:107F100006E07E4890F85400401C7C4981F85400EB
:107F200000207A4981F848000BE000207849487029
:107F3000764981F8230081F8810081F8480081F8B2
:107F4000540009B0BDE8F08F2DE9F04F87B000BFB5
:107F500000BF00BF00BF7048007AC0F34000002897
:107F60007ED06B48807A01287BD069484079002810
:107F700077D1684890F8E600012814D1674AD169A2
:107F800090692FF0D2FA01906448016A01982FF0AD
:107F9000CCFA634902902FF052FB03902FF0F7FDCB
:107FA00004460D460EE05D4AD16990692FF0BDFA96
:107FB0004FF0804102902FF042FB03902FF0E7FD3D
:107FC00004460D46554988692FF0E1FD22462B46AF
:107FD000CDE902012FF012FC06460F46002213469F
:107FE000304639462FF0E6FD01D287F000474B4975
:107FF000C8692FF0CCFD22462B46CDE902012FF0B7
:10800000FDFB8046894600221346404649462FF034
:10801000D1FD01D289F000494049086A2FF0B7FD2F
:1080200022462B46CDE902012FF0E8FBCDE9040101
:1080300000221346DDE904012FF0BCFD03D287F0D6
:108040000040CDE9046000221346204629462FF067
:10805000B1FD01D285F000450022324B204601E0FF
:108060003DE148E129462FF0A5FD04D84FF0000A74
:10807000DFF8B4B011E02D4948882FF0C5FC224646
:108080002B46CDE900012FF0BFFB294A294BCDE952
:1080900002012FF0B9FB82468B4652465B463046C2
:1080A00039462FF09FFD47D2184890F84900042820
:1080B0001FDD17488078012822D0012014498870DC
:1080C000422025F073F9114890F88200022803DA63
:1080D00001200E4981F824000C4890F88200FA280B
:1080E0000EDA0A4890F88200401C084981F88200A4
:1080F00006E0064890F84900401C044981F8490010
:108100000020024981F85500F5E000009019002098
:10811000321A00208E220020EA2D0020062E002098
:10812000000040400000F03F00407F40872D0020CD
:10813000FCA9F1D24D62503F52465B46404649464B
:108140002FF050FD30D2FB4890F8490004281FDD85
:10815000F9488078022822D00220F749887042200E
:1081600025F024F9F34890F88200022803DA02206F
:10817000F04981F82400EF4890F88200FA280EDADE
:10818000EC4890F88200401CEA4981F8820006E041
:10819000E84890F84900401CE64981F84900002071
:1081A000E44981F85500A6E0E44890F8E60001288B
:1081B00066D152465B46DDE904012FF013FD30D253
:1081C000DC4890F8490004281FDDDB48807803284C
:1081D00022D00320D8498870422025F0E7F8D548FE
:1081E00090F88200022803DA0320D24981F82400A3
:1081F000D04890F88200FA280EDACE4890F8820033
:10820000401CCC4981F8820006E0CA4890F8490039
:10821000401CC84981F849000020C64981F8550032
:1082200069E0C44890F8550004281DDDC2488078F4
:10823000012804D141F2420025F0B8F810E0BE4810
:108240008078022804D141F2420025F0AFF807E01F
:10825000B9488078032803D141F2420025F0A6F8FE
:108260000020B549887006E0B24890F85500401CDF
:10827000B04981F855000020AE4981F849003AE044
:10828000AC4890F8550004281DDDAB4880780128E3
:1082900004D141F2420025F089F810E0A648807828
:1082A000022804D141F2420025F080F807E0A248FC
:1082B0008078032803D141F2420025F077F80020AE
:1082C0009D49887006E09B4890F85500401C9949EC
:1082D00081F855000020974981F849000BE0002003
:1082E00095498870934981F8240081F8820081F8CB
:1082F000490081F8550007B0BDE8F08F2DE9F04F37
:1083000087B000BF00BF00BF00BF8D48007AC0F338
:10831000800000287ED08848807A01287BD086485B
:108320004079002877D1854890F8E600012814D1DB
:10833000844A916A506A2FF0F8F803908148C16A24
:1083400003982FF0F2F8804904902FF078F9059007
:108350002FF01DFC04460D460EE07A4A916A506AE1
:108360002FF0E3F84FF0804104902FF068F905906A
:108370002FF00DFC04460D467249486A2FF007FCA9
:1083800022462B46CDE904012FF038FA06460F4667
:1083900000221346304639462FF00CFC01D287F0FC
:1083A00000476849886A2FF0F2FB22462B46CDE948
:1083B00004012FF023FA80468946002213464046E6
:1083C00049462FF0F7FB01D289F000495D49C86AA0
:1083D0002FF0DDFB22462B46CDE904012FF00EFAEB
:1083E00082468B4600221346504659462FF0E2FB48
:1083F00001D28BF0004B5349486A54492FF026FCB8
:108400001FD95049486A52492FF02AFC19D35149C3
:10841000888801E068E173E12FF0F6FA22462B46E6
:10842000CDE900012FF0F0F94B4A4C4BCDE90201A8
:108430002FF0EAF932463B46CDE904012FF0BAFBB2
:1084400030D23C4890F84A0004281FDD3A48C078F2
:10845000012822D001203849C870432024F0A6FF0B
:10846000344890F88300022803DA0120314981F86A
:108470002500304890F88300FA280EDA2D4890F84D
:108480008300401C2B4981F8830006E0294890F8BE
:108490004A00401C274981F84A000020254981F8FC
:1084A00056002DE12749886A28492FF0CFFB1CD3BD
:1084B0002449886A26492FF0D3FB16D3254988889A
:1084C0002FF0A2FA22462B46CDE900012FF09CF9AD
:1084D000214A224BCDE902012FF096F942464B4644
:1084E000CDE904012FF066FB46D2124890F84A000D
:1084F000042835DD1048C078022838D002200E4903
:10850000C870432024F052FF0A4890F883000228E4
:1085100003DA0220074981F82500064890F8830015
:10852000FA2824DA034890F88300401C014981F8B6
:1085300083001CE090190020321A00208E220020B7
:10854000EA2D0020062E0020000040400000964347
:108550000000FA43872D0020FCA9F1D24D62503F64
:10856000F74890F84A00401CF54981F84A0000207D
:10857000F34981F85600C3E0F24890F8E60001287C
:1085800076D1F149C86AF1492FF060FB1CD3EE495E
:10859000C86AEF492FF064FB16D3EE4988882FF0A4
:1085A00033FA22462B46CDE900012FF02DF9EA4A95
:1085B000EA4BCDE902012FF027F952465B46CDE99F
:1085C00004012FF0F7FA30D2DD4890F84A00042871
:1085D0001FDDE348C078032822D00320E049C8709B
:1085E000432024F0E3FED64890F88300022803DA03
:1085F0000320D34981F82500D14890F88300FA2858
:108600000EDACF4890F88300401CCD4981F88300F2
:1086100006E0CB4890F84A00401CC94981F84A005E
:108620000020C74981F856006AE0C54890F8560016
:1086300004281EDDCA48C078012804D141F2430055
:1086400024F0B4FE10E0C648C078022804D141F2FC
:10865000430024F0ABFE07E0C148C078032803D1F3
:1086600041F2430024F0A2FE0020BD49C87007E09B
:108670000BE0B34890F85600401CB14981F8560011
:108680000020AF4981F84A003AE0AD4890F8560022
:1086900004281DDDB248C078012804D141F243000E
:1086A00024F084FE10E0AE48C078022804D141F2E4
:1086B000430024F07BFE07E0A948C078032803D1DB
:1086C00041F2430024F072FE0020A549C87006E084
:1086D0009B4890F85600401C994981F856000020AC
:1086E000974981F84A000BE000209D49C8709449E1
:1086F00081F8250081F8830081F84A0081F856004E
:1087000007B0BDE8F08F10B59648007AC0F3C000FE
:10871000002875D09248807A012839D09048407955
:10872000002835D18848008E8A498979884230DD11
:10873000834890F84C0004281FDD8948807901287F
:1087400022D0012086498871442024F02FFE7C48E5
:1087500090F88500022803DA0120794981F8270082
:10876000774890F88500FA280EDA754890F8850069
:10877000401C734981F8850006E0714890F84C0070
:10878000401C6F4981F84C0000206D4981F8580069
:10879000CEE16D48408E6F498979884231DD684865
:1087A00090F84C0004281FDD6D488079022822D003
:1087B00002206B498871442024F0F8FD604890F84D
:1087C0008500022803DA02205D4981F827005C4811
:1087D00090F88500FA280EDA594890F88500401C78
:1087E000574981F8850006E0554890F84C00401C38
:1087F000534981F84C000020514981F8580097E115
:108800008AE15148808E53498979884230DD4C484D
:1088100090F84C0004281FDD51488079032822D0AD
:1088200003204F498871442024F0C0FD444890F84B
:108830008500022803DA0320414981F827004048D7
:1088400090F88500FA280EDA3D4890F88500401C23
:108850003B4981F8850006E0394890F84C00401CFF
:10886000374981F84C000020354981F858005FE114
:108870003548C08E37498979884230DD304890F8D4
:108880004C0004281FDD36488079042822D00420BB
:1088900033498871442024F089FD294890F88500E7
:1088A000022803DA0420264981F82700244890F89A
:1088B0008500FA280EDA224890F88500401C2049ED
:1088C00081F8850006E01E4890F84C00401C1C49C9
:1088D00081F84C0000201A4981F8580028E1194815
:1088E00090F8E600012876D11748008F1949897958
:1088F000884245DD124890F84C00042834DD1848C1
:108900008079052837D0052015498871442024F046
:108910004DFD0B4890F88500022803DA0520084930
:1089200081F82700064890F88500FA2823DA0448E1
:1089300090F88500401C024981F885001BE000008A
:10894000901900208E220020062E00200000964361
:108950000000FA43872D0020FCA9F1D24D62503F60
:10896000321A0020EA2D0020F84890F84C00401CF4
:10897000F64981F84C000020F44981F85800D7E00E
:10898000F348408FF3498979884231DDEF4890F808
:108990004C00042820DDF0488079062823D00620EA
:1089A000ED498871442024F001FDE84890F88500E5
:1089B000022803DA0620E54981F82700E34890F809
:1089C0008500FA280FDAE14890F88500401CDF495D
:1089D00081F8850007E055E0DC4890F84C00401C29
:1089E000DA4981F84C000020D84981F858009FE00E
:1089F000D64890F85800042838DDD74880790128F7
:108A000004D141F2440024F0D1FC2BE0D24880791B
:108A1000022804D141F2440024F0C8FC22E0CE48F0
:108A20008079032804D141F2440024F0BFFC19E00E
:108A3000C9488079042804D141F2440024F0B6FCEE
:108A400010E0C5488079052804D141F2440024F0A3
:108A5000ADFC07E0C0488079062803D141F244000C
:108A600024F0A4FC0020BC49887106E0B74890F8C7
:108A70005800401CB54981F858000020B34981F8DE
:108A80004C0055E0B14890F85800042838DDB24851
:108A90008079012804D141F2440024F087FC2BE0C6
:108AA000AD488079022804D141F2440024F07EFCD4
:108AB00022E0A9488079032804D141F2440024F03F
:108AC00075FC19E0A4488079042804D141F24400DF
:108AD00024F06CFC10E0A0488079052804D141F214
:108AE000440024F063FC07E09B488079062803D10A
:108AF00041F2440024F05AFC00209749887106E0B6
:108B0000924890F85800401C904981F85800002085
:108B10008E4981F84C000BE000208F4988718B4909
:108B200081F8270081F8850081F84C0081F8580011
:108B300010BD10B58948007AC0F34010002879D0E4
:108B40008548807A012841D08348407900283DD16A
:108B50007F4890F854007F49C979884206DC7C48F8
:108B600090F854007B49097A884230DA774890F8C7
:108B70004D0004281FDD7848C079012822D001204B
:108B80007549C871462024F011FC704890F88600A1
:108B9000022803DA01206D4981F828006B4890F81B
:108BA0008600FA280EDA694890F88600401C67496A
:108BB00081F8860006E0654890F84D00401C634946
:108BC00081F84D000020614981F85900ECE16048CE
:108BD00090F855005F49C979884206DC5C4890F8F6
:108BE00055005C49097A884231DA584890F84D00BE
:108BF000042820DD5848C079022823D00220564995
:108C0000C871462024F0D2FB504890F88600022814
:108C100003DA02204D4981F828004C4890F886007C
:108C2000FA280FDA494890F88600401C474981F835
:108C3000860007E0ACE1454890F84D00401C4349F0
:108C400081F84D000020414981F85900ACE14048CD
:108C500090F856003F49C979884206DC3C4890F8B4
:108C600056003C49097A884230DA384890F84D007D
:108C700004281FDD3848C079032822D00320364954
:108C8000C871462024F092FB304890F886000228F4
:108C900003DA03202D4981F828002C4890F886003B
:108CA000FA280EDA294890F88600401C274981F8F6
:108CB000860006E0254890F84D00401C234981F8C5
:108CC0004D000020214981F859006DE1204890F8BD
:108CD00056002049C979884206DC1D4890F85600A4
:108CE0001C49097A88423BDA184890F84D0004285C
:108CF0001FDD1948C079042822D004201649C87104
:108D0000462024F053FB114890F88600022803DA2D
:108D100004200E4981F828000C4890F88600FA28B3
:108D20000EDA0A4890F88600401C084981F886004F
:108D300006E0064890F84D00401C044981F84D00BB
:108D40000020024981F859002EE10000901900200E
:108D5000062E0020872D0020321A0020EA2D002048
:108D6000FE4890F8E600012871D1FD4890F85800BF
:108D7000FC49C979884206DCF94890F85800F9495D
:108D8000097A884230DAF84890F84D0004281FDD4F
:108D9000F648C079052822D00520F449C87146203C
:108DA00024F004FBF04890F88600022803DA05203E
:108DB000ED4981F82800EC4890F88600FA280EDA90
:108DC000E94890F88600401CE74981F8860006E0F3
:108DD000E54890F84D00401CE34981F84D00002023
:108DE000E14981F85900DFE0DD4890F85800DD499D
:108DF000C979884206DCDA4890F85800D949097ADE
:108E0000884231DAD84890F84D00042820DDD74850
:108E1000C079062823D00620D449C871462024F002
:108E2000C5FAD14890F88600022803DA0620CE4918
:108E300081F82800CC4890F88600FA280FDACA4852
:108E400090F88600401CC84981F8860007E055E08C
:108E5000C54890F84D00401CC34981F84D000020E2
:108E6000C14981F859009FE0BF4890F85900042893
:108E700038DDBE48C079012804D141F2460024F013
:108E800095FA2BE0B948C079022804D141F2460096
:108E900024F08CFA22E0B548C079032804D141F2CD
:108EA000460024F083FA19E0B048C079042804D1C0
:108EB00041F2460024F07AFA10E0AC48C079052867
:108EC00004D141F2460024F071FA07E0A748C079C6
:108ED000062803D141F2460024F068FA0020A34995
:108EE000C87106E0A04890F85900401C9E4981F8DE
:108EF000590000209C4981F84D0055E09A4890F8AF
:108F00005900042838DD9948C079012804D141F27C
:108F1000460024F04BFA2BE09448C079022804D193
:108F200041F2460024F042FA22E09048C07903283A
:108F300004D141F2460024F039FA19E08B48C07997
:108F4000042804D141F2460024F030FA10E08748AA
:108F5000C079052804D141F2460024F027FA07E041
:108F60008248C079062803D141F2460024F01EFA57
:108F700000207E49C87106E07B4890F85900401CEB
:108F8000794981F859000020774981F84D000BE0BC
:108F900000207649C871744981F8280081F886005C
:108FA00081F84D0081F8590010BD2DE9F0410024F1
:108FB0006F48007AC0F38010002871D06B48807A27
:108FC00001286ED06948407900286AD1644D3C354B
:108FD000624890F8E600012814D195F800802E78B8
:108FE000002701240BE0285D404501DA15F80480D4
:108FF000285DB04201DD2E5D2746601CC4B2062C00
:10900000F1DB13E095F800802E78002701240BE0B7
:10901000285D404501DA15F80480285DB04201DD85
:109020002E5D2746601CC4B2042CF1DBA6EB0800C1
:109030004C49497A88427DDD002F7CD1484890F820
:109040004200142843DA2A2E41DB4948007A0121E4
:10905000B1EBD01F32D1444890F852000B2821DDEB
:1090600042480079012824D001204049087140205D
:1090700024F09CF93C4890F88900022803DA01208A
:10908000394981F82B00384890F88900FA2810DA1D
:10909000354890F88900401C334981F8890008E080
:1090A000F4E34FE2304890F85200401C2E4981F81A
:1090B000520000202C4981F85E0043E200202B4939
:1090C0000871294981F8520081F85E00F5E72648C9
:1090D00090F85E0004280EDD24480079012803D1B1
:1090E0004FF4825024F062F90020204908711E4993
:1090F00081F82B0006E01C4890F85E00401C1A49DD
:1091000081F85E000020184981F85200084690F866
:109110004E0004282EDD1548007A012831D00120A8
:1091200012490872472024F041F90F4890F887004F
:10913000022801E050E329E003DA01200A4981F81E
:109140002900094890F88700FA281ADA064890F8AA
:109150008700401C044981F8870012E08E2200201D
:10916000062E0020872D002090190020321A0020A2
:10917000EA2D0020FE4890F84E00401CFC4981F882
:109180004E000020FA4981F85A00D6E3012F7CD125
:10919000F84890F84300142841DA2A2E3FDBF648BD
:1091A000007AC0F3400080B3F14890F852000B28D9
:1091B0001FDDF2480079022822D00220EF49087111
:1091C000402024F0F3F8EA4890F88900022803DAF6
:1091D0000220E74981F82B00E54890F88900FA2839
:1091E0000EDAE34890F88900401CE14981F88900D3
:1091F00006E0DF4890F85200401CDD4981F852003B
:109200000020DB4981F85E0097E3FFE70020DB499F
:109210000871D74981F8520081F85E008DE3D44887
:1092200090F85E0004280EDDD4480079022803D1AE
:109230004FF4825024F0BAF80020D0490871CC498C
:1092400081F82B0006E0CA4890F85E00401CC8492F
:1092500081F85E000020C64981F85200084690F867
:109260004E00042821DDC548007A022824D00220BF
:10927000C2490872472024F099F8BD4890F8870049
:10928000022805DA0220BA4900E01AE081F8290034
:10929000B74890F88700FA280EDAB54890F88700AA
:1092A000401CB34981F8870006E0B14890F84E00B1
:1092B000401CAF4981F84E000020AD4981F85A00AA
:1092C0003BE3022F7ED1AB4890F84400142847DAE4
:1092D0002A2E45DBA848007A0121B1EBD01F36D1F8
:1092E000A34890F852000B2825DDA44800790328F4
:1092F00028D00320A1490871522024F057F89E4835
:10930000007A0121B1EBD01F1CD1994890F8890057
:10931000022803DA0320964981F82B00944890F83C
:109320008900FA280EDA924890F88900401C90498A
:1093300081F8890006E08E4890F85200401C8C4964
:1093400081F8520000208A4981F85E00F5E2002091
:109350008A490871864981F8520081F85E00ECE282
:10936000834890F85E0004280EDD844800790328C5
:1093700003D141F2520024F019F800207F4908710E
:109380007B4981F82B0006E0794890F85E00401C8C
:10939000774981F85E000020754981F8520008463F
:1093A00090F84E00042821DD7448007A032824D068
:1093B000032072490872472023F0F8FF6C4890F8A8
:1093C000870000E01EE0022803DA0320684981F8E4
:1093D0002900674890F88700FA280EDA644890F868
:1093E0008700401C624981F8870006E0604890F8D9
:1093F0004E00401C5E4981F84E0000205C4981F817
:109400005A009AE2032F7CD15A4890F8450014285C
:1094100047DA2A2E45DB5848007A0121B1EBD01FEC
:1094200036D1534890F852000B2825DD5348007977
:10943000042828D0042051490871402023F0B6FFA9
:109440004D48007A0121B1EBD01F1CD1484890F85B
:109450008900022803DA0420454981F82B0044489A
:1094600090F88900FA280EDA414890F88900401CEB
:109470003F4981F8890006E03D4890F85200401CC1
:109480003B4981F852000020394981F85E0054E2DE
:1094900000203A490871364981F8520081F85E008F
:1094A0004BE2334890F85E0004280EDD3348007923
:1094B000042803D141F2520023F078FF00202F4905
:1094C00008712B4981F82B0006E0294890F85E00CE
:1094D000401C274981F85E000020254981F8520090
:1094E000084690F84E00042821DD2448007A04281C
:1094F00024D0042021490872472023F057FF1C483C
:1095000000E020E090F88700022803DA04201849E0
:1095100081F82900164890F88700FA280EDA1448D6
:1095200090F88700401C124981F8870006E0104837
:1095300090F84E00401C0E4981F84E0000200C4966
:1095400081F85A00F9E1042F7ED10A4890F84600CC
:10955000142850DA2A2E4EDB0748007A0121B1EB9D
:10956000D01F3FD1024890F852000B282EDD07E0B3
:1095700090190020062E0020EA2D0020321A00202B
:10958000FE480079052828D00520FC4908714020B4
:1095900023F00CFFFA48007A0121B1EBD01F1CD157
:1095A000F84890F88900022803DA0520F54981F887
:1095B0002B00F44890F88900FA280EDAF14890F868
:1095C0008900401CEF4981F8890006E0ED4890F8D9
:1095D0005200401CEB4981F852000020E94981F813
:1095E0005E00AAE10020E5490871E64981F85200D1
:1095F00081F85E00A1E1E34890F85E0004280EDDEA
:10960000DE480079052803D14FF4825023F0CEFEC6
:109610000020DA490871DB4981F82B0006E0D948BF
:1096200090F85E00401CD74981F85E000020D549C3
:1096300081F85200084690F84E00042821DDCF48FA
:10964000007A052824D000E027E00520CB490872E5
:10965000472023F0ABFECB4890F88700022803DABE
:109660000520C84981F82900C64890F88700FA28E3
:109670000EDAC44890F88700401CC24981F8870080
:1096800006E0C04890F84E00401CBE4981F84E00EC
:109690000020BC4981F85A004FE1052FA1D1BA48FA
:1096A00090F84700142847DA2A2E45DBB448007AA0
:1096B0000121B1EBD01F36D1B24890F852000B28EF
:1096C00025DDAE480079062828D00620AB49087170
:1096D000402023F06BFEAA48007A0121B1EBD01F95
:1096E0001CD1A84890F88900022803DA0620A54971
:1096F00081F82B00A34890F88900FA280EDAA148D7
:1097000090F88900401C9F4981F8890006E09D4837
:1097100090F85200401C9B4981F852000020994962
:1097200081F85E0009E1002094490871954981F8AB
:10973000520081F85E0000E1924890F85E00042833
:109740000EDD8E480079062803D14FF4825023F0B5
:109750002DFE0020894908718A4981F82B0006E016
:10976000884890F85E00401C864981F85E00002021
:10977000844981F85200084690F84E0004281FDD05
:109780007E48007A062822D006207C4908724720AD
:1097900023F00CFE7B4890F88700022803DA0620AD
:1097A000784981F82900774890F88700FA280EDA7E
:1097B000744890F88700401C724981F8870006E0E1
:1097C000704890F84E00401C6E4981F84E00002011
:1097D0006C4981F85A00B0E06A4890F85A000428B1
:1097E0003BDD6648007A012804D141F2470023F0AE
:1097F000DDFD2BE06148007A022804D141F24700E8
:1098000023F0D4FD22E05D48007A032804D141F220
:10981000470023F0CBFD19E05848007A042804D112
:1098200041F2470023F0C2FD10E05448007A0528B9
:1098300004D141F2470023F0B9FD07E04F48007A18
:10984000062803D141F2470023F0B0FD00204B4928
:1098500008724C4981F8290006E04A4890F85A00FD
:10986000401C484981F85A000020464981F84E00C2
:10987000084690F85E0004283CDD40480079012845
:1098800005D14FF4825023F091FD2CE03EE03B489F
:109890000079022804D14FF4825023F087FD22E0A2
:1098A00036480079032804D141F2520023F07EFDAE
:1098B00019E032480079042804D141F2520023F023
:1098C00075FD10E02D480079052804D14FF4825031
:1098D00023F06CFD07E029480079062803D14FF4F6
:1098E000825023F063FD002024490871254981F846
:1098F0002B0006E0234890F85E00401C214981F8C7
:109900005E0000201F4981F8520016E000201B492C
:1099100008721C4981F8290081F8870081F84E00FF
:1099200081F85A0015490871164981F82B0081F811
:10993000890081F8520081F85E00BDE8F08110B521
:1099400004460E48407900287ED10D48407AC0F385
:10995000001000282FD009480079012803D00748BB
:109960000079022828D104200449487104F0040039
:10997000042871D0522023F019FD07E0321A00208C
:10998000EA2D002090190020062E0020FE4890F8B5
:109990008400022803DA0120FB4981F82600FA48F6
:1099A00090F88400FA2857DAF74890F88400401CB1
:1099B000F54981F884004FE0F4480079032803D08A
:1099C000F248007904281FD10220F049487104F0C0
:1099D0000200022840D0522023F0E8FCEA4890F828
:1099E0008400022803DA0220E74981F82600E648CD
:1099F00090F88400FA282FDAE34890F88400401C9D
:109A0000E14981F8840027E0E0480079052803D087
:109A1000DE48007906281FD10120DC49487104F096
:109A20000100C8B9522023F0C1FCD74890F8840047
:109A3000022803DA0320D44981F82600D24890F89E
:109A40008400FA2808DA00E02EE0CF4890F884007D
:109A5000401CCD4981F8840004F00400042809D199
:109A6000CA48407900F00400042803D041F25200B3
:109A700023F09CFC04F00200022809D1C34840797D
:109A800000F00200022803D041F2520023F08EFCC5
:109A900004F0010040B1BD48407900F0010018B960
:109AA00041F2520023F082FC10BD08B50020009066
:109AB000FDF723FF6846FDF785FFFFF776FA9DF86F
:109AC0000000FFF73CFFFEF718F8FEF73DFAFEF73F
:109AD00015FCFEF718FEFFF72CF808BD2DE9F04144
:109AE000AB4890F8E600012871D1A848407900F011
:109AF000010030B3A74A916A506A2DF016FD8046E6
:109B00002EF045F806460022A34B2DF07DFE0446BC
:109B10002EF080F89E49C1F8B5009E4AD16C906C39
:109B20002DF003FD80462EF032F8064600229A4BB7
:109B30002DF06AFE04462EF06DF89549C1F8B90083
:109B40008BE09248407900F00400042809D1914844
:109B5000C06A8F49C1F8B5008E48006DC1F8B900E0
:109B60007BE08A48407900F00200022809D1894848
:109B7000C06A8749C1F8B5008648006DC1F8B900D0
:109B80006BE0844A916A506A2DF0CFFC054681480B
:109B9000C16A28462DF0C9FC044680492DF04FFDCE
:109BA0007B49C1F8B5007B4AD16C906C2DF0BDFCAF
:109BB00005467848016D28462DF0B7FC04467749E4
:109BC0002DF03DFD7249C1F8B90046E0FFE76F484E
:109BD000407900F00400042809D16E48806A6C497D
